:020000040800F2
:10000000F0FF0010751E070871F80008B11605080A
:10001000151F0708151F0708151F07080000000017
:100020000000000000000000000000006DF8000863
:1000300069F800080000000065F8000849DA0408C3
:10004000151F0708151F0708151F0708151F0708A4
:10005000151F0708151F07089D2E0508652E0508A2
:100060002D2E0508F52D0508BD2D0508A9CD06087E
:1000700099CD060889CD060879CD060865CD060814
:1000800051CD06083DCD0608151F0708151F0708A6
:10009000151F0708151F0708151F0708852D0508D8
:1000A00025C00408A5C0040815C00408C9C0040878
:1000B00099C0040889C0040879C00408A50A070883
:1000C000AD0A0708990A0708A10A0708151F0708BB
:1000D000151F070859DE04089DDD0408E1DC04084B
:1000E0004D2D0508151F07082911010805C0040832
:1000F00035C00408F5BF040859C0040829CD060816
:10010000151F070841AA060869C00408151F07083B
:1001100025DC040869DB0408D1080408BD080408CC
:1001200015CD060801CD0608EDCC0608D9CC060889
:10013000C5CC0608151F0708151F0708151F070857
:10014000151F0708151F0708151F0708F1F10008FC
:10015000B1CC06089DCC060889CC0608ADDA0408A7
:100160008D0A0708950A0708151F0708151F0708B5
:10017000151F0708151F0708151F0708151F070873
:08018000151F0708151F0708F1
:0828000000C00F0800001008E1
:10800000F0B401292A4C2B4D23684FF0000694BF91
:1080100000270127EE626662A6626763676B47EA24
:1080200042076763EE63EC6B002A38D144F4957421
:10803000EC631C6824F001041C601C68E407FCD499
:10804000490289085960D8601968EAB921F04001ED
:10805000196019498B421DD018494FF47410C8603B
:10806000196841F01E011960596941F08001596198
:10807000196841F00101196022B90E4AD36A43F030
:108080000803D362F0BC704741F0400119600A490F
:108090008B42E1D14FF0746041F8500CE0E744F0BE
:1080A0001A04EC63EC6A44F00804EC62C1E700BF18
:1080B000281E0020002C0140586402400064024049
:1080C0001148002302461178032902F1060216D056
:1080D0000133062BF7D10D4AD36D052B0ED0591C59
:1080E00003EB4303D16500EB4303032040F2EB3184
:1080F00040F2FF32187059809A807047704703EB46
:10810000430300EB4303F0E7601E0020281E00201D
:1081100070B4C3080D4CE25C00F00706B24004EBFB
:10812000D004D2B20020C6F108038B4228BF0B4610
:10813000C3F108052A419840C91A40EA02004FF0ED
:10814000000614F8012FEED170BC7047C81E002045
:10815000084AD2E9553199420AD0D118013391F831
:108160005C110170C3F30A03C2F854310120704757
:1081700000207047281E0020064AD2F85C39D2F849
:108180006029934294BF4FF400600020013B9B1A8A
:1081900018447047281E0020012380F85130704792
:1081A00007B501A8FFF7D4FF0028FAD09DF8040016
:1081B00003B05DF804FB044BD3E95503984288BF34
:1081C00003F50063181A7047281E0020012070472D
:1081D000024BC3F86429C3F868197047281E0020B1
:1081E000024BC3F86C29C3F870197047281E002091
:1081F0007047704730B4134DD5E955239A4286BF76
:1082000003F50064A21A9A1A0A44B2F5006F13D853
:10821000A9B101444A1E013810F8014FE918824201
:1082200003F1010381F85C41C3F30A03F4D1C5F8FB
:108230005831002030BC7047022030BC70470846DF
:10824000F8E700BF281E0020F8B51A4C94F87439DE
:10825000002BFBD159B301444E1E451ED4F86029B2
:10826000D4F85C1915F8017F531CC3F30A038B4241
:108270002CBF4FF400600020C91A22440144012998
:1082800082F87879C4F860390FD1012045F038FBC5
:10829000D4F85C39D4F860198B4294BF4FF4006273
:1082A00000225B1A1344012BEFD0B542D6D1002037
:1082B000F8BD00BF281E002010B590F85010002314
:1082C00080F8503081B10B4CD4F8802072B1D4F8D2
:1082D0008020052A0CD13C30D4F88430FFF7B4FF5D
:1082E000D4F88430012010BD0120FCE71046FAE7E5
:1082F0001846F8E7202F0020002280F85120DBE705
:1083000090F85020531C0244DBB280F8503082F8C1
:108310003C1090F851200AB1132B00D9CCE77047DC
:1083200010B5094CD4F88030084611465BB1D4F83A
:108330008030052B07D1002AD4F8843003DDFFF705
:1083400083FFD4F8843010BD202F0020212838B5B9
:108350000C4605D022282FD0202813D0002038BD6D
:108360000029FBD0072AF9D11A4BD3F8880093F8DB
:108370008C1093F88D2093F88E30206021716271FB
:10838000A371EBE70029E9D0072AE7D1124AD2F816
:1083900068391BB1D2F86409096898470D4B256804
:1083A00020796179A279C3F8885083F88C0083F82A
:1083B0008D1083F88E20D1E70029CFD0022ACDD1AD
:1083C000054AD2F87039002BC8D00988D2F86C0958
:1083D0009847C3E7202F0020281E0020024B0020D2
:1083E000C3F88000704700BF202F0020054B064ACD
:1083F00000200521C2F88010C3F87009C3F868098D
:10840000704700BF281E0020202F0020704700BFAB
:10841000704700BF704700BF704700BF704700BF84
:10842000704700BF704700BF042301480B807047AE
:108430008801002010B4074A074B92F890001224DC
:1084400003F114020C8001280CBF184610465DF899
:10845000044B7047202F00208C01002000487047FB
:10846000B01E002000487047B01E0020034B93F858
:108470008400032894BF002001207047281E00209C
:10848000034B93F88400032894BF00200120704719
:10849000281E0020034B93F88400003818BF0120E9
:1084A000704700BF281E0020A0B182680D4B12B19A
:1084B00007229A7070471978DA6003294FF0040098
:1084C0000CBF80214FF48071C3E901111A611A7544
:1084D00098707047034B41F2E47101225A545A706C
:1084E000704700BF94A000200378022B10D00069D1
:1084F00008B9012070470C4B1B78032B0EBF0B4BA8
:1085000080B24FF6F773984294BF00200120704765
:108510000549436841F650028A58B3EB422F2CBFFD
:1085200001200020704700BF94A00020F7FFFF0F3C
:108530000378022B14D030B4104A4368006941F626
:10854000480402F5C2511559096841F63C042B4014
:1085500012595B0A023801FB0030104430BC7047EE
:10856000064B426841F6340141F63000595818581C
:1085700000EB410000EB5220704700BF94A00020A8
:108580002DE9F84F494B98420ED003F56853083354
:1085900098424ED0464B0020C3E94000A3F8FC00AF
:1085A000A3F80801BDE8F88F414C424FDFF8108175
:1085B0000223C4F8943004F198060025FB6AAB420C
:1085C000294605F1010503D0D4F8180159F0B8FA8D
:1085D00094F81C31D4F8182186F8243032623046E1
:1085E000414659F0C1FCD4F894309D4206F1300662
:1085F000E4DB002384F80A31D4E92803D4F894108A
:10860000B4F89C20B4F8A850C4F8283112FB01F249
:1086100003FB01F3A4F8FC20B4F89E10264AA4F84A
:108620000851C4E94003A4F8FE10C4F8F820012062
:10863000B8E71F4C1F4F0223C4F8943004F198058B
:108640004FF0000B4FF4806A4FF040094FF4006880
:10865000FA6A01265A455946B34403D0D4F81801A2
:1086600059F06EFAD4F8181194F81C21296285F893
:1086700024204FF400314FF00062C5E90212A5F842
:1086800004A0A5F81090A5F80680AE74FFF718FDB9
:1086900028466E7659F0B4FBD4F89420074B45F881
:1086A000303B9345D4DB84F80A61A5E71971EF00EC
:1086B000202F002088010020D8460708AC46070874
:1086C0001940EF002DE9F04FD84DDFF89083DFF827
:1086D0009CA307460E4693460FCD44462DED068BD0
:1086E0000FC40FCD0FC495E8070089B09AF82E315A
:1086F000CDF808B084E80700CDE90476042B00F239
:108700006781DFE813F0D201650160010500E20135
:108710009FEDC78ADFEDC78AC749C8F81C10C74953
:10872000C74BC84AC8F818100299002918BF134649
:1087300038EE887AF5EE006A86EE87AAC24EDFF838
:1087400030B3C8F824300025DFEDC07A9FEDC09A21
:1087500028EE278AF0EE679A059BAB4200F02D8148
:108760001BF8013B0AEB030292F83341002C00F0A6
:108770003481DFF800C3002202E0152A00F02D81C9
:1087800002EB420157001CF80100A04202F1010275
:10879000F3D1514491F85111002900F08481204611
:1087A000039343F0A1FF039B81464846039343F0A4
:1087B000BBFF0178002940F01081039B574401332F
:1087C000DBB2032287F8913187F89021B9F1000FCD
:1087D00000F003812709013F052F04F00F0000F28C
:1087E0004D819C4C04EB4701B1F884C04CFA00F178
:1087F00011F0010100F04281012101FA00F001387D
:1088000000EA0C002744039369F066F997F890702A
:10881000DFF864C2039B38440CEBC0070322FB71F2
:10882000BA715CF83000776100F13F4303F57E03D5
:1088300004EB9324012194F8983099F8082003F070
:108840001F045B09032B01FA04F100F01D81042BC6
:1088500000F02481022B00F01C81BB880693B3FA40
:1088600083F3C3F11F03C3F3CC0100EB810103F0D9
:1088700007030C6A9B000F279F4024EA07040C6241
:108880000C6A02FA03F323430B62022306A907933F
:108890000CF09EFE029B002B00F0AE80BAF82C314B
:1088A00000EE103AB8EEC00AFCEEC07A17EE901A4D
:1088B000D9F80030684A934200F09B80A2F58062AC
:1088C000934200F0968002F58042934200F091803E
:1088D00002F58062934200F08C8002F58062934240
:1088E00000F08780DAF8BC2450084FF6FF73B0FB25
:1088F000F1F21A44120CB0FBF2F20298002800F0D8
:108900008480B2FBF1F19AF82E0104288BB200F0BA
:10891000828007EE902AF8EE676A66EE887A29EE82
:10892000677A9AF82F0104990091A8EEA67A01902F
:1089300049463046C6ED027A86ED037A37F0B0FC40
:10894000002D40F39D807368D8F83820934200F0E2
:108950009980012D00F09480D8F85020934200F0C7
:108960009180022D00F08C80D8F86820934200F0AE
:108970008980032D00F08480D8F88020934200F095
:108980008180042D7CD0D8F8982093427AD0052D90
:1089900076D0D8F8B020934274D0062D70D0D8F895
:1089A000C820D31A18BF012301350122082D3374C2
:1089B000727406F118067FF4CFAE284809B0BDECFA
:1089C000068BBDE8F08F9FED268AF0EE488AA3E67D
:1089D0009FED248AF0EE488A9EE6234A194BC8F898
:1089E0001C200020C8F8243009B0BDEC068BBDE87F
:1089F000F08FDAF8BC0478E7B0EE4A0A6AF072FA4F
:108A0000FCEEC07A17EE901A52E79AF82E0104286D
:108A100019467FF47EAF07EE901A07EE102AF8EEA3
:108A2000677AF8EE476A67EEA97A78E7044707089D
:108A3000ACC5A737ACC5A736F1CB030849A60408D7
:108A400085C603083DA604083C0000106F12833A57
:108A500000007A44AC4607080004014008000010FA
:108A6000282930386F1203397DC90308202F0020D0
:108A70005E30002070300020DC300020716109E79A
:108A8000012391E700238FE7114B1C6C21431964EC
:108A9000E3E60F4B5C6C21435964DEE60C4B1C6B28
:108AA00021431963D9E689467FE69FED0A8A0A4B7E
:108AB000C8F818300023094A049301230293C8F828
:108AC0001C20074BF0EE488A32E69FED068AEEE75F
:108AD000003802406F12833A49A60408F1CB03081C
:108AE0003DA6040800000000F8B5104ED6F8BC44BE
:108AF000054600680F4664080CF06EFCB4FBF7F105
:108B0000B1F5803F03D3012CFAD96408F6E7224679
:108B1000284689B243F09CFB054BC6F8243D284605
:108B20000449BDE8F840002243F0D6BA202F0020C7
:108B3000B93F0208443C002010B5044C04480A46E2
:108B400021460BF08BFA204610BD00BF4C3C0020A4
:108B500078E0070810B5044C04480A4621460BF09B
:108B60007DFA204610BD00BF4C3C002088E007087D
:108B700010B5044C04480A4621460BF06FFA204613
:108B800010BD00BF4C3C002094E0070810B5044C19
:108B900004480A4621460BF061FA204610BD00BF8A
:108BA0004C3C0020A0E0070810B5044C04480A46DD
:108BB00021460BF053FA204610BD00BF4C3C00206C
:108BC000ACE0070810B50D4C94F852210023C4F80E
:108BD000803012B10A4AC2F82C3E61F091FF20B1F8
:108BE0000423022084F8843010BD054BD3F8843070
:108BF0006367092384F8843010BD00BF281E00205D
:108C0000202F002070B50D4D95F88430042B0446BC
:108C10000E460AD0082B06D1EB6F83420CD0FFF72B
:108C2000D1FF022801D0012070BD0823C5E91F46ED
:108C300085F88430022070BD022070BD281E0020FF
:108C400070B50379234C002B14BF0123002384F853
:108C5000B03003D1002384F8843070BD1E4D002154
:108C600095F9332E032045F029FB0028F2D0466801
:108C7000304645F011FB84F851010028EAD095F800
:108C8000313E003B18BF0123304684F8523162F078
:108C9000C5FE0BF091F938B994F8783084F8840067
:108CA000013384F8783070BD62F014F840B194F864
:108CB00078300022013384F8783084F8842070BD45
:108CC000D5F884306367012384F8780084F8843011
:108CD00070BD00BF281E0020202F002010B561F0BD
:108CE000F9FF58B10C4C94F878300133DBB2072B04
:108CF00084F8783003D9002384F8843010BD0BF059
:108D00005BF90028F7D0054A0123D2F88420626776
:108D100084F8843010BD00BF281E0020202F0020C2
:108D20002DE9F041884C94F8B050002D00F0FA8005
:108D300094F88420854E0227531E082B41D8DFE883
:108D400003F03739A0406A511540050061F0D8FEA4
:108D5000002840F0EE80636FD6F88420FA33934207
:108D60002CD2FFF7BBFF94F88420E5E761F0C8FE42
:108D70000028F0D0D4F880300022012B84F878202D
:108D800040F2DB80E16F94F85201013B0131C4E90C
:108D90001F1310B16D4BC3F82C2E082284F88420C9
:108DA000A2F10805B5FA85F56D092846BDE8F08100
:108DB00084F8847061F0A4FE002843D194F88420E4
:108DC000531EDBB2022B0AD8604B616FD3F884309C
:108DD0005B1AC82BE4D9FFF781FF94F88420042A9A
:108DE000DED1E2E7236B002BDAD1584BE66ED3F8E5
:108DF00084306367072284F88420002ED0D0D4E921
:108E00001821236F0120B047D8E7636FD6F884108C
:108E100064338B42C4D2D4F82C80B8F1000FF4D163
:108E200061F06EFE00289ED0E66E84F87880042300
:108E300084F88430002E7AD0D4E91821236F40467C
:108E4000B047BBE761F002FB0028B7D196F8353E8A
:108E5000002BA3F10203B3FA83F314BF0222012211
:108E60005B0984F8792084F87A3061F0EFFA002801
:108E70007FF477AF364A0323926CC4F8882084F8D5
:108E8000843061F0E3FA002898D1304BC4F88000B8
:108E900093F8646EB3F8660ED3F868EED3F868CE34
:108EA000D3F8687ED3F8682E84F88E6093F86C1E31
:108EB000A4F88C0093F86D6E84F8922093F86D0EF0
:108EC000D3F8702EC4F89420B3F8768EB3F8762ECB
:108ED00084F89310B3F8761EC2F30B1343EA1823F9
:108EE00003F00F0301F00F024FEA1E6E4FEA1C4C15
:108EF0003F0A360900F00F0003F5FA63042184F8F5
:108F0000990084F88FE084F890C084F8917084F818
:108F10009860A4F89A3084F89C2084F8841028463D
:108F2000BDE8F08184F884502846BDE8F08105460C
:108F30003BE7042384F8843037E7FAD1FFF742FE99
:108F400094F88420531E3CE7281E0020202F002088
:108F5000583D00202DE9F84FBA4C94F8901E054674
:108F6000C1F34001D4F8980E48F080FB94F8901EAD
:108F7000D4F8940EC94301F0010148F077FB002DAD
:108F800000F0CD806E1EB04FB04D5FFA86FB4FF003
:108F90001008D4F8980E48F0CFF9D4F8940E48F0A1
:108FA000CBF9B4F8A03E002B40F0438194F8A21E08
:108FB000D4F8A40E48F05AFB4FF0FA094FF47A7037
:108FC0004FF0010C7B68C3F30803002B40F00881CD
:108FD000EFF31183002B40F00381D4F88420A968BB
:108FE000D4F884309A42F8D1D4F8C83E9942F4D8E3
:108FF000D4F8C46E00FB06F35B1AB3FBF6F300FB78
:1090000002327B68C3F30803002B40F0A880EFF323
:109010001183002B40F0A380D4F88430D5F808A049
:10902000D4F884108B42F7D1D4F8C81E8A45F3D8FF
:10903000D4F8C46E00FB06F1A1EB0A01B1FBF6F116
:1090400000FB03139B1AB3F57A7FDAD3B9F1010958
:10905000B8D1D4F8980E48F06FF9D4F8940E48F0CF
:109060006BF9B4F8A03E002B40F0D78094F8A21E14
:10907000D4F8A40E81F0010148F0F8FA4FF0FA0C90
:109080004FF47A704FF0010E7B68C3F30803002B96
:1090900040F08680EFF31183002B40F08180D4F8FC
:1090A0008420A968D4F884309A42F8D1D4F8C83E14
:1090B0009942F4D8D4F8C49E00FB09F35B1AB3FBC1
:1090C000F9F300FB02327B68C3F308034BBBEFF3F9
:1090D000118333BBD4F88430D5F808A0D4F88410B9
:1090E0008B42F7D1D4F8C81E8A45F3D8D4F8C49E71
:1090F00000FB09F1A1EB0A01B1FBF9F100FB03133D
:109100009B1AB3F57A7FDED3BCF1010CBCD10BF115
:10911000FF365FFA86FBBBF1FF0F7FF43AAFBDE885
:10912000F88FEFF3118988F31288AE682B68DB03A0
:1091300044BFC4F8C0EEAE68D4F88430D4F8C01E82
:109140005FFA89F989F31188D4F8C49E0B4400FBB7
:1091500009F1891BB1FBF9F100FB0313D0E7EFF331
:10916000118E88F31288D5F808A02B68D90344BF64
:10917000C4F8C0CED5F808A0D4F88430D4F8C01E06
:109180005FFA8EFE8EF31188D4F8C46E0B4400FB98
:1091900006F1A1EB0A01B1FBF6F100FB031351E765
:1091A000EFF3118188F31288D5F808902B68DA0361
:1091B00044BFC4F8C0EED5F80890D4F88430D4F891
:1091C000C02EC9B281F31188D4F8C41E1A4400FB22
:1091D00001F3A3EB0903B3FBF1F300FB023272E7E7
:1091E000EFF3118188F31288AE682B68DB0344BF6C
:1091F000C4F8C0CEAE68D4F88430D4F8C02EC9B25A
:1092000081F31188D4F8C41E1A4400FB01F39B1BA0
:10921000B3FBF1F300FB0232F3E6D4F8BC3E002BC3
:109220003FF42CAFD4F8A83EC3F8009084F8B99E60
:1092300024E7D4F8BC3E002B3FF4BEAE44F024FC3F
:10924000BAE600BF202F002000ED00E010E000E0B3
:109250002DE9F84FB74CB84F94F8901ED4F8980EFB
:10926000B64DC1F3400148F001FA94F8901ED4F8CD
:10927000940EC94301F0010148F0F8F94FF0050BD5
:109280004FF01008D4F8980E48F056F8D4F8940E21
:1092900048F052F8B4F8A03E002B40F0438194F817
:1092A000A21ED4F8A40E48F0E1F932264FF47A70E9
:1092B0004FF0010C7B68C3F30803002B40F00781DB
:1092C000EFF31183002B40F00281D4F88420A968C9
:1092D000D4F884309A42F8D1D4F8C83E9942F4D8F0
:1092E000D4F8C4EE00FB0EF35B1AB3FBFEF300FBF5
:1092F00002327B68C3F30803002B40F0A780EFF332
:109300001183002B40F0A280D4F88430D5F808A057
:10931000D4F884108B42F7D1D4F8C81E8A45F3D80C
:10932000D4F8C4EE00FB0EF1A1EB0A01B1FBFEF193
:1093300000FB03139B1AB3F57A7FDAD3013EB9D150
:10934000D4F8980E47F0F8FFD4F8940E47F0F4FFE5
:10935000B4F8A03E002B40F0DA8094F8A21ED4F8B6
:10936000A40E81F0010148F081F94FF0320C4FF466
:109370007A7001267B68C3F30803002B40F08780D6
:10938000EFF31183002B40F08280D4F88420A96889
:10939000D4F884309A42F8D1D4F8C83E9942F4D82F
:1093A000D4F8C49E00FB09F35B1AB3FBF9F300FB8E
:1093B00002327B68C3F308033BBBEFF3118323BB8B
:1093C000D4F88430D5F808A0D4F884108B42F7D1B3
:1093D000D4F8C81E8A45F3D8D4F8C49E00FB09F11E
:1093E000A1EB0A01B1FBF9F100FB03139B1AB3F5E2
:1093F0007A7FDED3BCF1010CBCD10BF1FF3616F045
:10940000FF0B7FF43FAFBDE8F88FEFF3118988F3CE
:109410001288D5F808A02B68DB0344BFC4F8C06EDF
:10942000D5F808A0D4F88430D4F8C01E5FFA89F9C2
:1094300089F31188D4F8C49E0B4400FB09F1A1EB19
:109440000A01B1FBF9F100FB0313CFE7EFF3118E33
:1094500088F31288D5F808A02B68D90344BFC4F854
:10946000C0CED5F808A0D4F88430D4F8C01E5FFA76
:109470008EFE8EF31188D4F8C4EE0B4400FB0EF17F
:10948000A1EB0A01B1FBFEF100FB031352E7EFF37E
:10949000118188F31288D5F808902B68DA0344BF4D
:1094A000C4F8C06ED5F80890D4F88430D4F8C02E33
:1094B000C9B281F31188D4F8C41E1A4400FB01F329
:1094C000A3EB0903B3FBF1F300FB023271E7EFF307
:1094D000118188F31288D5F808E02B68DB0344BFBC
:1094E000C4F8C0CED5F808E0D4F88430D4F8C02E43
:1094F000C9B281F31188D4F8C41E1A4400FB01F3E9
:10950000A3EB0E03B3FBF1F300FB0232F1E6D4F858
:10951000BC3E002B3FF429AFD4F8A83E1E6084F86F
:10952000B96E22E7D4F8BC3E002B3FF4BEAE44F047
:10953000ABFABAE6202F002000ED00E010E000E0DA
:1095400000F01F0240090123032803FA02F304D0AC
:1095500004280CD0022805D07047074A116C0B4331
:1095600013647047044A516C0B4353647047024ABA
:10957000116B0B43136370470038024000285FD023
:109580000368374A2DE9F04103F13F4404F57E04B6
:1095900002EB9422012492F8982002F01F05520950
:1095A000032A04FA05F456D0042A4FD0022A48D0E0
:1095B0008588B5FA85F0C0F11F00C0F3CC0603EB37
:1095C000860600F0070082000F24306A944020EAEB
:1095D00004003062306A01FA02F202430021326272
:1095E0004FF0010E0A464FF0030C02270EFA02F864
:1095F00038EA050002F101021CD118680CFA01F4E6
:1096000020EA04001860186807FA01F606431E6095
:109610009E6826EA04069E6098689860586820EA6A
:109620000800586058685860D86820EA0400D8607C
:10963000D868D860102A01F10201D7D1BDE8F081C5
:109640007047084A556C2C435464B1E7054A156BC2
:109650002C431463ACE7034A156C2C431464A7E74E
:10966000AC46070800380240134B0268196821EA2B
:1096700002011960596821EA0201596019680A4318
:109680001A609968026821EA02019960D96821EAA2
:109690000201D9604179102907D001F1804303F517
:1096A0009E3319680A431A6070479968114399609C
:1096B000D9680A43DA607047003C014000286BD04B
:1096C000F0B58388B3FA83F3202B85B00446C3F149
:1096D0001F024CD0314D32484FF00041104405EB91
:1096E000820205F60C7731FA03F390F8A060C2F815
:1096F000CC7E05D02B4A116821EA03011160536129
:109700002046002143F052FAA3882268B3FA83F47A
:10971000C4F11F0303F0FC0101F1804101F59C310C
:1097200003F0030398000F2702F13F438A68874044
:1097300022EA070203F57E038A60C3F3872383408E
:1097400088684FF000420343354422FA04F48B60EA
:109750004FF44062012302A88DF80E300294ADF858
:109760000C20FFF781FF95F8103FF02B01D805B0D2
:10977000F0BD0D4B9B5D8DF80430F02103224FF4BA
:10978000807301A885F8101F8DF80520ADF806300C
:109790000BF0D4FC05B0F0BD704700BF202F0020B7
:1097A000AC460708003C01402CE10708002869D0BE
:1097B000F0B58388B3FA83F3202B85B00446C3F158
:1097C0001F024AD0304E314D16444FF0004005EB99
:1097D000820230FA03F396F8A060C2F8CC1E05D0DE
:1097E0002B4A116821EA03011160536120460021D0
:1097F00043F0DCF9A3882268B3FA83F4C4F11F03B1
:1098000003F0FC0101F1804101F59C3103F00303F9
:1098100098000F2702F13F438A68874022EA070237
:1098200003F57E038A60C3F38723834088684FF083
:1098300000420343354422FA04F48B604FF4006283
:10984000012302A88DF80E300294ADF80C20FFF72A
:109850000BFF95F8103FF02B01D805B0F0BD0D4B74
:109860009B5D8DF80430F02103224FF4807301A832
:1098700085F8101F8DF80520ADF806300BF05EFC62
:1098800005B0F0BD704700BFAC460708202F002090
:10989000003C01402CE10708034BD3F8B820136AC1
:1098A000002BFCD1704700BF281E002030B5134AA2
:1098B000134B8DB0082102F1B80082F850110693C5
:1098C000694400230DF107050124CDE90733029314
:1098D0008DF8143009938DF828300B93CDE903549B
:1098E0004AF05CFBFFF7D8FF9DF80700A0F1FF00EE
:1098F000B0FA80F040090DB030BD00BF281E002036
:109900001116010870B51C4D90B00024FD220DF118
:10991000030305F1B800012601A98DF80320069381
:10992000CDE90144CDE90A44CDE90C44C5F88040B5
:109930008DF81040059407948DF824408DF8384038
:109940000F94039608964AF029FBFFF7A5FF3046CF
:109950000AF0E8FAFF2809D0084BD3F884306B6787
:109960002046092385F8843010B070BD04230220FE
:1099700085F8843010B070BD281E0020202F0020F4
:10998000F0B50379284C002B14BF012200228BB0C4
:1099900084F8B02003D184F884300BB0F0BD0546C4
:1099A00004F1B80795F9001038464AF067FCAD7825
:1099B0006DBB1E4B1E48C4F84C310126C4F8C05084
:1099C00084F8C4604AF090FC03464FF47A70A4F81F
:1099D000BC3043F095FFD4F8C00047F041FE282288
:1099E000684600216AF011FE0A2369463846029350
:1099F0004AF0D4FAFFF750FF0E4B84F88460D3F896
:109A000084306367002384F878300BB0F0BD2846BB
:109A100047F0DAF9054608B11E23C380092128461C
:109A200043F0A0FAC5E700BF281E0020881E0020D2
:109A3000801A0600202F002070B5064690B008203E
:109A40000D460AF06FFAFF2821D0FE2802D002202E
:109A500010B070BD002402230E48089301A9CDE97F
:109A60000265CDE90544CDE90A44CDE90C440194F1
:109A70008DF8104007948DF824408DF838400F94ED
:109A80004AF08CFAFFF708FF204610B070BD0120A5
:109A900010B070BDE01E002030B593B040F0400221
:109AA0000B0E0D0C04468DF80810080A8DF80420E2
:109AB000952101AA8DF805308DF806500023062562
:109AC0008DF807008DF809100DF1030001210392B4
:109AD000134A0493CDE90733CDE90D33CDE90901EC
:109AE0008DF818308DF82C300F938DF8403011938D
:109AF00005950C92FFF7DAFE00B974B9094B0822FC
:109B000003F1B80003A983F850214AF047FAFFF7A0
:109B1000C3FE9DF8030013B030BDFF2013B030BD6D
:109B2000E9150108281E00202DE9F8431A4C94F885
:109B30008460042E0546894690461F4608D0082EAC
:109B400002D00020BDE8F883FFF7DCFE0228F8D140
:109B5000D4F8C00047F07EFD94F87A309BB96902D2
:109B60001120FFF799FFA0B90C4BC4F86090D3F80F
:109B7000842065660523C4E91B87626784F8843006
:109B80000120BDE8F88329461120FFF785FF002852
:109B9000EAD00AF0EDF9D4E7281E0020202F00209B
:109BA00070B51E4C94F88430042B06460D4608D040
:109BB000082B22D1E36F83422DD0FFF7A3FE0228AA
:109BC0001BD1D4F8C00047F045FD00213720FFF736
:109BD00063FF29461720FFF75FFFB0B994F87A308A
:109BE0006BB971021920FFF757FF70B90823C4E958
:109BF0001F6584F88430022070BD012070BD31469D
:109C00001920FFF749FF0028F0D00AF0B1F90AF057
:109C1000E5F9032070BD022070BD00BF281E0020A2
:109C20002DE9F0412D4C0546884617461E4694F80E
:109C30008400042836D0082806D1E36FAB4206D052
:109C4000FFF760FE0228F2D00120BDE8F0814FF05E
:109C5000FC0CD4F8B8202248117B224B80F817CF97
:109C6000C3F8588051B1526942B194F84021002A9A
:109C70000CBF4FF480724FF4007201E04FF4807219
:109C80001A66194919484AF089F901220623C4E9DC
:109C90001885C4E91B7684F8682084F88430002095
:109CA000BDE8F081D4F8C00047F0D4FC94F87A30D5
:109CB0005BB969021820FFF7EFFE40B994F88430D1
:109CC000082BC4D04FF0FE0CC3E72946F2E70AF098
:109CD0004FF90AF083F90320B7E700BF281E0020E0
:109CE000202F002088010020B8010020E01E002065
:109CF0002DE9F04FD14C94F8B06095B0002E00F0F3
:109D0000978194F88420CE4F04F1B80804F1A0099B
:109D1000531E082B00F2A180DFE813F0370060002B
:109D20002F019F008E00B1001A009F000900FFF76D
:109D3000BDFD002840F03982636FD7F88420FA33E4
:109D4000934280F087800AF049F994F88420DFE795
:109D5000FFF7ACFD0028EFD0D4F880300022012BB3
:109D600084F8782040F23782E26F013B511CC4E94D
:109D70001F13082284F88420A2F10806B6FA86F69A
:109D80007609304615B0BDE8F08FD4F8C00047F032
:109D900061FC00210846FFF77FFE05460AF0E8F85F
:109DA000012D57D1D4F8C0004FF0000A84F879A0F3
:109DB00047F050FC40F2AB110820FFF76DFE05287C
:109DC00000F08F81012800F056810AF0D1F894F854
:109DD0007920002ACED0022384F88430D4F8C00041
:109DE00047F038FC94F87930022B0CBF4FF08045D7
:109DF000002500213720FFF74FFE29462920FFF7D5
:109E00004BFE05460AF0B4F825BB94F87930022BD6
:109E100000F07C8184F87A50D4F8C00047F01AFC36
:109E200000210920FFF738FE002875D00AF0A0F8BD
:109E300094F88420531E10E0206E4FF40071FFF759
:109E4000FBFD012800F03581022800F0398100284F
:109E500000F04A8194F88420531EDBB2022B0AD80A
:109E6000774B616FD3F884305B1AC82B84D90AF022
:109E7000B5F894F88420042A7FF47EAF81E7D4F803
:109E8000B820117B136A002900F0DE805269002A95
:109E900000F0DA8094F84021002A00F0D580B3FA6F
:109EA00083F35B09002BD5D004A900250DF10F0326
:109EB00002220591404605A94FF0010ACDE90B3A6F
:109EC0000792CDE90955CDE90E55CDE91055ADF80C
:109ED000105006958DF820508DF834508DF848506C
:109EE00013954AF05BF8FFF7D7FC9DF80F3003F0AD
:109EF0001F03052B00F062810AF070F8D4F86CB0F3
:109F0000BBF1000F00F0EA802A46236F616E5046D5
:109F1000D84794F88420FBE610214846FFF78CFDD3
:109F20008246002882D101217F20FEF7F1F8012826
:109F300005467FF47BAF50460221FEF7E9F8002882
:109F400000F0148101287FF471AF16213A20FEF74A
:109F5000DFF801308002C4F888000AF009F8D4F86C
:109F6000C00047F077FB00210A20FFF795FD00288D
:109F700040F0F580032384F88430102105A8FFF712
:109F80005BFD00287FF466AF9DF821309DF822101C
:109F90009DF81C209DF815009DF816501B01DBB2A2
:109FA00043EA111303F5FA63A4F89A30DDF81D3083
:109FB00001F00F0184F89C101BBA110902F00F0286
:109FC00045EA002084F8981084F899209DF8141030
:109FD0009DF81720C4F89430069BC4F89030A4F87C
:109FE0008C0084F88E1084F88F2009F0C1FF94F85B
:109FF0007A3073B9D4F8C00047F02CFB4FF40071ED
:10A000001020FFF749FD054609F0B2FF002D7FF44F
:10A010009AAE0C484AF068F900220423A4F8BC0068
:10A020003046C4F8802084F8843015B0BDE8F08F45
:10A03000304684F8846015B0BDE8F08F281E0020FB
:10A04000202F002040787D01236E94F868106A4824
:10A0500003EB012100224FF480734AF065FB94F872
:10A0600068300133DBB284F86830A3F10203B3FA3D
:10A0700083F35B0916E7042304AA5F48079305A945
:10A080000692CDE909AACDE90BAACDF814A08DF866
:10A0900020A08DF834A0CDF838A049F07FFFFFF75D
:10A0A000FBFB9DF81330AB2B04BF022384F87930FF
:10A0B0008BE6636FD7F8842064339342BFF4CAAE53
:10A0C00009F056FF09F08AFFE56E3DB10022104607
:10A0D000236F616EA84794F8842019E694F88420D1
:10A0E00016E684F8795070E6019009F041FFE56EBC
:10A0F000019884F87800042384F88430002D3FF41C
:10A1000040AED4E91821236FA847A3E6D4F8C000D5
:10A1100047F0A0FA29463A20FFF7BEFC04AA82467F
:10A12000042305A9404606920793CDE90955CDE9D8
:10A130000B5505958DF820508DF834500E9549F04B
:10A140002DFFFFF7A9FBBAF1000F08D109F010FFAE
:10A15000049B1BBAC3F3807384F87A305CE609F081
:10A1600007FF09F03BFF94F88420D1E504212C205F
:10A17000FDF7CEFF032182464E20FDF7C9FF0C21DB
:10A1800083463620FDF7C4FF0BF1020B421C02FA96
:10A190000BF205FA0AF5A2FB0501420A42EAC15296
:10A1A000C4F8882009F0E4FED9E6019009F0E0FE49
:10A1B00001980423064684F88430E2E50F4BE56EEF
:10A1C000D3F884306367072284F88420002D3FF49D
:10A1D000D3AD504695E708D0042384F8843009F0C5
:10A1E000C7FE94F88420531E37E6FFF78BFB022846
:10A1F0007FF430AE1AE600BFE01E0020202F0020C2
:10A2000010B4B8B10D4CD4F8183F102B05D15DF83F
:10A21000044B0521002042F0F1BF03EB430222442E
:10A2200082F81D1F01210B4482F81C0F82F81E1FAB
:10A23000C4F8183F5DF8044B704700BF202F002082
:10A2400080782021DCE700BF2DE9F04FDFF8ACA3D8
:10A250002DED028B9AF8601F002297B0CAF8502F9C
:10A26000CAF8542FCAF8582FCAF85C2FCAF84C2FD6
:10A2700019B19AF8612F8AF84C2F9AF8622F1AB107
:10A280009AF8632F8AF85B2F9AF8662F1AB19AF81A
:10A29000672F8AF8562F9AF8642F1AB19AF8652F0B
:10A2A0008AF8512F9AF8683F05935A1ED3B257B2D5
:10A2B00003937B1C00F0AA80C54AC64E52F8379023
:10A2C000029602EBC70200231279019308EE102ACE
:10A2D0001D46344698462678394630464AF05AFD9F
:10A2E00083463046BBF1000F1ED046F06DFDEA1DDF
:10A2F0001321D2B220B14FF0000E827180F807E036
:10A3000042F030FE20784AF077FD4FF0070308F165
:10A31000010223714FF0010384F802806070CDF8D0
:10A3200004B05FFA82F8E3700135042D04F10504EE
:10A33000D1D118EE100A029ECDF81080FFF700F977
:10A34000A549A64A4868024042F440324A600FB923
:10A35000019B5BB9A24C4820FFF7F2F8204602218E
:10A3600066F0B6FBA26842F00102A2609A489C4ADD
:10A370004168BAF86A4F41F400014160516821F424
:10A3800080515160916B21F4401141F4801191632F
:10A39000D16841F46001D160956B85F44011C1F33F
:10A3A000015101EB81011F2000FA01FC25EA0C0C90
:10A3B000112505FA01F141EA0C019163D16841F4DC
:10A3C000E011D160956BC5F30151C1F10401C9B22F
:10A3D00001EB810188404FF0100C25EA00000CFAD7
:10A3E00001F108439063E4B1BAF86C1FCAF8744FE6
:10A3F000A1B1BAF86E2FCAF8781F62B1019B7948F3
:10A40000521A90FBF2F2CAF87C2F6BB917B0BDEC70
:10A41000028BBDE8F08F744A1288EFE7734A118807
:10A42000E7E7734A1488DFE74846049966F050FB73
:10A43000684B012003F114080723F278441CE4B2AE
:10A4400052B375783279A5F10A0101EB410105EBB0
:10A45000450C092D03FA01FE03FA0CFB02FA01F187
:10A4600040F2A080D9F80C2022EA0E0E41EA0E013B
:10A47000C9F80C10421E02EB82021F21062801FAC5
:10A4800002FC05FA02F273D8D9F8341021EA0C0163
:10A490000A432046C9F834200536B045CDD1D9F855
:10A4A0000820039942F40072C9F80820D9F808205E
:10A4B00042F48072C9F80820D9F80820574442F0C5
:10A4C0000102C9F8082097F9702F022043F0F6FE28
:10A4D000044600289AD04668304643F0DDFE454ADF
:10A4E000431E242101FB032393F89C50002D8DD1A2
:10A4F000059983F89D10062283F89C20002885D0BA
:10A50000304643F0C9FE61F0B5F960680AF0ACFE70
:10A5100007A80AF06BFE049EA26837480792012E36
:10A520008CBF4FF4806300230D9309F14C034FF46B
:10A530008072CDE90A56089309904FF400336068A1
:10A540000C9507A94FF400674FF40056CDE910238E
:10A55000CDE90E760AF05CFE6268136843F00103F1
:10A560001360D9F8083043F08043C9F808304DE74C
:10A57000C11FA0F10D0201EB81014FF01F0E02EB94
:10A5800082020C280EFA01FC0EFA02F005FA01F123
:10A5900013D8D9F8302022EA0C0211432046C9F81A
:10A5A000301079E7D9F8101002FA0CF221EA0B0BFF
:10A5B00042EA0B02C9F810205CE7D9F82C1005FA22
:10A5C00002F221EA00010A432046C9F82C2063E781
:10A5D0005C4707086C3E002000230140E030FCFF90
:10A5E00000200140803801002E7AFF1F2C7AFF1FC7
:10A5F0002A7AFF1F88010020A03E0020202F002083
:10A600002DE9F0472E4C054600EB800004EBC0041A
:10A61000D4F88C7F2FB10E4694F8A11F01F0FF08EB
:10A6200021B14FF000084046BDE8F08799469246B8
:10A6300043F03AF971000123C9B284F8A21F84F8EB
:10A64000A3AF84F8A53F84F8A68F84F8A43F84F8CC
:10A65000A13F84F8A08FBA88C4F8A89F9105064648
:10A66000C4F8AC9F1CD43B88DA050FD442F20F74B7
:10A6700004E043F019F9831BA34215DC3B889B05DA
:10A68000F7D43B889BB243F480733B80BB889BB27A
:10A6900043F440734FF00108BB804046BDE8F087AB
:10A6A00098464046BDE8F087064A32F8F83C013348
:10A6B0009BB2284622F8F83C65F02CFDB3E700BFBA
:10A6C000202F00201840002070B5464E16F8F64C9A
:10A6D00004EB440306EBC303650013F8F43C032BBF
:10A6E0006ED8DFE803F059291E02254406EBC505A4
:10A6F00055F8F00C002870D116F8943C9C425FD0BD
:10A70000013404F00302934206F8F62C58D002EB11
:10A71000420406EBC404022344F8F00C04F8F43CB1
:10A7200070BD2B1906EBC30353F8F02C72B1013A3C
:10A7300043F8F02C002070BD2B1906EBC30353F82F
:10A74000F02C002AF3D1022203F8F42C254406EB66
:10A75000C50515F8E83C013BDBB205F8E83C8BBBCE
:10A76000214B16F8946CD3F8C01255F8EC0C621C0F
:10A7700002F003024B1E0324B242034405F8F44CDA
:10A78000B3FBF1F045F8F00C1AD0994218D8013813
:10A7900045F8F00C012070BD4AF0FEF980B1124B73
:10A7A0002C44D3F8C02206EBC404012102F51C534B
:10A7B00004F8F41C0F33B3FBF2F344F8F03C70BD23
:10A7C000012070BD084BD3F8C022012002F2E7330C
:10A7D000B3FBF2F345F8F03C70BD013845F8F00CDE
:10A7E000002070BD1840002088010020054B13F8A0
:10A7F000932C002AFBD1D3F8D03A03491B6801F10E
:10A800000C00184718400020883F00202DE9F84F21
:10A810003249DFF8D4B091F8351E012402290746E9
:10A8200019461046CBF82C404FF000022C4C1D4628
:10A8300018BF7F02FDF7E4FB2A4B63626B02A36241
:10A84000E36A40F2FF5943F093034FF400704FF472
:10A850008A62E3620121C4F83890A0601020E260AF
:10A860005FF040FF012D40F251434E46C4F838904E
:10A87000CA4640F252488EBF4FF0120998464FF038
:10A8800011090A25C4F838A00121A7604846C4F878
:10A890000C805FF027FF03464FF0000C40F2774238
:10A8A00001213720A6632BB900231846CBF82830A6
:10A8B000BDE8F88FA663C4F808C0E2605FF012FF3D
:10A8C000013DA6630028EFD015F0FF05DAD103465D
:10A8D000CBF82C50CBF82830BDE8F88F202F002083
:10A8E000002C014000E1F505281E00202DE9F84369
:10A8F000DFF8748098F88450042D04468946174682
:10A900001E4608D0082D02D00020BDE8F883FEF7CF
:10A9100059F90228F8D101234A4620460021FFF7C1
:10A9200075FF68B1FEF7DAF9D8F86C40002CEBD06F
:10A930000022D8F87030D8F864101046A047E3E73A
:10A94000084BC8F86090D3F88420C8F86440052309
:10A95000C8E91B76C8F8742088F884300120BDE867
:10A96000F88300BF202F0020281E00202DE9F84F7B
:10A970002F49DFF8C49091F8351E1E4602292D4B51
:10A9800007464FF0010418BF4702012E40F2594814
:10A990001C6398BF4FF48B683B469346474640F292
:10A9A000FF55B0468CBF4FF0190A4FF0180A0A2421
:10A9B0001E4640F2FF53C9F838300121C9F808603B
:10A9C0005046C9F80C705FF08DFE03464FF0000C46
:10A9D00040F2774201213720C9F83850A3B95846D0
:10A9E00041460122FDF70CFB4646134A134B5362C6
:10A9F00076029662D36A43F09103D3620D4B002135
:10AA000008469962BDE8F88FC9F83850C9F808C0FF
:10AA1000C9F80C205FF066FE013CC9F838500028E8
:10AA2000DDD014F0FF04C4D1024B1C63BDE8F88FE5
:10AA3000202F0020281E0020002C014000E1F505F9
:10AA40002DE9F047374C82B005460E46174698462A
:10AA500094F8840004280CD0082806D1E36FAB4298
:10AA600007D0FEF7AFF80228F2D0012002B0BDE80F
:10AA7000F087DFF8B8A02666DAF82C9E6566C9F381
:10AA80004F210F294FEA592223D8D4F8803001935F
:10AA9000FBB194F85201E0B1B9F5005F13D0224840
:10AAA00031464FF40072484469F04EFD09F50072DA
:10AAB000C2F34F211029CAF82C2E4FEA522202D09D
:10AAC000019B012B21D192B2013A174EAD1A0B46D0
:10AAD00000E0012332462846062601250021E766CC
:10AAE000C4F8708084F8685084F88460FFF73EFFF3
:10AAF0000028BBD0FEF7F2F8E66E86B12846236F39
:10AB0000616E0022B0470320B0E7E26F013B0132E3
:10AB10000421C4E91F2384F884100220A6E703203F
:10AB2000A4E700BF281E002094700020202F0020E2
:10AB3000144A154BD2F8BC24B3EB920F15D2B3EBE9
:10AB4000D20F14D2B3EB121F13D2B3EB521F12D297
:10AB5000B3EB921F11D2B3EBD21F10D2B3EB122F73
:10AB600034BF4FF48070802070470220704704206B
:10AB70007047082070471020704720207047402001
:10AB8000704700BF202F00208096980003681A7835
:10AB9000012A01D00020704793F90430044A03EBE6
:10ABA000830302EBC30393F8A10FC0B2704700BF49
:10ABB000202F0020F0B53B4CD4F8D45A2B78022B30
:10ABC00095B018D0012B02D0002015B0F0BD95F93A
:10ABD00004506B1CF8D0022DF6DC0091134694F85B
:10ABE000D81A0246284665F037FC0028ECD02846E3
:10ABF00065F0E2FCE9E72B6A002BE5D10DF10F0CC3
:10AC00008DF80F00002601200027CDE90833CDE99B
:10AC10000A12CDE90E6705938DF81C300D93109341
:10AC20001293CDF810C006908DF830008DF84400D6
:10AC3000EFF31180102383F31288D4F8D43A1B6AFF
:10AC400013B3069B04AE32461BB1D3691432002BFA
:10AC5000FBD12B6A13B3996839B993420AD01968AA
:10AC600029B15B6899680029F7D01433F3E70E4ADD
:10AC7000C3E90026C0B280F31188D4F8D42A136A3D
:10AC8000002BFCD10120A0E704ABC0B22B6280F303
:10AC9000118804F6D42062F041F9EEE7024A1A6006
:10ACA000FFDE00BF18400020EC4A002070B50368AA
:10ACB0001D78022D14D0012D01D0002070BD044656
:10ACC00093F904000A4B421C83F8A05BF5D00228DC
:10ACD000F3DC0A4603F53A632179BDE870408FE45E
:10ACE0001B6A002BE9D1012249F07EFC012070BDD6
:10ACF0001840002010B50B4CD4F8D43A1B78022B26
:10AD00000FD1D4F8DC0A46F0ABFCD4F8DC0A08B169
:10AD10002123C380012142F025F9FFF709FFA4F8A0
:10AD2000D80A10BD1840002030B583B00D4601236D
:10AD300001460DF107020446074849F0C5FD9DF89C
:10AD4000072035EA020304D003482A43214649F08C
:10AD500051FE03B030BD00BFEC4A002038B50546B7
:10AD60000A460C460648294649F03EFC45F080015B
:10AD7000034849F0E3FA231A5842584138BD00BF4E
:10AD8000EC4A002013B53A4C0023D4F8B02B8DF8D0
:10AD90000730137803F0FD01012905D194F8B41BA5
:10ADA00011B90C2184F8B41B022B1ED0032B2DD01B
:10ADB00001220B212F485DF01FFC042042F0A0FD72
:10ADC0002C4801230DF1070200215DF037FC00281B
:10ADD00038D09DF80730482B34D1274BC4F8A43B1A
:10ADE000264BC4F8A83B02B010BDD4F8B80B46F00F
:10ADF00037FCD4F8B80B08B13523C380012142F0E9
:10AE0000B1F8FFF795FEA4F8B40BD1E71C4B5068DE
:10AE10001B6846F2A8111961002380F888301222BD
:10AE200037215DF0BDFBD4F8B03B0D2258682421DA
:10AE30005DF0B6FBD4F8B03B302258686A215DF073
:10AE4000AFFBB5E7D4F8B03B1A78022A03D0032A47
:10AE500007D00020C7E7D4F8B80B48F0F7F9002076
:10AE6000C1E75868102237215DF09AFBF1E700BF77
:10AE700018400020C84B00209B8606081D87060846
:10AE8000785000202DE9F04FB64CB74E95B0002316
:10AE900005464FF4F0728B4604F56B70202184F860
:10AEA000A83384F8A933019569F0AFFB202104F29F
:10AEB0008C504FF4F07269F0A8FBDFF8C4C2AB49C4
:10AEC00032274FF0100E4FF47A704FF00108DCF883
:10AED0000430C3F30803002B40F0BC80EFF3118370
:10AEE000002B40F0B780D6F884208D68D6F88430E7
:10AEF0009A42F8D1D6F8C83E9D42F4D8D6F8C49EFE
:10AF000000FB09F35B1BB3FBF9F300FB0232DCF837
:10AF10000430C3F30803002B7BD1EFF31183002B24
:10AF200077D1D6F88430D1F808A0D6F88450AB4257
:10AF3000F7D1D6F8C85EAA45F3D8D6F8C49E00FB70
:10AF400009F5A5EB0A05B5FBF9F500FB03539B1AC0
:10AF5000B3F57A7FDBD3013FB9D194F86D27002A8E
:10AF600052D094F86E37013B022B4DD803EB83018E
:10AF700004EBC1007E4D90F8707705EBC1014FF0F6
:10AF8000010C022FC4F8E81784F870C800F0C382DF
:10AF9000DBB204EB0313D3F88038C0F874379BB3EB
:10AFA00002234FF4807780F8703705F18803C435A9
:10AFB000A0F87C77C0F88837C0F88C571509013D98
:10AFC000052D02F00F0200F289826A4F07EB45035C
:10AFD000B3F8840040FA02F3DB0740F17F820123DB
:10AFE00003FA02F2013A10403D4466F075FD95F80F
:10AFF0009020614B104403EBC000C4F8F007837944
:10B00000002B47D0412B45D06FF0010015B0BDE8B3
:10B01000F08FEFF311898EF31288D1F808A00B6836
:10B02000DD0344BFC6F8C08ED1F808A0D6F884303E
:10B03000D6F8C05E5FFA89F989F31188D6F8C49E04
:10B040002B4400FB09F5A5EB0A05B5FBF9F500FB60
:10B0500003537CE7EFF311858EF31288D1F8089043
:10B060000B68DB0344BFC6F8C08ED1F80890D6F851
:10B070008430D6F8C02EEDB285F31188D6F8C45EC0
:10B080001A4400FB05F3A3EB0903B3FBF5F300FB44
:10B0900002323CE72323C380092141F087FDD4F825
:10B0A000F037002B00F065821A68D4F8E8179B8807
:10B0B0001383D6F8BC24314BB3EB920F80F031826E
:10B0C000B3EBD20F80F02F82B3EB121F80F02F82F0
:10B0D000B3EB521F80F02F82B3EB921F80F02F82D0
:10B0E000B3EBD21F80F02F82B3EB122F80F02D82B2
:10B0F0004FF480720023FF200DF10F08A4F8EC2715
:10B100000122CDE90483CDE90833CDE90A338DF876
:10B110000F000D9306928DF81C208DF83020EFF370
:10B120001180102383F31288D4F8E8371B6A002BB0
:10B1300000F0D881069B04AD2A461BB1D3691432B6
:10B14000002BFBD10B6A002B00F01C82996839B9E7
:10B150009A421AD01968A9B15B6899680029F7D09A
:10B160001433F3E710510020202F002010E000E0FE
:10B1700080580020AC460708DC300020404B4C00D3
:10B1800000ED00E0B74AC3E90025C0B280F31188A2
:10B19000D4F8E8170B6A002BFCD18C220120CDE9F2
:10B1A00008330DF10E0A05938DF81C300D931093A2
:10B1B00012938DF80E2000230022CDE90E23CDF846
:10B1C0002880CDF810A006900B908DF830008DF8F7
:10B1D0004400EFF31180102383F31288D4F8E8378A
:10B1E0001B6A002B00F08781069B2A461BB1D3699E
:10B1F0001432002BFBD10B6A002B00F0C38199683D
:10B2000039B99A420AD0196829B15B68996800294E
:10B21000F7D01433F3E7934AC3E90025C0B280F3B3
:10B220001188D4F8E827136A002BFCD19DF80F3061
:10B230001B2B40F09081D4F8F037012284F8A8232A
:10B240000BB12322DA80DFF81C92402248460A2103
:10B2500049F0CAF98A21002301228DF80E1000203E
:10B260000021CDE90E01CDE90833D4F8E817CDF877
:10B2700010A0CDF8288005938DF81C300D93109305
:10B28000129306920B928DF830208DF84420EFF344
:10B290001180102383F31288D4F8E8371B6A002B3F
:10B2A00000F03181069B2A461BB1D3691432002B72
:10B2B000FBD10B6A002B00F06281996839B99A4280
:10B2C00009D0196829B15B6899680029F7D014334F
:10B2D000F3E7C3E90095C0B280F31188D4F8E827FA
:10B2E000136A002BFCD19DF80F2094F86C17C2F361
:10B2F000801284F8B028002900F0D480022900F0E0
:10B30000B980D6F8BC345849B1EB930F80F01F8157
:10B31000B1EBD30F80F00981B1EB131F80F00981ED
:10B32000B1EB531F80F00981B1EB931F80F00981CD
:10B33000B1EBD31F80F00D81B1EB132F34BF4FF46D
:10B340008076802694F8B418A4F8B268182914D12D
:10B35000464F474800215B08B3FBF6F3A7FB037396
:10B360000F465B0B66F30F076BF30F0163F31F4789
:10B3700062F31F41C4F8B81847603A48A4F8EC6774
:10B380000222002149F030F9C82042F07FF8D4F8B9
:10B39000E8074FF0800B0026002700230122CDE9AB
:10B3A0000E67CDE908338DF80EB0CDF810A0CDF8BA
:10B3B000288005938DF81C300D93109312930692FC
:10B3C0000B928DF830208DF84420EFF3118210237A
:10B3D00083F31288D4F8E8371B6A002B38D0069B19
:10B3E000002B3DD02B46D96914330029FBD1006ACC
:10B3F000002800F0C180816839B9834209D0016812
:10B4000029B1406881680029F7D01430F3E7C0E91A
:10B410000095D2B282F31188D4F8E807036A002BB2
:10B42000FCD19DF80F3013F00203B6D1019841789A
:10B430008278007884F8C008C1F12001C2F11002BE
:10B44000184684F8C11884F8C22815B0BDE8F08FFA
:10B450000562D2B282F31188024861F05FFDDBE73A
:10B460002B46C4E7F8580020809698005917B7D1AA
:10B47000C8590020D6F8BC344448B0EB930F73D2BF
:10B48000B0EBD30F51D2B0EB131F52D2B0EB531F1E
:10B4900053D2B0EB931F54D2B0EBD31F34BF8026EE
:10B4A00040264FE7D6F8BC343949B1EB930F4ED262
:10B4B000B1EBD30F39D2B1EB131F3AD2B1EB531F1B
:10B4C0003BD2B1EB931F3CD2B1EBD31F41D2B1EBD6
:10B4D000132F34BF4FF48076802633E70023C4F85F
:10B4E000F037E6E504ADC0B20D6280F3118829485B
:10B4F00061F014FD4CE60D62C0B280F3118825485E
:10B5000061F00CFD8DE60D62C0B280F311884846F3
:10B5100061F004FDE2E690F87D37634480F87D3702
:10B520004CE50222E6E50422E4E504260AE70822C7
:10B53000E0E5082606E71022DCE5102602E72022D7
:10B54000D8E52026FEE64022D4E58022D2E5022678
:10B55000F8E64026F6E6D4F8F00738B1202141F0AD
:10B5600025FB4FF0FF3051E50E46EBE64FF0FF3084
:10B570004CE5D4F8E8179CE5C0F80090FFDEC3F86E
:10B580000090FFDE034A1A60FFDE00BF002D31018C
:10B59000404B4C00F85800200146014848F0CEBE10
:10B5A000D4590020094B93F82E31042B08D9053BC0
:10B5B000032B08D801231A4600B1037010467047C8
:10B5C00000230122F8E700231A46F5E7202F002088
:10B5D000F0B40D6800240CE0BCF1050F18D8A0F100
:10B5E00037030A2B14D104EB840415F8010B03EB89
:10B5F0004404A0F13003DEB2092EA0F16107A0F1EE
:10B60000410CF0D9052FE7D8A0F157030A2BEAD057
:10B610000D601460F0BC70479FED727A07EE901ACF
:10B6200020EE070AF8EE677A27EE800AFDEEC07A70
:10B6300017EE903A2033402B00F2C480DFED6A7A97
:10B64000B4EEE70AF1EE10FAF0EE407A0CDD9FED71
:10B65000676ADFED676AB0EE677AB4EEE67AF1EE1C
:10B6600010FA77EEC67AF6DC9FED627AF4EEC77ACE
:10B67000F1EE10FA0CD59FED5D6ADFED5F6AB0EE7A
:10B68000677AB4EEE67AF1EE10FA77EE867AF6D4BF
:10B690009FED5A7AF4EEC77AF1EE10FA00F38A8041
:10B6A0009FED577AF4EEC77AF1EE10FA44BF9FEDA2
:10B6B000517A77EE677A27EEA76ADFED525A9FED4F
:10B6C000527ADFED526AA6EE257A67EE865AE6EEEA
:10B6D000076AB6EE007AE5EEA67A27EE877ADFED06
:10B6E000476A70EE267ABDEEE76A16EE103A20330E
:10B6F000402B64D8B4EEE60AF1EE10FA0CDDDFED73
:10B700003B5A9FED3B6AF0EE676AF4EEC66AF1EED3
:10B7100010FA77EEE57AF6DCDFED366AF4EEE67ADB
:10B72000F1EE10FA0CD5DFED315A9FED336AF0EEF1
:10B73000676AF4EEC66AF1EE10FA77EEA57AF6D4EF
:10B74000DFED2E6AF4EEE67AF1EE10FA3DDDDFED84
:10B75000266A76EEE77A67EEA75A9FED2A5A9FEDA2
:10B760002A6ADFED2A6AA5EE856A27EEA55AE5EE7C
:10B77000866AB8EE006AE5EE267A67EE867AC7EE4C
:10B78000206AB7EE006A76EE865A76EE666A86EE34
:10B79000257A80ED091A67EE277A66EE876AC0ED92
:10B7A000017AC0ED037A80ED007A80ED027AC0ED77
:10B7B000046A70479FED0C7A77EE677A7BE7DFEDDE
:10B7C000147ADCE79FED127A89E7DFED0D6AF4EE7B
:10B7D000E67AF1EE10FA44BFDFED066A76EEE77A1C
:10B7E000B9E700BF27D4D236DB0F4940DB0FC94091
:10B7F000E4CB1641DB0F49C0E4CB16C1DB0FC93FD8
:10B80000DB0FC9BF92E741B99730083C15A82ABEA3
:10B81000000000002DE9F843E14FDFF8E4E3D7ED45
:10B820003E7A2DED028BF8EE670A9EF85C4907F22E
:10B830006C63C3ED000A002C6FD1DFF8C8C397F822
:10B840007866C7F874469CF80040002E39D0BEF8E0
:10B8500062399FEDD46A9FEDD47A07EE903AF8EE04
:10B86000677A20EE877AC6EE276AD04B0022012E37
:10B870001A6076EE876AC7EE267AC3ED017A20D089
:10B88000022E9A60C3ED037A1BD0032E1A61C3ED1A
:10B89000057A16D0042E9A61C3ED077A11D0052ED1
:10B8A0001A62C3ED097A0CD0062E9A62C3ED0B7AA8
:10B8B00007D0072E1A63C3ED0D7A02D09A63C3ED49
:10B8C0000F7ABB4B9FEDBB6A93F84E319FEDBA7A6E
:10B8D0009FEDBA0ABA4A07EE903AF8EEE77A9CF87A
:10B8E000583BC6EE276A1C4414FB06F6F6B207EE78
:10B8F000906A60EE870AF8EEE77AC2ED006AA7EE7A
:10B90000A00A67F0FBFBBDEC028BFCEEC07A17EEE1
:10B91000903A87F8C837BDE8F883BCEEE06A9FED3F
:10B92000A97A9EF85D39BEF860299FEDA72ADFED60
:10B93000A76ADFF8D0C297F87866C7F874C6F8EE41
:10B94000465A07EE903A87EE255A8CF8004007EEEB
:10B95000102ABEF85E298CED025A16EE103AF8EE67
:10B96000677A06EE102AB8EEC77A27EE822AB8EE7A
:10B97000466A67EE266ACCF81430012322EE252AA7
:10B98000CCED017A8CED036ACCED046A87F8703651
:10B99000002E96D0DFED8E7A9FED8E4ADFED8E5A27
:10B9A000C7EE871AC6EB0615A6EB06190CEBC50504
:10B9B0004FEAC9094FF00008B1EE611A9FED876A9E
:10B9C00009EB05009FED863ADFED863ADFED866AEA
:10B9D0000346002207EE902AB8EEE77A27EE027AB5
:10B9E000FDEEC77A17EE901A2031402900F2D08080
:10B9F000B4EEC47AF1EE10FAF0EE477A0CDDDFED2A
:10BA00007B4A9FED7B5AF0EE672AF4EEC52AF1EEF1
:10BA100010FA77EEE47AF6DCF4EEE57AF1EE10FA5D
:10BA20000CD5DFED724A9FED735AF0EE672AF4EE03
:10BA3000C52AF1EE10FA77EEA47AF6D4F4EEC67ABF
:10BA4000F1EE10FA40F39A8074EE677A27EEA75A67
:10BA5000B0EE630AA5EE030ADFED674AE5EE004AA1
:10BA600065EE272AB7EE005AE2EEA47AB0EE458AD8
:10BA7000F0EE454AA1EEA78AE1EE274AC5EE088A14
:10BA800084EE880A77EE067ABDEEE75A15EE101AB4
:10BA9000203140296FD8B4EEC67AF1EE10FA0CDDF1
:10BAA0009FED525A9FED527AF0EE674AF4EEC74A84
:10BAB000F1EE10FA77EEC57AF6DCF4EEE57AF1EE07
:10BAC00010FA0CD59FED495A9FED4A7AF0EE674A7D
:10BAD000F4EEC74AF1EE10FA77EE857AF6D4F4EE7A
:10BAE000C67AF1EE10FA3CDD74EE677A27EEA75ABB
:10BAF000F0EE632AE5EE032A9FED3F7AA5EE227A67
:10BB000065EE274AB8EE005AE4EE877A67EE857A4A
:10BB100087EE887A0132A24203F1280343ED048ABA
:10BB200003ED037A03ED017A43ED028A83ED000A07
:10BB3000C3ED056AC3ED026AC3ED016AC3ED046A91
:10BB4000C3ED036AFFF646AF783085427FF43AAF23
:10BB500008F57078B8F5346F05F570757FF42EAF81
:10BB600075E69FED267AF4EEC77AF1EE10FA48BF3B
:10BB700075EEE77ABAE7F0EE667AC9E79FED1F5AED
:10BB8000F4EEC57AF1EE10FA48BF75EEE77A5DE79C
:10BB9000B7EE000AF0EE408AB0EE408A72E700BFCE
:10BBA0000800001083F9223EBD378635745A002004
:10BBB000202F0020555555406E12833A48E1FA3E39
:10BBC000CC0700100060EA4827D4D2360AD7233CBD
:10BBD00000004842DB0F4940DB0F49C0DB0FC93F83
:10BBE00092E741B99730083C00000000DB0FC940E4
:10BBF000E4CB1641E4CB16C115A82ABEDB0FC9BFA2
:10BC0000105100204C1800102DE9F04F07EE900A5B
:10BC10002DED068B9FEDF07AF04BDFEDF16AB3F876
:10BC2000A429F04F93F8AA59C7F81C08B8EE679AF0
:10BC30000AEE102A87EE095AB3F8A629C7F8D85792
:10BC400083B008EE102AB3F8A829DFEDE77AB8EE42
:10BC50004AAA08EE902AB8EEC88A3AEE0A7AF8EEB6
:10BC6000E88AB4EEC78AF1EE10FA68EEA77AB4EE6D
:10BC7000E65A07F2CC73B8BFB0EE478A0022F1EE65
:10BC800010FA83ED028A83ED01AAC3ED007AC7F8AA
:10BC9000DC2700F1038307EE905AF8EEE77AB7EE5F
:10BCA000007AC7EE279AD14BDFF878A319461431F2
:10BCB0009C4601919AF8982003F12C04F6EE005A64
:10BCC00065EE256AF7EE007A86EE887ADFEDC83AEF
:10BCD000DFEDC84A9FEDC86AD3ED05AAB4EEE77A56
:10BCE000F1EE10FAB8BFB0EE677ABDEEC77AB0EEEB
:10BCF000004A17EE106AB8EEC77AC7F8786AC5EE40
:10BD0000076A87EE875A66EEA36AACEC015A8AEEA0
:10BD1000267AC8EE267A37EE257A77EEA57AB4EE43
:10BD2000C47AF1EE10FAB8BFB0EE447AF4EEE47AD9
:10BD3000F1EE10FABDEEC77A88BFF0EE647A17EE26
:10BD4000100AFDEEE77A00F1FF3B17EE901ABBF107
:10BD5000230FA8BF4FF0230BCCED006A012E01F199
:10BD6000010CB8BF0126BCF1230F2BEAEB7BE046A8
:10BD700029EE066AA8BF4FF02308E345C8BFD8469E
:10BD8000C7F8840AC7F8881A83ED046AA8EB0B0782
:10BD900097FBF6F70137002A40F0E380DFED970AC2
:10BDA000DFEDA15A9FEDA12A9FED955ADFEDA32A61
:10BDB0009FEDA33ADFEDA33A9FED924ADFEDA21A81
:10BDC0000AF19C0107EE902AB8EEE76A66EE207A47
:10BDD00037EEA57AFDEEC76A16EE903A2033402B77
:10BDE00000F21582F3EE026AB4EEE66AF1EE10FAA2
:10BDF0000CDDDFED904ADFED8E6AB0EE471AB4EE4F
:10BE0000E61AF1EE10FA37EE647AF6DCB4EEC57A93
:10BE1000F1EE10FA0CD5DFED874ADFED876AB0EE60
:10BE2000471AB4EEE61AF1EE10FA37EE247AF6D499
:10BE3000B4EEE57AF1EE10FA40F3FE81DFED726ABE
:10BE400036EEC77A67EE076AB0EE431AA6EEA21A7C
:10BE5000B0EE630AA1EE260A67EE264AFDEEE76A17
:10BE6000A4EE807A16EE903A2033402B27EE047A27
:10BE700000F2D781DFED656AB4EEE66AF1EE10FA02
:10BE800040F300829FED6B0A9FED691AF0EE676A3E
:10BE9000F0EE664AF4EEC14AF1EE10FA76EEC06AB0
:10BEA000F6DC9FED591AF4EEC14AF1EE10FA13D503
:10BEB0009FED601ADFED604AB0EE660AB4EEE40A68
:10BEC000F1EE10FA76EE816AF6D4DFED506AB4EE48
:10BED000E66AF1EE10FA0CDD9FED566ADFED546A6A
:10BEE000F0EE674AF4EEE64AF1EE10FA77EEC67A23
:10BEF000F6DCF4EEC57AF1EE10FA0CD59FED4D6A42
:10BF0000DFED4D6AF0EE674AF4EEE64AF1EE10FA24
:10BF100077EE867AF6D4F4EEE57AF1EE10FA40F395
:10BF20008381DFED396A76EEE77A67EEA76AF0EE95
:10BF3000434AE6EEA24AB0EE631AA4EEA61A27EE32
:10BF4000A66AE6EE017A67EE847A0132242A81ED50
:10BF5000007AC1ED017A01F108017FF433AFDFED22
:10BF60002CAA4FF0000944E9059B44E902764FF4FE
:10BF700090720021204644F80C8C68F046FB4FF488
:10BF80009072A018002168F040FB224B04F5157454
:10BF9000A342E8D1019BDFED207AC3ED00AA012383
:10BFA00029EE279A8AF89830002D00F02B81DFEDDA
:10BFB0001B7A1B4E9FED142ADFED112AC7EEA81A3B
:10BFC000A6F1140406F5117738EE4A8AB1EE611A2B
:10BFD00069EE889A3EE000BF0024744910510020A9
:10BFE0000000FA44080000100AD7233C840A00101D
:10BFF000398E633C00000C429C534937C3B8B23DB4
:10C00000DB0F49C072F97F3FDB0F4940000010424F
:10C01000BC297E3FAC11001027D4D2360000484224
:10C02000E807001000110010DB0FC93F00000000FE
:10C03000E4CB1641DB0FC940E4CB16C192E741B90E
:10C040009730083C15A82ABEDB0FC9BF000010C2FC
:10C050000000807F5FED0C5A5FED0C6A234630468E
:10C060000022B7EE005A07EE902AF8EEE77AB6EE15
:10C07000007A77EE877AB0EE4A7AA7EEA97AF0EEE8
:10C08000477A29EE077AE0EC017AFDEEC77A17EEDF
:10C09000901A2031402900F2D780B4EEC27AF1EE36
:10C0A00010FAF0EE477A0CDD1FED1E4A5FED204AD4
:10C0B000B0EE676AB4EEE46AF1EE10FA77EEC47A95
:10C0C000F6DCF4EEE27AF1EE10FA0CD51FED274A19
:10C0D0005FED274AB0EE676AB4EEE46AF1EE10FA5B
:10C0E00077EE847AF6D4F4EEE57AF1EE10FA40F3C6
:10C0F000B58072EE677A67EEA74A5FED303A1FEDC2
:10C10000304A1FED306AA4EEA34A67EEA43AA4EECB
:10C11000246AF0EE454AE3EE867AB0EE456AE1EE37
:10C12000274AA1EEA76A84EE864AC5EE064A77EE54
:10C13000257AFDEEE73A13EE901A2031402900F2FD
:10C140008A80B4EEE57AF1EE10FA0CDD1FED473A85
:10C150005FED493AB0EE677AB4EEE37AF1EE10FAA9
:10C1600077EEC37AF6DCF4EEE27AF1EE10FA0CD553
:10C170001FED503A5FED503AB0EE677AB4EEE37AD5
:10C18000F1EE10FA77EE837AF6D4F4EEE57AF1EE7A
:10C1900010FA6DDD72EE677A27EEA73A5FED590A65
:10C1A0005FED593A1FED597AE3EE203A63EE270A24
:10C1B000A3EE237AF8EE003AE0EE877A67EEA37AF0
:10C1C00087EE867A0132AA4203F12803C3ED0B4AB7
:10C1D00083ED0C7A83ED0E7AC3ED0D4A83ED0F4AA1
:10C1E00083ED145AC3ED116AC3ED106AC3ED136AEF
:10C1F000C3ED126A7FF437AFC834A74206F11406C4
:10C200007FF428AF03B0BDEC068BBDE8F08FFDEEE8
:10C21000E76AB0EE427A16EE903A2033402B7FF672
:10C2200029AEF0EE427A90E6F4EEE17AF1EE10FA01
:10C2300048BF75EE677A78E6B4EEE17AF1EE10FA6F
:10C2400048BF35EE477AFDE5B7EE004AF0EE444AC6
:10C25000B0EE446A6BE7F0EE667AB1E71FED866AEE
:10C26000F4EEC67AF1EE10FA48BF72EEE77A42E7D2
:10C270001FED8B7AF4EEC77AF1EE10FA48BF72EE3A
:10C28000E77A89E75FED8F6AB4EEE66AF1EE10FABD
:10C2900048BFF0EE676A3FF50BAE2AE65FED949A71
:10C2A000C7F8D8271546FEE408480023024611784F
:10C2B000022902F1060204D00133062BF7D1002037
:10C2C000704703EB430300EB43007047601E002000
:10C2D00000B50021084B83B00846C3F8AC1933F011
:10C2E000B5FF0422054B01930DEB0201062033F04C
:10C2F000A1FF03B05DF804FB105100205475C52A5E
:10C3000070B5461E00F13105344614F8011F601E59
:10C31000801BFF29C0B201D033F098FFAC42F4D1AA
:10C32000A02056F053FB0121022033F08FFF40F292
:10C33000E93401E0013C04D04220FFF72DF9002848
:10C34000F8D16220FFF728F91321242033F07EFF73
:10C350002520092133F07AFFBDE87040A02056F077
:10C3600035BB00BF00231B88FFDE00BF38B50C4C77
:10C370000546A11CD52254F06BFD2B68A342C5E9EC
:10C380000043A3EB04000AD004F14002611C2960C1
:10C39000237802F8013BD5E90041A142F6D138BD2E
:10C3A000C05A002010B5204B84B0C82403F51F618B
:10C3B00003F6B1122128CDE9022183F8B04918D043
:10C3C0000CD802281ED0082825D102A801900AF016
:10C3D000E9FE0198FFF7CAFF04B010BD29281AD161
:10C3E00002A801900AF098FD0198FFF7BFFF04B082
:10C3F00010BD02A801900AF0D9FD0198FFF7B6FF21
:10C4000004B010BD02A801900AF018FF0198FFF7D0
:10C41000ADFF04B010BD02A801900AF039FE0198EA
:10C42000FFF7A4FF04B010BD1051002010B582B07A
:10C430000A788DF80720040A18238DF804308DF847
:10C4400006008DF8054056F04FF901AA0348114641
:10C45000042348F069F902B010BD00BFD459002090
:10C4600010B582B0040A192200238DF801408DF81E
:10C4700000200C468DF803308DF8020056F034F998
:10C480006A4605481146052348F04EF99DF80430E8
:10C49000237002B010BD00BFD459002010B58CB07D
:10C4A00000234CF20502044601A9CDE90633CDE98B
:10C4B0000833ADF800208DF8023003220B930123DE
:10C4C000CDE903128DF814308DF82830CDF808D05E
:10C4D00048F070F9204602A947F060FD204648F078
:10C4E00069F99DF806000CB010BD00BF2DE9F043BE
:10C4F000764D774F83B005F138002422002168F093
:10C5000084F897F8314A0023EB65002C39D1714E3D
:10C51000D6F8F83053B39B6A43B36F4898478368A3
:10C5200023B303886D4F013B9BB2BC4638460021C4
:10C530000678032E00F106001CD001310629F7D140
:10C5400000223978022907F1060700F09E800132A7
:10C55000062AF6D1E96D052908D0481C02FB01C264
:10C56000E86502200021938010705180204603B0BE
:10C57000BDE8F083062303FB01514B8F013B9BB2C7
:10C58000DEE797F8300A07F63823C7F8343A10B9CF
:10C59000504E0024BCE744F017FCC7F8400A18B11D
:10C5A00083790BB1412BF3D121464D4847F066FE0C
:10C5B00004460028ECD0D7F8343A474A9868C3F8C4
:10C5C000942008B12023C380092140F0CBFCD7F888
:10C5D000343A404E986845F043F84248D7F8348AD8
:10C5E00047F082FE4FF00109A8F804003220C6F897
:10C5F000188186F81C9141F083F90423D7F8340A96
:10C600004FF0000C0DEB03029F21CDF804C047F062
:10C6100097FF9DF805809DF804309DF806104FEABD
:10C62000082848EA034848EA0108414606F1F800AC
:10C6300055F09AFC00287FF46BAF4046FBF7A0FF53
:10C64000034600287FF464AF9DF806009DF805209E
:10C650009DF80710000240EA0240234A0843904236
:10C6600017D0C6E94033A6F8FC30A6F80831FBF72E
:10C6700087FF804600287FF44BAF97F8300A44F0DC
:10C68000A3FB46F0E3FD444642E7062101FB02C25C
:10C6900067E7164AC6F8FC204FF400334FF00062FB
:10C6A000C6F800314023A6F80831C6F8042186F800
:10C6B0000A91FBF705FD06F1F80086F8119155F097
:10C6C0009FFB0B4BC6F8F83022E700BF281E002066
:10C6D00010510020202F002018300020601E002064
:10C6E000485B0020404B4C0021AAEF0000040008EA
:10C6F000AC4607082DE9F041C94BCA4ECA4DCB4C98
:10C700000822C3F88820336B82B043F001033363FF
:10C7100007464FF4C052284640F202338846694625
:10C72000CDE9002308F054FF6B6AC14ADFF848C323
:10C7300023F470436B626B6A43F420436B626B6A51
:10C7400023F470236B626B6A43F420236B62736C77
:10C75000B84D43F4804341F2B4017364736B44F801
:10C76000018041F2BC0143F08003675041F2B80EF2
:10C77000B14973630227C4F8D41AB04EB04BB14923
:10C7800044F80E5084F8D87A4FF0A045AE4FC4F864
:10C79000DC5AC4F8E06AC4F8E83AC4F8241B05F58A
:10C7A000326506F5A07603F51073A1F5D071C4F8D3
:10C7B000EC7AC4F8285BC4F8F06AC4F82C3BC4F8DF
:10C7C000F41A012307F51077A5F5E465A6F5A06630
:10C7D000A1F58C61C4F8D0CAC4F8307BC4F8E45A1F
:10C7E000C4F89C6B84F8DB3A05F5A075536106F537
:10C7F000B076C4F8601B84F8E23B1946934B944A28
:10C80000C4F8685BA7F5BC67A035C4F8746B914E9B
:10C81000C4F8707BC4F8783B07F5D45703F5695327
:10C82000C4F87C5B4FF050250020DFF850E2DFF8C1
:10C8300050C2C4F8A02BC4F8A47B02F5A04207F5AF
:10C84000A047C4F8A86BC4F8AC3B06F5A046A3F516
:10C850004853C4F8B05B04F52D65C4F8B42BC4F894
:10C86000BC6BC4F8DC3BC4F864EBC4F86CCB024688
:10C87000C4F8B87B2B4684F8E40B402683F81C21CF
:10C88000A3F822210132042AC3E9496083F81D116B
:10C8900083F81F01C3F8300103F12803EED1002211
:10C8A00011462B46402083F87423A3F87A230132E3
:10C8B000042AC3E9DF0183F8751383F87713C3F8FB
:10C8C000881303F12803EED14FF0A04362489A6821
:10C8D00022F001029A60DA6842F04002DA6007F062
:10C8E000FDFE94F8D93A0022212161F317420BB1E1
:10C8F00042F4801294F8D31AD4F8DC3A01299A63EE
:10C9000000F0E380DA68D4F8DC6BD4F8E00AC2F314
:10C91000076121F0600141F0400161F31F620021D5
:10C92000DA603160026861F3CC22026094F8DB2A9D
:10C93000012A00F0B7801021484808F021FA474842
:10C9400008F004FAD4F8E00A94F8D13A00224FF043
:10C95000FF31026142618161C26153B305F1140785
:10C960003F4E114607EB83074FEA830C4FF0FF0E53
:10C9700056F8042F1368002BACBF00234FF09043F0
:10C98000B74213601161C2F808E0F1D105F150031C
:10C99000344963440027FF2651F8042F1568002D01
:10C9A000ACBF00254FF09045994215601761966025
:10C9B000F2D1036994F8D31A43F480730129036117
:10C9C00060D0D4F8DC2A28480023936100294FF076
:10C9D000FF336FF0804151615360516114BF0023F8
:10C9E0001023906143F47013916943F4605343F052
:10C9F00008030B43936141F2B8019368615843F017
:10CA0000010393600B689847184B194ADA6068462F
:10CA1000184B009308F092FB02B0BDE8F08100BF14
:10CA200000E100E000380240000002401051002008
:10CA3000003C01404C040020400040010008005030
:10CA400000090050000B005020090050C0050050A4
:10CA50000010005000300050EC5B0020E05B002034
:10CA6000F45B0020305C00200008008000ED00E056
:10CA70000005FA05430200010804010020050050EA
:10CA800060050050D4F8DC2A144B03636FF080413A
:10CA9000134D00234FF0FF3093615161506051619D
:10CAA00095619FE701680F4A0F4E41F00301016055
:10CAB000802159629E62C3F80421E022C3F8082154
:10CAC000C0F24002C3F80C2135E79A6822F03E011B
:10CAD00041F02A0161F307029A6013E70301810024
:10CAE00000080080A00040008000200010B51A4C13
:10CAF00014F8330CC0B9194B83F8B100C3F8B40073
:10CB000014F8303C012B05D0022B21D054F82C3CDA
:10CB10001BB910BD124B44F82C3C12495B68BDE8B0
:10CB20001040A1F10C00184744F04EF914F8312CD4
:10CB30000A49003A18BF012281F8B120C1F8B400B7
:10CB40000028DDD01F22C280202140F00BFAD7E759
:10CB5000054B44F82C3CE0E708620020281E00202A
:10CB60008C040020E06100206804002091B10A6B71
:10CB7000824214D9144B5A69914220D34C399142C4
:10CB80001DD30B6B9842F9D38B6B9842F6D80B46AA
:10CB9000184670470C4B59690A6B904212D30B68C8
:10CBA0000BB9F5E70A6B90420B4602D38A6B9042B1
:10CBB000EED951F84C3F002BF4D1184670470023B2
:10CBC000184670470A46D9E7086200202DE9F04769
:10CBD000CC0143D10346224A43F8082B4FF0FF32E1
:10CBE0004260022418467E26DFF87880D8F8189034
:10CBF0002644013E051D49466FF070474FF0010A7B
:10CC000008E0A3421CD0631C45F8043C321B1C46C0
:10CC10000435CAB10B6BA34202D88B6BA34204D27A
:10CC20002046FFF7A3FF014690B10A794B6B002A1B
:10CC3000E7D1A34204D0E6D245F8042C631CE5E713
:10CC400045F8047C631CE1E7C8F81810BDE8F087DC
:10CC500045F804AC321B631C4946D8E78026C3E77D
:10CC6000F8FFFF0F0862002070B4447941BB0368ED
:10CC70004FF400524FF40076202502213CBB1A8C61
:10CC800022F001021204120C1A841A8B188C22F062
:10CC9000F30280B2120420F00A00120C014342F0A9
:10CCA000010241F001011A8319841A8B22F00C024F
:10CCB0001204120C1A831A8B92B270BC1A8370473A
:10CCC00000220368164615461146002CD7D0042CC6
:10CCD00021D0082C38D0198C21F480510904090C7A
:10CCE00019849C8B1D8C45F6FF7040F6FF4128404F
:10CCF0002140024342F4805241F4807199831A84A6
:10CD00009A8B22F440621204120C9A839A8B92B28C
:10CD100070BC9A8370471A8C22F010021204120C15
:10CD20001A84188B198C89B240F6FF4221F0A001B9
:10CD300002400D4342F4807245F010051A831D84B1
:10CD40001A8B22F44062B3E71A8C22F48072120428
:10CD5000120C1A84998B1A8C21F0F30192B20904F7
:10CD600022F42062090C324342F4807241F0010146
:10CD700099831A849A8B22F00C02C4E738B50E4DC1
:10CD80000446006808F028FBD5F8BC242046520869
:10CD90004FF6FF713FF05CFA20460021FFF764FF79
:10CDA000064BC5F8283D05F6285120460022BDE86F
:10CDB00038403FF091B900BF202F002055130208E2
:10CDC000036870B55E6A26B133460522BDE870403F
:10CDD000184704460D464E1D00E023689B68204618
:10CDE00098470028F9D0236815F8011B1B682046D6
:10CDF0009847B542F1D170BD036870B55E6A26B13F
:10CE000033460822BDE87040184704460D4601F13C
:10CE1000080600E023689B68204698470028F9D060
:10CE2000236815F8011B1B6820469847B542F1D1CD
:10CE300070BD00BF0A44914217D010B40139541E8E
:10CE400011F8013F08225840430010F0800F08BF3E
:10CE5000400083F0D50314BFD8B2C0B2013AF3D179
:10CE6000A142EDD15DF8044B704770472DE9F047C2
:10CE7000164D0746002095F9259005F12C0684B043
:10CE800007EB010805F5337504464FF0B60A336821
:10CE9000ABB193F83830142B11D019F1020F01D037
:10CEA0004B450CD1002269463046CDE90244CDE91C
:10CEB0000078ADF808A08DF80D4034F0D3FDE036D1
:10CEC000B542E4D104B0BDE8F08700BF086200209D
:10CED0002DE9F0479AB0DDE9226ADDF8909004462A
:10CEE0000D461746984602E0206841F045FA206852
:10CEF00041F04AFA0028F7D10146642201A867F000
:10CF000084FB264B8DF80450CDF85CA00293002DD5
:10CF100040D0AB1E012B3FD9042D14BF00220322A9
:10CF20001F4B0396D3F884308DF805201E4401234F
:10CF3000CDE9059404968DF85B3037B14246394609
:10CF400007A867F001FB8DF85A80164E96F80E93ED
:10CF500000231893B9F1000F19D196F80D0364223C
:10CF600002FB006001A900F5447067F0EDFA0123AF
:10CF700086F80D9386F80E33236843B143463A464C
:10CF8000294620461AB0BDE8F04712F017B81AB08B
:10CF9000BDE8F0870522C3E70222C1E7D464002080
:10CFA000202F0020086200200C480D4BD0F8901371
:10CFB00010B40C4CC0F880338A1E2231B0F8AE3366
:10CFC0001B01A4FB03C3DB08A3F5B06322F8023FF7
:10CFD0009142F3D15DF8044B704700BF0862002016
:10CFE000517E0208CDCCCCCC70B5084C251D2E4608
:10CFF00014F8010B37F026FA28B1037805F8013B45
:10D00000B442F5D170BDFF23F8E700BFDC65002016
:10D010002DE9F0471D4F012607F10805B2464FF0F4
:10D020003C094FF0000817F8010B43F0CDFE044611
:10D0300090B180F80690C671FB7803F07F02012A58
:10D0400018D013F0800F20460DD185F8048044F0ED
:10D0500001FB85F805802C600136052E05F10805D9
:10D06000E1D1BDE8F08785F804A044F0F9FA85F82D
:10D0700005A0F0E71B0605D4012120463FF072FF12
:10D08000FB78DEE744F0ECFAF6E700BFE465002049
:10D090002DE9F04FDFF8FC91DFF8FCA183B009F136
:10D0A0000C06012419F8018BB8F1000F00F0C680BE
:10D0B0004FEA1815013D052D08F00F0200F2C1805E
:10D0C0000AEB4503B3F8840040FA02F717F00107B2
:10D0D00000F0D28001239340013B1840554464F096
:10D0E000FBFC95F89030664F184407EBC00704230B
:10D0F0007761FC71BB71002302E0152B00F09E806C
:10D1000003EB43025F49895C41454FEA430B03F15E
:10D110000103F2D15C4B1A4492F85111002900F03E
:10D12000AD8040463FF0E0FA054628463FF0FCFA65
:10D130000378002B40F08280534B5B44042283F839
:10D14000914183F89021002D78D0002F5DD03B686D
:10D15000287A03F13F4202F57E020AEB92224FF059
:10D16000010C92F8982002F01F015209032A0CFAD0
:10D1700001F171D0042A67D0022A75D0B7F804E013
:10D18000BEFA8EF2C2F11F02C2F3CC0103EB8101A1
:10D1900002F007020F6A92004FF00F0C0CFA02FC2B
:10D1A00027EA0C070F620F6A90403843002208629A
:10D1B0004FF0010B11460BFA01FC3CEA0E0001F1A5
:10D1C00001011ED118680327974020EA0700186064
:10D1D000D3F800800220904040EA08001860986868
:10D1E00020EA0700986098689860586820EA0C0068
:10D1F000586058685860D86820EA0700D860D86836
:10D20000D860102902F10202D5D1204B204AB3F890
:10D210000414B3F806340091002001340190B2FBED
:10D22000F3F330469BB22946E4B233F039F80123D8
:10D23000092C737406F118067FF434AF03B0BDE80F
:10D24000F08F0027776156E7DFF850C0DCF8302018
:10D250000A43CCF8302091E7DFF840C0DCF84020EA
:10D260001143CCF8401089E7DFF830C0DCF84420E7
:10D270001143CCF8441081E777613CE70D4654E751
:10D28000DC30002070300020202F002008620020B9
:10D2900040420F0010660020AC46070800380240EC
:10D2A00070B5044684B04FF4004039F035F880B3CF
:10D2B00000234FF4E131032590F904000293CDE9F6
:10D2C00000151A464FF4004139F083F8124BC3F8A9
:10D2D000D404F0B1012C40F6980208BF4FF49662D6
:10D2E0000E480F4DA3F8E0244FF461710D4AC3F8C6
:10D2F000EC040A2683F8D844C3F8DC64A3F8E214EB
:10D30000A3F8E414C3F8E854C3F8F024012004B0EF
:10D3100070BD0020FBE700BF08620020F113020887
:10D3200015FF010809FF01082DE9F041214E224FA8
:10D3300096F8133587F8903E06F5A26607F69465D1
:10D3400000244FF0050816F8010B20BB28600134BB
:10D35000032C05F10405F6D197F8901ED7F8940E2A
:10D36000C94301F0010144F081F997F8901ED7F804
:10D37000980E81F00201C1F3400144F077F997F86B
:10D38000901ED7F89C0E81F00401BDE8F041C1F376
:10D39000800144F06BB943F017FD0134012128608E
:10D3A000E3B210B180F80680C37128683FF0DAFD5F
:10D3B000CEE700BF08620020202F00202DE9F041B9
:10D3C0002A4C2B4DB4F81865A5F8A06E82B0EEB9C2
:10D3D00094F8140543F0F8FC94F81525C5F8A40E4C
:10D3E000003A18BF012285F8A22E48B194F816150C
:10D3F0002B22002914BF11210121C2803FF0B2FD70
:10D40000002002B0BDE8F04145F058BC94F8148506
:10D41000002240462B213FF0BDF90746404643F02D
:10D42000D3FCF8B1F7B12B22C5F8BC0EC280397A13
:10D43000FCF7A4F84FF000080E4AB2FBF6F3C3F372
:10D440004F0000909BB23946CDF8048005F6A860E5
:10D45000A4F81A6532F024FFD5F8A83EC3F800807E
:10D4600085F8B98E02B0BDE8F08100BF08620020E7
:10D47000202F002040420F002DE9F84F254C94F852
:10D48000283584F81C3504F21F57002604F23C545A
:10D490005FFA86FB0BF101085FFA88F8012117F8A3
:10D4A000010F42460E448A463FF074F94FF00009DE
:10D4B000054640B3387804F80E9C04F80D9C04F837
:10D4C0000FBC04F810AC44F8045C43F07DFC18B1C8
:10D4D00080F806A080F80780297AFCF74FF80E4AFA
:10D4E000002128463EF0B4FE0C4B23600C4B221D5D
:10D4F00021462846C4E901393EF0EEFD69792868E5
:10D500004A4632F049FE082E04F11C04C0D1BDE8A1
:10D51000F88F00BF0862002040420F00D1010408CC
:10D5200055C4030870B52C4C2C4B94F85406C4F821
:10D530004C3600220221C4F80C26C4F81026C4F888
:10D540001426C4F84826A4F850263FF023F90028F2
:10D5500041D0234B0668054603F1C0015A7C12B145
:10D560005A6896422BD018338B42F7D1002394F897
:10D570005406C4F8385584F82C3543F025FC08B11E
:10D580000223C380297AFBF7F9FF2846154A0021B8
:10D590003EF05EFE144A1549C4F83C150026111FE2
:10D5A0002846134BC4F84035C4F844653EF094FD5A
:10D5B000697928683246BDE8704032F0EDBD3046EA
:10D5C0005DF074FD328D0B4992B2531CB0FBF3F049
:10D5D00081F82803CAE770BD0862002000FFFF0041
:10D5E0003C00001040420F00486700207DC4030843
:10D5F00019C60308880100202DE9F04FC04F87B0FD
:10D600000B460446C022BF480393002166F0FDFF8D
:10D6100097F855368BB9BC4DD5F82432002B7ED007
:10D620000022039883F82C00012183F82D101A633F
:10D6300083F82E2007B0BDE8F08F97F85636002B00
:10D640007CD0DFF8D88298F83C31012B00F0A18023
:10D65000022B00F08180AD4EAB4D98F832C198F8A6
:10D660002E710FCE05F5F87404940FC40FCE0FC4BD
:10D6700096E80700BCF1000618BF0126A44B85F808
:10D680002862072F84E80700C5F8083200F21881E5
:10D69000042F00F25581DFF86CA2DFF88CB200266F
:10D6A000039BB3424FF0030137DD1BF8019B08EBEE
:10D6B000090309F1010793F83341FFB220463A46C6
:10D6C0003FF068F8034620461C46002B00F010810E
:10D6D00043F07AFBCAF8140018B14FF003038371CA
:10D6E000C77198F82F2198F82E31F1B2002A00F076
:10D6F000FD80E27982F00102009220464A4601361E
:10D700005EF070FA002800F0F3804FF00103082E5D
:10D710008AF811300AF1180AC2D1049B9EE07D4EAE
:10D720007D4C0FCE0FC40FCE0FC496E80700A4F1B6
:10D73000200384E80700C5F824327BE7774B039980
:10D7400093F83021704D003A204618BF0122FAF7B5
:10D75000B9FFC5F824025FE798F83231002B3FF497
:10D760007AAF98F82E31082B13D1684E664D684F6A
:10D770000FCE05F5F87404940FC40FCE0FC496E8CD
:10D780000700012384E8070085F82832C5F80872ED
:10D7900099E05D4D624E039BC5F82C320FCE05F526
:10D7A000DE740FC40FCE0FC496E8070098F832C19C
:10D7B0000023BCEB030C84E8070018BF4FF0010CFA
:10D7C0001946584898F82E3187F890364FF44C7225
:10D7D00085F828C287F858168B4666F016FF494B25
:10D7E0000593514B049305F50E76D5F82C325B4525
:10D7F0005EDD049A12F8013B0492434493F83341EE
:10D8000020463FF04DF88146204643F0DDFA98F877
:10D810002F310446002B4DD099F8073083F0010AD0
:10D820000AF0010995F8280209F1010987F85796CD
:10D8300008B18AF0010A002C49D0A17989B14129A7
:10D840000FD03A4B3A493B4AC5F8D831012387F803
:10D850005836C5F8D411C5F8E0210023C5F82432A4
:10D86000DAE6204645F068FA4FEA49110BF1010B60
:10D8700041F009014FF0030371617060F46086F8B4
:10D8800010A084F807B0A37120463FF06BFB1AF09C
:10D89000010F204611D043F0DDFE059AF368536175
:10D8A000BBF1080F02F1180306F1200605939CD185
:10D8B000214BD3E799F807A0B2E743F0D1FEECE79C
:10D8C000082F7FF4E8AE1D4BC5F83032E3E6204662
:10D8D00045F032FA4FEA491949F009010BF1010B01
:10D8E00071617060F46086F810A0CDE7E27903E71B
:10D8F000104B0E4AC5F81432C5F80C220023ADE7D0
:10D90000086200203C00001000110010A04707082A
:10D91000899406087447070864680020202F0020B7
:10D92000CC4707089C6800205E30002045A604080C
:10D9300049A604083DA60408BC1200100D350508D0
:10D9400098F83131064AC5F83022012B05D0022B58
:10D9500006BFBCFA8CF35B09002385F834329AE6E3
:10D960003D350508F8B56D4F97F8A80397F8A9530A
:10D9700043F02AFA60B12D23C380202104463FF0F2
:10D98000F1FA0A203FF082FD204645F0CBF918B9A4
:10D99000D7F8C439DA0000D5F8BD013D092DFBD810
:10D9A00097F8A743D4B9402038F0B6FC0028F3D04C
:10D9B00090F9043097F87913092BC8BF143B3B4406
:10D9C0000A2993F8C84900F09B8093F8D43997F856
:10D9D000A623002A08BF1C46002CDDD0204643F0B9
:10D9E000F3F90546002800F083802D23C380012130
:10D9F0003FF0B8FA0121084643F040FE2B68AA88A0
:10DA00001A833C203FF07CFF0021012043F036FECA
:10DA100097F8A933002B4CD0414C00261FE02B680F
:10DA2000AA885A833FF032FD94F8901ED4F8940EE1
:10DA300001F0010143F01AFE94F8901ED4F89C0EF8
:10DA4000C1F3800143F012FE2B68AA881A83782064
:10DA50003FF01CFD97F8A93301369E4229DA94F86D
:10DA6000901ED4F8940EC94301F0010143F0FEFD6D
:10DA700094F8901ED4F89C0E81F00401C1F380014B
:10DA800043F0F4FD7820002DC9D178203FF0FEFC52
:10DA900094F8901ED4F8940E01F0010143F0E6FDD5
:10DAA00094F8901ED4F89C0EC1F3800143F0DEFD83
:10DAB000CDE797F8A7339BB9D7F8A83303F0FF1346
:10DAC000B3F5803F7FF468AFD7F8C43913F08053C3
:10DAD0007FF462AF87F8A933BDE8F84053F00ABB82
:10DAE00032203FF00DFF284600213FF03BFAE3E7EC
:10DAF00001213FF037FA0121084643F0BFFD80E7DE
:10DB0000D7F8EC395B057FF547AF0AF053F90028E9
:10DB10007FF442AF002C7FF461AF3DE70862002044
:10DB2000202F0020084B03F51F600DC8904202DC37
:10DB3000114602460846984204DD9A42B8BF1A468A
:10DB400010467047704700BF08620020144AD2F8A0
:10DB5000FC09D2F8003AD2F8081A984230B4D2F848
:10DB6000044AD2F80C2A02DC1D460346284691429C
:10DB700002DC15460A4629468842A8BF0846934259
:10DB8000B8BF1346844202DB224604461046984240
:10DB900003DD9C422046B8BF184630BC704700BF2A
:10DBA000086200200B6810B414681B1B03605468E3
:10DBB0004B681B1B43608B6892685DF8044B9B1A93
:10DBC000836070472DE9F047041E0D4612DB092CD7
:10DBD00026DC824A0B468248A0FB0410C00800EBFA
:10DBE0008000A4EB40000021125C1A705970284696
:10DBF000BDE8F08764422D23092C01F8013B24D8AD
:10DC0000764A774BA3FB0403DB0803EB8303A4EB07
:10DC100043030020D35C48700B702846BDE8F087B2
:10DC20006F4B632CA3FB04264FEAD60621DC6B4A1C
:10DC30000B466B49A1FB0601C90801EB8101A6EB6C
:10DC40004101515C03F8011BC5E7654A632CA2FB47
:10DC500004364FEAD60637D8604A614BA3FB060369
:10DC6000DB0803EB8303A6EB4303D35C01F8013B22
:10DC7000C7E7A3FB0627B4F57A7F4FEAD7070DD293
:10DC8000564A0B465649A1FB0701C90801EB810121
:10DC9000A7EB4101515C03F8011BCAE7A3FB07286E
:10DCA00042F20F7294424FEAD80836D84B4A0B46DC
:10DCB0004B49A1FB0801C90801EB8101A8EB410117
:10DCC000515C03F8011BDDE7A2FB0637B4F57A7F50
:10DCD0004FEAD7070CD2414A414BA3FB0703DB08AD
:10DCE00003EB8303A7EB4303D35C01F8013BB4E7E9
:10DCF000A2FB073842F20F739C424FEAD80821D8A2
:10DD0000364A374BA3FB0803DB0803EB8303A8EB7E
:10DD10004303D35C01F8013BDEE7324AA3FB080969
:10DD200094424FEAD90921D82C4A0B462C49A1FB31
:10DD30000901C90801EB8101A9EB4101515C03F81C
:10DD4000011BB5E7274BA2FB08099C424FEAD90902
:10DD500021D8224A224BA3FB0903DB0803EB8303F0
:10DD6000A9EB4303D35C01F8013BCAE71E4AA3FBBE
:10DD7000090394424FEAD30A21D80B461849174A9F
:10DD8000A1FB0A01C90801EB8101AAEB4101515C29
:10DD900003F8011BCAE7144BA2FB09029C424FEA9D
:10DDA000D20A13D80E4B0D4AA3FB0A03DB0803EB80
:10DDB0008303AAEB4303D35C01F8013BCAE70A22C1
:10DDC000BAFBF2F052F022FF0346D7E70A22BAFB71
:10DDD000F2F052F01BFF0146E4E700BFC4E0070881
:10DDE000CDCCCCCC9F8601003F420F0070B43448AC
:10DDF00090F8103AA3F13001092957D800F52164B1
:10DE0000224600F61F2012F8015FA5F13001092912
:10DE100004D88242F7D1002070BC7047141B022C3A
:10DE20004ADD2848002101E010F8013B01EB8101A7
:10DE300003EB4103161A303B022E044603F0FF01A8
:10DE4000F2DC214B03FB01F1A2424FF000030DD99C
:10DE500003EB830314F8016B5B00303B3344A242B5
:10DE600003F0FF03F4D1194800FB03F32E2D06D075
:10DE70001748A0FB032301EB930070BC70470132ED
:10DE800004200024157804EB8404303D6400092D3F
:10DE900000F1FF30A4B202D82C44A4B2013210F039
:10DEA000FF00EFD1642202FB0433E1E700211D46AD
:10DEB00000F521620B46D9E7064C0021C4E700BFFC
:10DEC00008620020196C00208096980040420F00E4
:10DED000ABAAAAAA186C002038B504460D460A461B
:10DEE0000068FF2166F091FB21682944216038BD5C
:10DEF00083B50C461646054636F0B4FC204636F08F
:10DF0000B1FC0021204B0846002E08BF1E4643F0FE
:10DF1000B5FB0021012043F0B1FB284640F034FA64
:10DF2000B0B10121002043F0A9FB284640F024FABB
:10DF30000746204640F024FA0028FAD03946204609
:10DF400040F026FA3846B0470021084643F096FBD9
:10DF5000204640F019FA0028DFD00121002043F0CC
:10DF60008DFB204640F008FA01462846019140F01A
:10DF700007FA01990028F8D0284640F009FA002154
:10DF8000084643F07BFBC8E769450408F0B5002369
:10DF9000C1E90033C1E902330B610268DFF888C0D0
:10DFA00089B004ADC2F385572E4647FA03F0C00787
:10DFB000344604D513F80C0004F8010B264601334F
:10DFC000062BF2D1164CDFF864C0C2F30320002305
:10DFD000205C33708DF81800C2F305370DF1190677
:10DFE00047FA03F0C007344604D513F80C0004F8D0
:10DFF000010B26460133062BF2D100233370C2F306
:10E00000834406ABCDE90134084602F00F0305490D
:10E010000095C2F3031252F0CDF909B0F0BD00BF74
:10E020001CE10708ECE0070824E1070814E10708F1
:10E0300070B5094CD4F8202A054662B10026D4F800
:10E04000200A2D21013646F0EFFCAE42F7DBBDE899
:10E05000704046F0C5BF70BD086200202DE9F04F4A
:10E060005FFA81F9002185B007460846164643F05D
:10E0700005FB0021012043F001FB42F083FE022E4C
:10E080000AD0042E44F6C01818BF4FF49648B9F1D0
:10E09000070F07D900200CE0B9F1FF0F4FF4164825
:10E0A000F5D10326CD4D95F8243A2BB90020C5F8BB
:10E0B000280A05B0BDE8F08F032EC94C0DD0A1444D
:10E0C000002299F8330103213EF064FB0028EDD0D3
:10E0D000C4F80405C3799A07E8D495F8240A84F8AB
:10E0E0001F6D002203213EF055FBC4F808090028EB
:10E0F000DCD0BC4ABC4BC4F8C03402F14800032356
:10E100004FF48061A4F8C434C4F8D404002302F2AC
:10E110004C404FF0010A032EC4F8C884C4F8EC3414
:10E12000C4F8CC14C4F8E034C4F8DC34C4F8D8041F
:10E13000C4F8D014C4F8E834C4F8E43484F8103DCA
:10E14000A4F80CADC4F8183DA4F81C3D84F81E3D9D
:10E1500091460ED0D4F804B59BF8040042F034FE8A
:10E16000C4F80005584615F039FE5146484615F0EA
:10E1700049FE32203FF0C4FB002E5FD1D4F808895D
:10E18000D8F8000007F028F94046984A22213EF0CE
:10E190005FF8974B9749C4F8243D324640463DF01E
:10E1A0009BFFD4F80485D8F8000007F015F98F4AD2
:10E1B0004FF6FF7140463EF04BF831464046FEF7C1
:10E1C00053FD8D4B8D49C4F8283D324640463DF005
:10E1D00083FFC5F8289A4FF0060A022E12D0D5F810
:10E1E000280A40F0D1F868B10121002043F046FA36
:10E1F000D5F8280A40F0C8F80146002840F09A8077
:10E2000043F03CFA384640F0BFF888B10121084697
:10E2100043F034FA4FF0050B4FF00008384640F059
:10E22000B3F80146002840F08E80012043F026FA22
:10E23000042ED4D005203FF063FBCEE7012E09D198
:10E24000D4F808094146FAF74FFCD4F80405FEF764
:10E2500095FDBEE7022E09D1D4F8040515F0ADFDF9
:10E26000D4F808094146FAF73FFCB2E7032E59D12A
:10E270004FF0000A5146624884F820AD402266F013
:10E28000C4F98DF80FA0DFF87CA19DF80F30072BA3
:10E2900009D95448012115F0B5FDD4F808094146C3
:10E2A000FAF722FC95E79DF80F3003EB43030AEBE6
:10E2B000C30393F8453073B39DF80F3003EB43036A
:10E2C0000AEBC3039B6C33B39DF80F30234493F8E0
:10E2D000330100B3002203213EF05CFA8346D0B143
:10E2E00015F06BFD9DF80F3094F8202D03EB4303E0
:10E2F0000AEBC30305EBC2019B6CC1F82C3A9BF8F7
:10E300000730DB0748BF012302F1010248BF81F853
:10E31000303A84F8202D9DF80F300133DBB28DF8B0
:10E320000F30B2E7042E7FF454AFD4F8040515F093
:10E3300044FD85E7D5F8280A40F01EF80146384626
:10E3400040F026F854E7384640F016F895F87A3A47
:10E3500001468BB9242803D14FF0010385F87A3A9E
:10E36000012E04D13846019140F012F80199D5F8F8
:10E37000280A40F00DF851E7012B06D14D280CBFBB
:10E380000223002385F87A3AEAE7022B06D13C28DB
:10E390000CBF0323002385F87A3AE1E7032B10D161
:10E3A0000A2802D985F87A8ADAE7042385F86D0A03
:10E3B00085F86C8A85F86F8A85F86E0A85F87A3A4E
:10E3C000CEE7042B20D195F86E3A85F87B0A4340BE
:10E3D00085F86E3A85F87ABAC2E700BF0862002075
:10E3E000202F0020E0330020F847070840420F00AC
:10E3F000913E0208443C002071120208483C002073
:10E40000346C002008000010052BA9D195F86C3A57
:10E4100095F86D9A95F86E0A4B4509D25A1C2B4413
:10E42000484085F86E0A85F86C2A83F8701A97E7D9
:10E430008842B7D195F87B3A85F87AAAF42B8FD128
:10E44000B9F1000F8CD12421384685F87A9A3FF033
:10E450009FFF4D2138463FF09BFF3E2138463FF05D
:10E4600097FF494638463FF093FFF42138463FF086
:10E470008FFFF42138463FF08BFF032E1BD0D4F8DA
:10E480000405437901689D080223AB40DB439BB23E
:10E490000B828D892B408B810079202115F07CFC2B
:10E4A000D4F804054A4649463DF016FED4F8043532
:10E4B000186806F091FF0022D4F8080911463DF0D3
:10E4C0000BFED4F80839186806F086FF0120F0E545
:10E4D00030B583B04D1C009303688572C2729C698D
:10E4E0000023A04703B030BD03685B6C0BB1022171
:10E4F0001847704770B51D4C0968D4F8805A1C4EF7
:10E50000D4F87C4AD6EDCB7ADFED1A6A491B00EECF
:10E51000901A0168F8EEE00A091B60EEA70A00EE07
:10E52000101A20EEA07AB8EEC00A1C46A0EE007ABF
:10E53000B1EE400AF1EEC77A67EEA67AFCEEE77A12
:10E54000C2ED007A53F0C0F89FED0B7ADFED0B7A45
:10E55000E0EE077AFDEEE77A17EE902A002ABCBFBC
:10E5600002F50C42A032226070BD00BF086200209C
:10E57000880100202C7D8E3FA00CB34500A00C46E6
:10E5800038B50F4C94F89B1A01F03F018B1C0246E2
:10E5900001F10A0584F8993A84F8965A04F6942011
:10E5A00084F8972A083120F065FB254485F8920A03
:10E5B00094F8963A1C44000A84F8930A38BD00BFC8
:10E5C0000862002038B50B4C00250122802120462E
:10E5D00037F08EFE30B194F9040037F0BBFE08B17D
:10E5E000006838BD0135092D04F10C04EDD100207F
:10E5F000F7E700BFC46C002038B5041F00F1080520
:10E6000054F8043FD81780EA430017F0D3FDA54221
:10E61000F6D138BDF8B5C94CDFEDC97A94EDCE7AA4
:10E6200094F8A033B4F8A2732DED028BB8EE478AAC
:10E6300028EE278A002B5FD1D4F8AC3394F8BD23A1
:10E64000002B40F30E8107EE902A9FEDBE6ADFEDAE
:10E65000BE6AF8EEE77AB7EE007AA7EE867AF0EEB9
:10E66000477A07EE103AF8EEC78AB7EE087A87EED7
:10E67000270AC6EEA87A20EE270A64F0C1FC0F280C
:10E68000B8BF0F2094F8A13385B2A4F8A253002B91
:10E6900000F04781AF4234D0B4F8A4339FEDAB6AA9
:10E6A00094F83C6307EE103A07EE905AB8EE477ABA
:10E6B000F8EE677AC6EE076A86EE277A76EE887AF3
:10E6C00037EE087AC8EE276AC8EE077AB6B394F830
:10E6D000A633B4F8A853C4EDD37AC4EDD77AC4ED09
:10E6E000DB7AC4EDDF6AC4EDE37AC4EDE77A002B90
:10E6F0005BD0BDEC028BF8BD94F8A133002B00F089
:10E70000858094F83C63002E40F00381B4F8A43374
:10E71000DFED8E6A07EE907A07EE103AB8EE676A80
:10E72000B8EE477AC6EE877A86EE867A77EE887AF2
:10E7300037EE087AC8EE276AC8EE077A94F8A6631F
:10E74000B4F8A8530023C4F84033C4F84433C4F8E1
:10E750004833C4F85033C4F85433C4F85833C4F8B9
:10E760006033C4F86433C4F86833C4EDD37AC4EDBD
:10E77000D77AC4EDDB7AC4EDDF6AC4EDE37AC4ED89
:10E78000E77AC4F87033C4F87433C4F87833C4F843
:10E790008033C4F88433C4F88833C4F89033C4F8A1
:10E7A0009433C4F89833002E66D1D4F8AC3394F87F
:10E7B000BD23002B40F38E8007EE902A9FED616A07
:10E7C000DFED616AF8EEE77AB7EE007AA7EE867AB7
:10E7D00007EE903AF8EEE77AB7EE086A86EE070A97
:10E7E00086EEA77A20EE070A64F00AFC0F28B8BF6D
:10E7F0000F2080B2A4F8A803002E3CD0A8423FF41A
:10E8000078AF00286DD1BDEC028BF8BDD4F8AC33E5
:10E8100094F8BE23002B40F3878007EE903AF8EE81
:10E82000E78A3D4607EE902A9FED466ADFED466A8D
:10E83000F8EEE77AB7EE007AA7EE867AF0EE477A3E
:10E84000B7EE087A87EE270AC6EEA87A20EE270AE6
:10E8500064F0D6FB0F28B8BF0F2080B2A4F8A40341
:10E8600018E794F8A1330F25A4F8A253002B7FF4E6
:10E8700011AF2846F2E7054694F8BC3384F8F93620
:10E88000002D3FF436AF07EE905A9FED306AD4ED7D
:10E89000F06A2F4BF8EE677ABDEC028B86EE277A92
:10E8A0001946002241F8042B012084F8F8060A607A
:10E8B0009A601A615A619A611A625A629A6237EED4
:10E8C000267AC6EE877AC3ED037AC3ED077AC3EDE5
:10E8D0000B7AF8BD0F20A4F8A80346B30F2D3FF420
:10E8E00008AF07EE900A9FED196AD4EDF06A194A55
:10E8F000F8EE677ABDEC028B86EE277A37EE267A41
:10E90000C6EE877AC2ED007AC2ED087AC2ED047ACB
:10E91000F8BD94F8A633B4F8A853002B7FF4E9AE01
:10E9200043E794F8BE237DE73D460F2096E794F831
:10E93000BC3384F8F9360546A5E700BF0011001086
:10E94000BD378635CDCCCC3D002474494E2DA63D37
:10E95000C8170010D4170010F8B5214C1D270E461B
:10E96000054684F82C7B20F0ABFA002020F04AFA10
:10E97000082020F047FA0E2020F044FA384620F014
:10E9800041FA042020F03EFA042020F03BFA002057
:10E9900020F038FA302020F035FA002020F032FA4A
:10E9A000304620F02FFA002020F02CFA20F074FAE4
:10E9B00004F62D3020F07AF9234670B194F82D2B0F
:10E9C00062B994F82E2B302A00D03AB993F82F2B45
:10E9D00022B993F8303B2B700120F8BD0120FCE7F1
:10E9E00008620020114B10B50446185C14F0AEFC10
:10E9F0000F4800EB8404D4ED007AFDEEE77A0A2399
:10EA000017EE901AB1F5FA6FA8BF4FF4FA61B1F59D
:10EA10007A7FB8BF4FF47A71A1F57A71BDE81040E2
:10EA2000B1FBF3F10920C9B214F0BEBCFCE0070849
:10EA3000486D00201D4991F8102AA2B3F0B40026B9
:10EA400005463346304637461BB991F8104A2D2CFF
:10EA500023D02E2A19D0CA1800EB800092F8104A51
:10EA6000A4F13002092A4FEA40009CBFA0F1300215
:10EA7000A0180E2B14D80133CA1892F8102A002AB5
:10EA8000E2D106B14042F0BC70470133002DF8D00E
:10EA9000CA182A4482F8107ADDE701231E46EBE704
:10EAA0000020F0BC70470020704700BF08620020C3
:10EAB0002DE9F0410C4F0124A0231825E6B2FF2BCD
:10EAC0000BDCC5F11B0103F10108D7F8880BDBB2A1
:10EAD0003246C9B2FFF7FCFC4346013DEFD1013499
:10EAE000052CEAD1BDE8F081086200201FB503AC17
:10EAF0008DF80C30009400238DF80D300CF090FE52
:10EB000004B010BDF8B50546262029F093FC154C3D
:10EB1000014610BBD4F88C0B90F838301E3B012B0B
:10EB200002D894F8993B0BB13FF032FC0E4F00260F
:10EB3000AE420ADBB4F8BA3B0133A4F8BA3B0B4B44
:10EB4000D3F88430C4F8CC3BF8BD17F8011BD4F8D7
:10EB50008C0B3FF01DFC0136EAE7002384F8C83B2C
:10EB6000EDE700BF08620020A26D0020202F0020EA
:10EB700010B58021044605F097FA2046002105F0E3
:10EB800093FA2046BDE8104005F0CEBD2DE9F041D6
:10EB9000B14C94F8E33BC4F8D00B82B088465A2BB2
:10EBA00000F2B980DFE813F0CC00B700B700DC005A
:10EBB000B700B700B700B700B700B700B700B7009D
:10EBC000B700B700B700B700B700B7000F01B70034
:10EBD000B700B700B700B700B700B7003301740043
:10EBE000B700B7007400B700B700B700B700B801AE
:10EBF000B7006201B700B7007C00B7000902B70098
:10EC0000B700B700B7005B00B700B700B700B700A8
:10EC1000B700B700B700B700B700B700B700B7003C
:10EC2000B700B700B700B700B700B700B700B7002C
:10EC3000B700B700B700B700B700B700B700B7001C
:10EC4000B700B700B700B700B700B700B700B7000C
:10EC5000B700B700B700B700B700B700E40194F8F9
:10EC6000E43B9B0700F16982B4F8EA3BD4F8E52B5A
:10EC7000D4F8241C5BBA9BB212BAD0188842C4F8EC
:10EC8000303CC4F82C2C03D905F0CEF9002854DB15
:10EC90000020A4F81C0C0546284602B0BDE8F0810F
:10ECA00094F8283C002B40F0FF8094F9E03B002BC7
:10ECB00031DAD4F8183C08469B689847002840F0A1
:10ECC0001E82B4F8EA0BD4F8E52BD4F8243C40BA01
:10ECD00080B212BA15189D42C4F8300CC4F82C2C1E
:10ECE00007D905F0A1F9002827DBD4F82C2CD4F89B
:10ECF000300CD4F8203CD4F8DC6B03FB00F003FBB1
:10ED000002F20225B042C4F82C2CC4F8300C84F86E
:10ED1000285C00F0CF8094F8F43B5A1CD2B204EB8C
:10ED2000C30305204FF40051042A84F8F42B83F820
:10ED3000F80BC3F8FC1B00F0A0814FF0FF35ABE7E8
:10ED4000D4F8DC3B002BE6D1D4F8183C08469B688D
:10ED500098470546002840F0D281A4F81C0C9BE798
:10ED60003E4B002203F1120103F8012F8B42FBD12D
:10ED70003B4994F81E3C94F8F40B70250D709842B2
:10ED80004FF00C05CD7110D004EBC300013390F8A7
:10ED9000F85B8D70B0F8FC0BDBB2042B40BA8881B5
:10EDA00014BF84F81E3C84F81E2C94F8E73B122212
:10EDB0009342A4F81C2C98BFA4F81C3C00252846BC
:10EDC00002B0BDE8F08194F8E43BDA0700F13E813F
:10EDD000D4F8183C94F8E70BDA6901EBC10102EBB7
:10EDE00081010A79531D834228BF0346A4F81C3CC5
:10EDF000002BE3D0013B1A489BB201331944034472
:10EE000011F8012D03F8012D8342F9D1D6E7154EF3
:10EE1000154F35460823073EC5F10700A4F81C3CF2
:10EE2000002202E092F884211D462B46B54203F8E9
:10EE3000012900EB030217FA82F2F3D1D4F8183C4F
:10EE40004046DB6898470028B8D0AB7863F07F0372
:10EE5000AB70002520E700BF0862002093900020DF
:10EE6000949000209B900020AC460708D4F8183CF2
:10EE7000C74A5B680846111D98470546002840F0C0
:10EE80003E81D4F8243CC34AD4F8201C013B180E20
:10EE90001070180C09BAD37050701B0A08209370B8
:10EEA0005160A4F81C0CF7E6D4F8306CD4F82C2C84
:10EEB000D4F8203CD4F8185CB2FBF3F24FF480573E
:10EEC000BE4228BF3E462D69B249A4F81C7C40468C
:10EED000B6FBF3F39BB2A8470028C0F2BC803346D0
:10EEE000AC4AD4F8D00B812105F012F9D4F82C2CBF
:10EEF000D4F8300CD4F83C3C3244851B9E1BC4F83B
:10EF00002C2CC4F8305CC4F83C6C002D7FF456AF58
:10EF1000032384F8283CBFE69E4E0027334606F1C3
:10EF20000C0203F8017B9A42FBD1D4F8183C40460E
:10EF30005B686A4601A998470546002840F0E980C9
:10EF4000019BBDF80020013B190E52BAF3713171DB
:10EF5000190C1B0A71710820B371022172810C23F4
:10EF6000BDF80220F07031727272A4F81C3C93E676
:10EF7000894E8A4F30460823073EC0F10705A4F8A2
:10EF80001C3C002202E092F88C211846034686427F
:10EF900003F8012905EB030217FA82F2F3D1D4F842
:10EFA000183C4046DB68984700283FF407AFF378E9
:10EFB00063F07F03F37000256EE694F8283C002B85
:10EFC00061D194F9E03B002BFFF6A5AED4F8183CD4
:10EFD00008469B689847002840F09180D4F8183C78
:10EFE0004046DB6898470546002840F0BA80B4F8F0
:10EFF000EA3BD4F8E52BD4F8241C5BBA9BB212BAD6
:10F00000D0188842C4F8303CC4F82C2C00F29F8001
:10F01000D4F8201CD4F8DC0B03FB01F302FB01F253
:10F020008342C4F82C2CC4F8303C7FF474AEB3F5A2
:10F03000805F28BF4FF480530121D4F8D00B554A8C
:10F0400084F8281C9BB205F08DF925E60723544966
:10F05000A4F81C3CCEE694F8F43B5A1CD2B204EB64
:10F06000C30304204FF48851824284F8F42B83F8C0
:10F07000F80BC3F8FC1B7FF460AE002384F8F43B6C
:10F080004FF0FF3508E6D4F8306CD4F8180CD4F8FB
:10F09000203CD4F82C2C4569B2FBF3F2B6F5805F26
:10F0A00028BF4FF480560846B6FBF3F339499BB2AC
:10F0B000A847002862DBD4F82C2CD4F8305CD4F8B4
:10F0C0003C3C3244AD1B9B1BC4F82C2CC4F8305C78
:10F0D000C4F83C3C2DB9D4F8D00B294605F096F97C
:10F0E000DAE5B5F5805F28BF4FF48055ABB2D4F8B0
:10F0F000D00B284A012105F035F90025CCE594F81C
:10F10000F43B5A1CD2B204EBC30302204FF4685103
:10F110000AE694F8F43B04EBC3020133DBB20220AD
:10F120004FF46851042B82F8F80BC2F8FC1B22D074
:10F1300084F8F43B4FF0FF35AEE594F8F43B5A1CED
:10F14000D2B204EBC30305204FF41051ECE504F0F8
:10F150006BFF0028FFF6F1ADD4F82C2CD4F8303C2E
:10F1600056E794F8F43B5A1CD2B204EBC3030220D6
:10F170004FF41C51D8E584F8F47BDEE594F8F43BB9
:10F180005A1CD2B204EBC30304204FF440716BE766
:10F19000286E0020949000209B900020AC46070829
:10F1A0002848070810B51C2041F00EFE1121044626
:10F1B0003DF0D8FE204642F04DFAC8203EF0A0FBBC
:10F1C0002046BDE8104042F04BBA00BF08B5002011
:10F1D00041F0FAFD054BC3F8440C08B12A23C38063
:10F1E000BDE8084040213DF0BDBE00BF08620020E0
:10F1F0002DE9F04FB34CD4F8DC3A5A69D2078BB002
:10F2000002D50BB0BDE8F08F5A699B6912EA030A78
:10F21000F7D0CAF307431AF4002F009340F002819D
:10F22000009B5D0743D41AF0020F5FFA8AF503D002
:10F23000D4F8DC3A02225A61BAF1000FC0F211820E
:10F240001AF4006FCAF3072740F084812E0708D50F
:10F250009D4B9E48D3F83C339847D4F8DC3A0822BB
:10F260005A61ED0600F1E981F80600F1A981B906BD
:10F2700000F12E81009BDA0609D5934B9348D3F811
:10F280004C339847D4F8DC3A4FF480125A61009B13
:10F290009B06B6D58C4B8D48D3F850339847D4F89D
:10F2A000DC3A4FF400125A610BB0BDE8F08FD4F88D
:10F2B000E02A9369D26913401FFA83FBBBF1000F68
:10F2C000B1D0DFF80882CDF80CA045464FF0000918
:10F2D00009E05FEA5B0B09F1010908F1040805F197
:10F2E000280500F0DA811BF0010FF2D0D4F8E01A03
:10F2F0005FFA89F708694A6B04EB8703FA40D3F891
:10F30000E83AD2019B68D2B202431A40D007D3B286
:10F3100016D54B6BD8F81820012000FA09F023EA23
:10F3200000034B63684B6948D3F834330121916083
:10F330003946984794F8D36A012E00F0FE810123E4
:10F340001A0703D5D8F8182008239360DE0603D5E2
:10F35000D8F8182010239360580603D5D8F8182041
:10F3600040239360990703D5D8F8182002239360AF
:10F370001A06AED5D5E94C60D5F82431D8F818C0B6
:10F38000311A8B42DCF8182028BF0B46033392B2A7
:10F39000B2EB930F9DD9D4F8E02A323704EB870300
:10F3A000CDE9019890469946B04238D2BEB3D5F81F
:10F3B000241194F8D33AD5F82821371AB94228BF36
:10F3C000394601F1030E4FEA9E0E83B98FB203371F
:10F3D000BF10D9F8D8AA0AD0013352F8040BCAF8E2
:10F3E00000009F42F8D1D5E94C60D5F82821DCF81F
:10F3F000183008440A44B042C5F82821C5F8340141
:10F400000AD195F81C11D8F83420012707FA01F128
:10F4100022EA0102C8F834209BB29E45C4D3DDE93C
:10F42000019856E7D4F8E03A9D69DB691D402D0C40
:10F430003FF4F6AE04F52D66DFF88CB0B046B14669
:10F44000002708E06D0807F1010706F1040608F13E
:10F4500028083FF4E5AEEB07F4D5F9B204EB8102DE
:10F46000D4F8E03AD2F8242B92685B691A40D007AE
:10F47000D3B218D594F8D30A726D012398429360E1
:10F4800007D11269D8F87C33C2F312029B1AC8F86C
:10F490008C33DBF830334846984794F8D33A012B45
:10F4A00000F0598101239A0702D5726D02239360FF
:10F4B0001B07C7D5DBF8383348469847736D0822D9
:10F4C0009A60BFE71051002088010020E05B002017
:10F4D000D4F8E03AD4F8E81A9A680868C2F341020E
:10F4E000022A08BF03224FF0000514BF65F30A008B
:10F4F00062F30A0008605A6842F480725A6006A8F3
:10F5000006F018F8D4F8DC2AD4F8E00AD368C04929
:10F51000079D6FF38D23D3608068C0F341000144E1
:10F5200091F89411032900F0D180BA49BA48012614
:10F53000294484F8D26A81424FF04006A4F8D46A84
:10F5400000F217810E2161F38D234FF40051D36037
:10F5500051618FE6B14B94F8E22BD3F84433B048B5
:10F5600000218DF817108DF817209847D4F8E01A6D
:10F57000D4F8DC2A94F8DA3A88684FF400615161D3
:10F58000002B3FF463AEC3077FF560AE94F8E53B14
:10F59000012B7FF45BAE9DF81730032B7FF456AE42
:10F5A000D4F8DC3B9F491A6842F001021A601A68DD
:10F5B00042F003021A600B6943F006030B6145E653
:10F5C000D4F8E02A964853684FF0000823F001036E
:10F5D0004146536005F0D4FB94F8D16A414656B1D8
:10F5E000914BFF2203EB860653F8045FD86BAA60A9
:10F5F0009E428260F8D1D4F8E03A89484FF0FF3259
:10F600009A614FF00112DA610B2262F3070162F393
:10F610000708C3F8148019611A686FF30A121A6098
:10F6200005F082F8D4F8DC2A7C4B7D48D3F84033CF
:10F630004FF480515161984719E6D4F8DC3A9A6941
:10F6400022F010029A611A6AC2F34340022802F0C3
:10F650000F0146D0062823D09A6942F010029A6121
:10F6600002E694F8DA3A3BB1D4F8DC2B136823F0C5
:10F67000030161F307031360D4F8E02A6749536874
:10F68000D1F84813664823F0010353608847D4F843
:10F69000DC3A4FF000425A61D2E5DDF80CA0C2E539
:10F6A000D4F8A05B614E286801EB810104EBC10135
:10F6B00041F29C0CC2F30A1244F80C00D1F85C0E23
:10F6C000024428683060C1F85C2EC5E700214FF481
:10F6D000007084F8D21A0921A4F8D40A61F38D23AA
:10F6E00033E747F6F0701042B6D001EB8100C2F369
:10F6F0000A1204EBC00002F1030C5FEAAC0CD0F874
:10F70000505ED4F8A0EB4FEA810818BF002006D065
:10F710000130DEF8006045F8046B8445F8D14144BF
:10F7200004EBC101D1F8505ED1F85C0E15440244DF
:10F73000C1F8505EC1F85C2E8EE7B9F1000F7FF47E
:10F74000FEAD94F8E13B042B7FF4F9AD344804F0AE
:10F75000EBFF3346F4E5002F7FF4A4AE94F8E12BE1
:10F76000052A7FF49FAE4846019304F0DDFF019B1C
:10F7700099E62F48A5F57401A1F51051814203D8EF
:10F780000D2161F38D23E0E62A492B48294481426B
:10F7900003D20C2161F38D23D7E62848A5F18C71A3
:10F7A000A1F54341814203D80B2161F38D23CCE6BF
:10F7B000234924482944814203D20A2161F38D233D
:10F7C000C3E6214921482944814203D2092161F33A
:10F7D0008D23BAE61E48A5F1B771A1F558518142B3
:10F7E00003D2082161F38D23AFE61A491A48294450
:10F7F000814203D2072161F38D23A6E617491848F9
:10F800002944814234BF0621052161F38D239CE602
:10F81000AC460708401E1BFF3F420F008801002036
:10F82000E05B002000ED00E0F45B0020B061002010
:10F83000DFC810002013FBFE20D61300FF6918005C
:10F8400000D3CEFE40771B00C05BB3FEC091210009
:10F8500040AC2700C01D6AFE40E13300803C36FE0C
:10F86000E09C4100704700BF704700BF704700BF79
:10F87000704700BF2DE9F0414FF0FF35324A334861
:10F880002C46002304E001330B2B02F1100215D0AB
:10F89000917A0429F7D103F5B17100EB0111C9790F
:10F8A000CF07F0D4661C116801D0A942EBD21C46E8
:10F8B00001330B2B0D4602F11002E9D1631C02D17A
:10F8C0000120BDE8F081214D04F5B17705EB071368
:10F8D0009988F1B9DFF880802601AB1958F82C2CF3
:10F8E0001B4916691B4A41F2186001EB4421185864
:10F8F0000023B047D0B1022808D141F2CC6205EB19
:10F900000717AB58013B0121AB50B9710020BDE88E
:10F91000F081DFF8448005EB041358F82C2C41F2F9
:10F920001860D268185826019047D6E741F2CC6299
:10F9300005EB0717AB580321B97141F2D061013BC8
:10F940000124AB506C54BCE7B0B6002094A000205A
:10F95000ACA0002075F9000808620020044B41F2B9
:10F96000E472995C09B90121995401225A707047D7
:10F9700094A0002038B5174D174B41F2D0640020F9
:10F98000285504E001300B2803F1100314D053F87C
:10F990000E4C8C42F6D11C78032CF3D16AB10F4B7C
:10F9A00003EB40239A4201D0FFF7D8FF00F5B17076
:10F9B00005EB00100123837138BD41F2CC6100F5E5
:10F9C000B1736A5805EB03130420013298716A5031
:10F9D00038BD00BF94A00020BAB60020ACA0002023
:10F9E00038B5134B00209C7B14B11D688D4205D0A7
:10F9F00001300B2803F11003F5D138BD72B10D4B66
:10FA000003EB40239A4210D0FFF7A8FF0A4B00F502
:10FA1000B17003EB00100123837138BD064B00F574
:10FA2000B17003EB0010827138BD022CECD1EDE710
:10FA3000ACB60020ACA0002094A000202DE9F84F27
:10FA400012F0020E9B4606D028B9FFF787FF022569
:10FA50002846BDE8F88F804C41F638056559002DE1
:10FA60005BD14FF0FF367D4FB146B046B246002520
:10FA70003B68984200F0B68097F80EC0BCF1000FCA
:10FA80005BD0BCF1010F15D105F5B17C04EB0C1C6A
:10FA90009CF807C01CF0010F0CD11CF07E0F09D19F
:10FAA0005FEADC1340F0A880D7F808C0D44501D243
:10FAB000E246A94601350B2D07F11007D8D1751C78
:10FAC00004D1B8F1FF3F00F09F80464641F2C8687C
:10FAD00006F5B17754F80850013544F8085004EBA6
:10FAE000061C41F21C694FEA07184CF8095044F80B
:10FAF000085041F2186904EB07154FF000084CF864
:10FB00000900C5F8048004EB0715AD79042D9CD8D5
:10FB1000DFE805F01A330F334D0004F5C25741F604
:10FB20003C063F68A65907FB0565A84299D3FFF735
:10FB300015FF00252846BDE8F88F2E4601350B2D10
:10FB400007F1100794D1BAE712F0010C70D104EB61
:10FB50000710D51090F80780BBF1030F65F3C718A5
:10FB600080F8078062D94FF6FF7083455B4628BF57
:10FB700003469BB204EB07108380BEF1000F16D042
:10FB800004EB061303F5B0531833987B04280ED00A
:10FB900041F2C8654FF0040C60590130605141F2E8
:10FBA000CC65586083F80EC0635901336351500728
:10FBB00005D504EB0710C37943F00103C371D306E5
:10FBC00008D504EB0714E379C3F34502013262F36D
:10FBD0004603E371224B012503EB46260E602846BF
:10FBE000BDE8F88F05F5B17704EB07164FEA071C5F
:10FBF000B67986B92E4669E7A84601350B2D07F17F
:10FC000010077FF435AF5AE7B9F1FF3F18BF4E46F2
:10FC10007FF45CAF8DE741F2C8682E4654F8085077
:10FC2000013544F8085044F80C506CE76346A1E7EE
:10FC30000C4B0B4953F82C3C0B4AD3F8088001EBD2
:10FC400046210023C04700283FF473AF04EB07149C
:10FC50000223A371FCE600BF94A00020ACB60020F4
:10FC6000ACA0002008620020E1F90008F0B5124DB8
:10FC70002B7841F63002022B0BBF070AC0F3D417D2
:10FC8000C4B200F07F04A85883B00E4600230122BE
:10FC9000384401A9FFF7D2FE01280AD12B78022BA4
:10FCA000019B16BF53F8243033F8143023F070430F
:10FCB000336003B0F0BD00BF94A0002010B514461F
:10FCC00002070B4610D50B4941F2C472581C8B58E1
:10FCD000834204D305D100232360012010BDFFF728
:10FCE0003DFE2060012010BD21461846BDE81040B1
:10FCF000BCE700BF94A000202DE9F0414268C2F3A8
:10FD000008030B44B3F5007F82B004460D4657D379
:10FD100090F91A30591C0AD0304A03F5B17302EB3E
:10FD20000313FF21DA796FF30002DA71817694F917
:10FD30001B305A1C0FD0294A03F5B17302EB031391
:10FD4000FF20DA79C2F34501013921EAE17161F35B
:10FD50004602DA71E0762378022B37D01F4A02F58B
:10FD6000C2531B68B5EB432F4FEA432824DC41F60E
:10FD700048036768D6583E407342AB421CDCAB195F
:10FD8000434511D32169207E01AAFFF797FF01287F
:10FD900012D16768236963614744019B2361A5EB26
:10FDA0000801BF1B67608D192046F8F79DFB20B93D
:10FDB0003D446560012000E0002002B0BDE8F08114
:10FDC00015444560012002B0BDE8F0816168012062
:10FDD0002944616002B0BDE8F08100BF94A000201A
:10FDE00070B5154604460E46FFF786FF50B994F8E5
:10FDF000280028B9022384F82830C4E90B5670BDC6
:10FE0000022070BD1DB12046A847012070BD012011
:10FE100070BD00BF10B4D0E9011390F91A208B42D5
:10FE200038BF0B46511C83600AD0144B02F5B172E7
:10FE300003EB0212FF21D3796FF30003D3718176B4
:10FE400090F91B305A1C0FD00C4A03F5B17302EB2A
:10FE50000313FF24DA79C2F34501013921EAE17184
:10FE600061F34602DA71C4760022436A5DF8044BFE
:10FE70004261426011460361B2E700BF94A00020D6
:10FE800038B544220021114864F0BFFB104B41F605
:10FE900002011A784FF6FF745C52022A41F2E871AF
:10FEA00018BF032203F5C05041F64C055A5441F6E1
:10FEB0000C0441F6010203215D5900F818191021C4
:10FEC0001D519954FFF7A6FF012038BD7CB80020D2
:10FED00094A000202DE9F041B1F904300F2B82B03D
:10FEE0000C461646054632D02846F8F721FB95F910
:10FEF0001B80B8F1FF3F074633D02D4B41F218620B
:10FF000003EB08118A58904211D1183303EB4823B0
:10FF1000A188013109B203EB4113A1802846336067
:10FF2000F8F706FB2060012002B0BDE8F081FFF782
:10FF300015FD2846F8F7D8FA28B1002301203360D0
:10FF400002B0BDE8F081002002B0BDE8F0814FF4BE
:10FF50000071FFF7D1FE0028F5D04FF6FF73A380A4
:10FF6000C2E72846F8F7C0FA0028E2D10FB9FFF738
:10FF7000F5FC38460023112201A9FFF75FFD012897
:10FF8000D7D1019B0B4A9A1A48BF02F2FF12B2F571
:10FF9000B05F4FEA622106D24FFA81F885F81B80E4
:10FFA000002BB5D1C5E7FFF7D9FC019BF6E700BFF1
:10FFB00094A00020ACA0002030B50446C06983B0F6
:10FFC00010B9012003B030BD0D460023032201A962
:10FFD000FFF734FD0128F5D1B4F92030002B03DA06
:10FFE000FFF7BCFC0220EDE7019A012D4FEA431117
:10FFF00002EB431303D0022D12D1E5255554A2681C
:020000040801F1
:10000000DA612278032A04D100221A775A779A7784
:10001000DA77626A5A83C2F30F429A8203B030BD24
:10002000E268DA61EDE700BF10B50378023B012B0F
:100030000446037E02D913F0060F5AD198063AD42B
:1000400094F91A30591C0AD02D4A03F5B17302EB0A
:100050000313FF21DA796FF30002DA71A17694F9C4
:100060001B305A1C0FD0264A03F5B17302EB031361
:10007000FF20DA79C2F34501013921EAE17161F328
:100080004602DA71E076237E1B070BD51C4841F24D
:10009000C873C35C072B01D0FFF760FC41F2C87343
:1000A0000022C254E26A0023237084F82830FAB197
:1000B000BDE81040104700231249E0691A018A5830
:1000C000904206D001330B2BBAD01A018A589042C5
:1000D000F8D10B4A03F5B17302EB0313DA79C2F3DB
:1000E0004501013921EAE17161F34602DA71A7E7BE
:1000F00010BD0121FFF760FF0128F9D1237E9DE7A4
:1001000094A00020ACB6002030B1027822B190F863
:1001100028201AB1002070470120704710B5D0E99F
:100120000142A242C16238BF22460321826080F8A8
:100130002810FFF779FF012010BD00BF2DE9F04F17
:10014000DFF868918A4699F80010DAF80030022941
:10015000174683B0834641F6300240F08B8059F851
:100160000250DEB2A6EB030805EB1325B8444FF4AA
:1001700080729044BB4208F1FF38B8FBF2F875D2A8
:10018000A844032906EB0704A4EB03040CBF802258
:100190004FF48072944228BF1446A8EB050366B959
:1001A00094422CBF0A220B2201A92846FFF746FCE5
:1001B000012809D003B0BDE8F08F0B2201A9284621
:1001C000FFF73CFC0128F5D199F80020DAF800107F
:1001D000022A01F1010321D0A64210D2019906F1B1
:1001E0008042013A081F00EB840001EB820242F8D2
:1001F000043F824203F10103F9D1DAF80010A61B93
:100200007318BBF1010FCAF800301BD09F4205F1F3
:1002100001052BD999F800100026B2E7A642EED2CC
:10022000DDF804C006F10042013AACF1020000EB37
:1002300044000CEB420222F8023F904203F101031A
:10024000F9D1DCE7BB42E1D199F80030022B21D093
:1002500004F18044019B013C4FF0FF3243F824201D
:10026000DAF800309F4205F10105D3D8012003B030
:10027000BDE8F08F59F8022003F07F060329C3F38D
:10028000D415A6EB03081544B84414BF4FF480728C
:1002900080226EE704F10044019B013C4FF6FF729F
:1002A000584623F8142003B0BDE8F08F94A0002036
:1002B0002DE9F04190F838300446032B51D8DFE89F
:1002C00003F002323B462D4BC0681978E76A03F50C
:1002D000C252032911680CBF80264FF4807601FBBF
:1002E00006F141F2C47C00EB412041F2A87841F2D2
:1002F000AC7E53F80C20E06053F80E0053F8085021
:100300002261A5EB4125A0EB4121901943F808504B
:1003100043F80E1043F80C00C4E90C205FBB626286
:10032000012384F8383016480021FFF745FE0128E4
:1003300011D1022384F83830626B04F130010120BE
:10034000FFF7FCFE012806D1032384F83830002192
:100350002046FFF731FE431EDBB2012B02D9BDE878
:10036000F081022094F82830062B04BF002384F883
:100370002830BDE8F081921B2263D1E794A00020D1
:1003800034B800202DE9F04FDFF8248198F80060A0
:10039000012887B08CBF00230123032E02930C4653
:1003A0000B68154639D0022E62D14FF480724FEAA5
:1003B0001329DFB201920138012823D801220392C8
:1003C0009D421AD9384E06F1880A06F11C0B326894
:1003D0001AB1DBF8001099424ED0DAF80000002381
:1003E0004844092205A9FFF729FB01281FD002284C
:1003F0000FD020B123689D42E9D82560032007B0C3
:10040000BDE8F08F87B1FFF7A9FA022007B0BDE879
:10041000F08F022007B0BDE8F08F80220192C3F375
:10042000D41903F07F07C6E7019A0392C8E7DDE914
:1004300002C1059ADDF804E098F80030022B14D0D0
:10044000032BE6D152F8273023F07043B3FA83F33D
:100450005B0963450F44236823D00B447745236031
:10046000EAD309F101090027C5E732F81730EDE7B3
:100470004FF480720192D2E70C490968013A02EB0D
:1004800041224902B2FBF1F203991344B3FBF1F2AA
:1004900001FB12320AB10B449B1A9D42236096D88D
:1004A000ABE7AB42ABD3A8E73CB80020D4B8002000
:1004B00094A00020F0B5104D2B7841F63002022BAD
:1004C0000BBF070AC0F3D417C4B200F07F04A858CA
:1004D00083B00E4600230322384401A9FFF7AEFA89
:1004E000012807D12B78022B019B0CBF23F8146045
:1004F00043F8246003B0F0BD94A000202DE9F04340
:1005000090F83C30002983B0044614BF022100213A
:10051000042B7BD8DFE803F0030C3C476900FFF7AE
:100520004BFD012870D1626B002A75D184F83C0024
:10053000404EDFF80881404D4FF6F7771DE01FFA77
:1005400080F9B94594BF4FF000094FF0010901A9A6
:10055000B9F1000F46D1FFF789FB0128494650D178
:10056000206BFFF7A7FF01284BD1019B2A6823636B
:10057000013B934228BF13462B603378206B032B3B
:10058000DDD1404594BF4FF000094FF00109DEE78F
:10059000426B04F130010020FFF7D0FD012833D178
:1005A000032384F83C30234BE16A41F2C47003F525
:1005B000C2521D581268195041F2A87741F2AC7628
:1005C000D8596D1A995902FB05F200EB422501EB4F
:1005D000422203F5BD500021DD519A51FFF7ECFC9A
:1005E000012811D1042384F83C3094F82830042BDE
:1005F00004BF002384F82830A36B8BB120469847B2
:10060000012003B0BDE8F0830228FAD194F8283025
:10061000042B09D00220F4E7022384F83C30B8E729
:10062000012003B0BDE8F083002384F828300220C5
:10063000E7E700BF94A00020D8B80020F7FFFF0F25
:1006400038B590F834300446052B46D8DFE803F07F
:100650001F033F101963006B4FF0FF31FFF72AFFB4
:1006600001283AD1E06A002839D1032384F83430D4
:1006700000212046FFF7A0FC01282ED1042384F896
:10068000343094F82830082B2DD0012038BD41F6A5
:100690003803224DEA5800F1300102320120FFF701
:1006A00071FE012824D00238C0B2012815D80523D4
:1006B00084F8343094F82830082B04BF002384F8E1
:1006C000283041F2E5730122EA54022038BDC06AA5
:1006D000216BFFF7EFFE0128C7D0002038BD0223B1
:1006E00084F83430F4E7002384F82830012038BD42
:1006F00005F5C252E3681168D4E90B2003EB4123EE
:1007000041F644016850C4E9033002B96062012334
:1007100084F83430A0E7014DCCE700BF94A000205E
:100720002DE9F04F436883B0C3F308081646002A4A
:1007300000F0E180714B05468946A3F1180B4FF09C
:10074000000AC8F5007495F91A70B44228BF3446FF
:10075000791C28462ED0F7F7EBFE0BEB071341F27E
:1007600018629B58984205D0FFF7F8F8504603B03E
:10077000BDE8F08F614B03EB4720224649464044D9
:1007800063F0E2FE002221462846FFF729FBA2443F
:100790000028EBD02B7E1B0706D5594B2A691B6816
:1007A0009A4201D3FFF7DAF8361BA1444FF0000854
:1007B000C7D1DBE7F7F798FE002849D12846F7F7BD
:1007C000B7FE6968C1F308032BBB21F4FF7323F064
:1007D000010303F50072AB689A422CBF0622072280
:1007E0002B7E03F00C030C2B1CD0002301A9FFF778
:1007F00025F90128BAD10198404BC31A48BF03F22A
:10080000FF13B3F5B05F4FEA63224FD257B2AF7612
:100810000028B2D1AAE72B7E03F00C030C2B4FF07B
:100820000702E2D19BF800C0364BBCF1030F1B68F6
:100830000CBF4FF0800C4FF4807C03FB0CF34FEAAD
:10084000432C0CF1FF3C0CEA0101A3EB5123CDE753
:100850002B7E1A072ED59BF800102A4B95F82820DE
:100860001B6803290CBF80214FF4807103FB01F347
:10087000062A4FEA43233FF479AF234908688342AD
:1008800030D891F83D30002B7FF470AF002A7FF410
:100890006DAF6B6985F83820062185F82810EB626A
:1008A0002846FFF705FD012888D05FE7FFF756F8D7
:1008B0000198ACE7154B1A78002A7FF457AF95F8EA
:1008C0002820002A7FF452AF082185F8342085F8CB
:1008D0002810D3F85F206B692846C5E90B32FFF773
:1008E000AFFEE0E741F2E573012250460BF803202A
:1008F00003B0BDE8F08F924638E700BFACA00020FF
:1009000058B80020D4B800203CB8002079B80020A6
:100910002DE9F04390F8384083B00546032C00F2EF
:100920009F80DFE804F0021A890BFFF789FE012897
:1009300011D002280BD1032385F838302B6C00200E
:1009400085F82800002B00F0878098470224204675
:1009500003B0BDE8F08385F838002B78022B77D000
:10096000404A6F6841F64803D3581F40C7F34F27EA
:100970002846F7F7DDFDDFF8F08006463F1A0AE06B
:10098000D8F80030013B99454AD2FFF7B5F908B9CC
:10099000FEF7E4FF0136022201A900233046FFF7EB
:1009A0004DF8BC1901281FFA84F94FF400724FF07A
:1009B00000010446CBD1019863F027FEEB694FF4A8
:1009C00000712846002BDBD06B68002BD8D1019B2F
:1009D0004FF020324FF02E0C1A605A6083F800C09E
:1009E000C3F807204FF0100E6C6A1A625A6283F83F
:1009F00020C083F821C0C3F8272083F80BE0EA6BFE
:100A00005C83C2F30F4CC4F30F4483F82BE09C8249
:100A10005A87A3F834C0D8F80030013B9945B4D3C5
:100A2000C3EBC35359022846FFF766F908B9FEF72E
:100A300095FF022385F838302B6C002285F828209A
:100A400063B1284698470124204603B0BDE8F083EF
:100A50006F68C7F34F278BE7022478E7012476E716
:100A6000002474E794A00020D4B800202DE9F04FB2
:100A700090F8303089B00446042B00F2A880DFE8FB
:100A800013F0A900B20005008A00E800B64D41F657
:100A90001003EB5C002B40F09A80B44F04F11C096A
:100AA000B84607F1380BBA4601AE324649464046D1
:100AB000FFF710FA012840F018810198002800F093
:100AC000FA800378E52B01D0002BEED1A84A821AD8
:100AD00048BF02F2FF12B2F5B05F4FEA622380F026
:100AE0003C811B01A34A13449A7B042A0CD041F297
:100AF000C86104266A5801326A5041F2CC615A60DA
:100B00009E736B5801336B5041F60202AB565E1C6C
:100B100009D003F5B17305EB0313FF26D979AE5461
:100B20006FF30001D97141F603016B565A1C0ED0C8
:100B300003F5B17305EB0313FF26DA796E54C2F3A4
:100B40004501013921EAE17161F34602DA7120229F
:100B5000002163F05AFD2346019A53F8311F58686B
:100B60005060116019899B7A93721181019B627E9A
:100B7000DA7205A850F074F8BDF81430002B40F07C
:100B80002F8144F28172019903200A82CB810A836A
:100B9000CB8284F83000237E980600F1A98020469D
:100BA000FFF738F92369002B00F0AE80237E03F0B5
:100BB000F70213F00403227640F0B480122A00F00A
:100BC000BA80002384F828302046E36A984709B0A9
:100BD000BDE8F08F6548FFF71DF94FF6FF7201235E
:100BE000228484F83030614F04F11C0801AE04F116
:100BF0003109324641463846FFF76CF901282FD0BB
:100C00000228E4D1584D41F60202AB56591C09D0D6
:100C100003F5B17305EB0313FF20D979A8546FF3E3
:100C20000001D97141F603016B565F1C0ED003F52C
:100C3000B17305EB0313FF20DA796854C2F3450161
:100C4000013921EAE17161F34602DA71042384F883
:100C500030300020E36A2070984709B0BDE8F08F7B
:100C6000019D0B2249462846002D00F087802B78F5
:100C7000002B00F0838095F80BA01AF0080FB8D174
:100C800063F0EFFC0028B4D1637E8AEA0303DB063D
:100C900040F1C780344D41F602016B565F1CC1D054
:100CA00003F5B17305EB0313FF26DA796E5460F395
:100CB0000002DA71B6E73B782F49022B4FF00902A8
:100CC0005046C3D00B78002BC0D1C1E905330A7060
:100CD0008BF800304A6B0B7351F8143CC1E90132B8
:100CE000FFF716FE01283FF4E0AE0228AED06EE713
:100CF000E0690023112205A9FEF7A0FE01283FF4B8
:100D00004EAF09B0BDE8F08F237E19077FF559AFCC
:100D1000154A41F2C873D15C00297FF458AF07210E
:100D2000D1544EE70023E26AA16884F828302046B7
:100D3000FFF756F84BE7626AE06AA0630421C4E952
:100D40000233C4E90B2284F83C30636384F8281032
:100D500063622046FFF75EF839E7FEF7FFFD019872
:100D60006FF00F03BEE600BF94A000207CB8002007
:100D7000ACA00020ACB60020A4B80020474D41F63E
:100D80000202AB565E1C09D003F5B17305EB0313E9
:100D9000FF20D979A8546FF30001D97141F60301FE
:100DA0006B56581C0ED003F5B17305EB0313FF20EF
:100DB000DA796854C2F34501013921EAE17161F33E
:100DC0004602DA71237EDA067FF540AF3448FFF73A
:100DD00021F84FF6FF720223228484F8303056E661
:100DE000304B05A9B3F9482C02A84FF057FF9DF8E6
:100DF0000C309DF80D609DF80A509DF80B20BDF851
:100E000008109DF80E00DB0243EA461342EA451241
:100E1000A1F2BC7143EA500342EA41229BB292B272
:100E2000B1E6A98A6B8B204A43EA014312686362E8
:100E3000EB69A3605202B3FBF2F102FB113109B17D
:100E400013445B1A154DE36041F6020184F819A0C2
:100E50006B565E1C09D003F5B17305EB0313FF203D
:100E6000DA7968546FF30002DA7141F603016B56C8
:100E7000581C0ED003F5B17305EB0313FF20DA798C
:100E80006854C2F34501013921EAE17161F3460278
:100E9000DA71032384F830307DE600BF94A000208F
:100EA0007CB8002008620020D4B800202DE9F0436F
:100EB00090F82830013B83B00446082B41D8DFE886
:100EC00003F048054D525865406A4300384B466868
:100ED000056B41F6480103F5C2525F58136837406D
:100EE000EA19B2EB432F4FEA432816D258E02169A2
:100EF000207EFEF7E3FE012823D1256B6668236977
:100F00006361A5EB08053D444644F61B019B666002
:100F1000A84525634F46236142D82046F7F7E4FAF7
:100F200001AA81460028E2D06668A368E26A9E4270
:100F300038BF1E460023A66084F828300AB1204638
:100F4000904703B0BDE8F083FFF7E2FC03B0BDE8D3
:100F5000F083FFF78BFD03B0BDE8F083FFF764F883
:100F600003B0BDE8F0830021FFF7C8FA03B0BDE885
:100F7000F0830121FFF7C2FA0128E2D10023216C9E
:100F800084F828302046FFF7BFF8DAE7FFF790F93A
:100F900003B0BDE8F083FFF753FB03B0BDE8F08377
:100FA0002046F7F7A1FA0028BFD12E446660BCE7BF
:100FB00094A000202DE9F04782B0054602AF184604
:100FC0001C460E46904660F0D9F8083020F0070025
:100FD000ADEB000D0DF1080A013CD14614F8013FBC
:100FE0005BB989F800304246CDF800A0314628466A
:100FF00042F0E0F8BD46BDE8F08718464FF09EFC91
:10100000C3B2A3F120023F2A88BF202309F8013B85
:10101000E4E700BF2DE9F04704460D469046002165
:1010200044221E46089F63F0F0FA01234FF6FF7238
:101030002676628384F828302B782E2B4CD02E46CF
:1010400004F1310A307804F1390968B12E280BD047
:101050004FF074FCC0B20AF8010BCA4506F1010654
:1010600007D030780028F1D120200AF8010BCA45BA
:10107000F7D130782E2808BF707804F1380908BFFE
:10108000013604F13B0A58B14FF058FCC0B209F8E0
:10109000010FD14506F1010607D030780028F3D1C1
:1010A000202009F8010FD145F7D118F0100F14BF17
:1010B0000323012384F819802370E7622B782E2BF9
:1010C00026D16B7823BB0323204684F83030FFF70A
:1010D000CDFC2046BDE8F0876B78002BAFD1114BDB
:1010E00041F2F47241F60C0041F2F0719A5818582E
:1010F0005958E26041F601026062A1609A5C627632
:1011000041F2E8729B5C2370E7622B782E2BD8D0DB
:101110000023204684F83030FFF7A8FC2046BDE8C5
:10112000F08700BF94A0002010B5114C94F8DA3A73
:1011300023B9104B4FF480225A6110BD0E4A136838
:1011400023F0060313605FF0D9FF94F8DA3A002B1E
:10115000EFD0D4F8E03A9B68DB07EAD5D4F8DC2B73
:10116000136823F0030161F307031360E1E700BF95
:1011700010510020003C014010ED00E008B50121B5
:10118000032004F023F872B650F034FB2DE9F04F41
:10119000CF4CDFF848938DB000270090A4F13705BD
:1011A00004F61D4A54F80B0C002800F0FE803DF0B8
:1011B000EBF80646002800F0D681D9F8843044F8D0
:1011C000073CE0260023A4F10B0B04F8033C7E430C
:1011D00054F80B0C3DF0D8F8002800F0E68054F8E5
:1011E0000B0C3DF0C9F814F8023C5A1E80460B2A3D
:1011F0000DD8DFE812F01F003A00460053008300CC
:101200009B00E30017013701420175018D0124287D
:101210000CD0009A3AB995F82A2B824240F07E8190
:10122000012204F8032C0D2BD2D186E0012304F80F
:10123000023CCDE700234D28C4F8C53084F8CD30FA
:1012400084F8CE3004D0582808D004F8023CBFE718
:10125000022204F8022C84F8C430B9E7032304F80E
:10126000023C022384F8C430B2E704233C2804F88B
:10127000023C0BD0B8F13E0F0CD0002304F8023C26
:10128000A6E70A233C2804F8023CF3D1002304F823
:10129000013C9DE7012304F8013C99E7D4F8C5001F
:1012A000AB190344421CC4F8C52083F8378094F876
:1012B000CD00022A88EA000184F8CD1088D1237875
:1012C000C02BDAD86278FF2A08D1052BD5D90123A3
:1012D00084F8C430072304F8023C79E7A4F8C1205D
:1012E00000229342C4F8C93014BF0523062384F8B2
:1012F000C320C4F8C52004F8023C69E7D4F8C5004F
:10130000AB190344421CC4F8C52083F8378094F815
:10131000CD00D4F8C93088EA00019A4284F8CD1093
:101320007FF456AF062304F8023C51E794F8CD3021
:101330008342A2D10D2304F8023C14F801CCBCF185
:10134000000F40F0F180634B08940FCB04AE86E8A9
:101350000F00D4F8C930D4F8D100ADF82AC0234426
:101360000993B4F8C130ADF8283094F8C3308DF843
:101370002C3001238DF82D30324603AB08A9CDF86F
:101380000CC035F0ABFC48B1049B059394F8C42025
:10139000514B04933146584630F064FB039E0023C2
:1013A00004F8023C002E40F0D6800137032F04F1F0
:1013B000E0047FF4F7AE0DB0BDE8F08FD4F8C500BF
:1013C000AA190244431CC4F8C53082F8378094F847
:1013D000CD2094F8CE00019388EA020284F8CD2053
:1013E0004146D5224FF056FD019B84F8CE00072BD5
:1013F0007FF4EEAEB4F80530C02B3FF63EAFB4F844
:101400000320A4F8C120A27884F8C32000229342CC
:10141000C4F8C93014BF08230923C4F8C52004F850
:10142000023CD5E6D522014694F8CE004FF032FDBD
:1014300094F8CD3084F8CE0088EA0303D4F8C500D0
:1014400084F8CD30AB190344421CC4F8C52083F89E
:101450003780D4F8C9309A427FF4BAAE092304F831
:10146000023CB5E694F8CD30434084F8CD3094F892
:10147000CE3083427FF401AF54E7D4F8C500AA19F7
:101480000244431CC4F8C53082F8378094F8CE007B
:101490000193D52241464FF0FDFC019B84F8CE001C
:1014A000052B7FF495AEB4F80120B4F80330A4F80E
:1014B000C120227884F8C32000229342C4F8C930A6
:1014C00014BF0B230C23C4F8C52004F8023C7FE6AC
:1014D0003F62002044480708848E0120202F00200E
:1014E000D522014694F8CE004FF0D4FC84F8CE000B
:1014F000D4F8C500AB190344421CC4F8C52083F8D6
:101500003780D4F8C9309A427FF462AE0C239CE64F
:1015100094F8CE3083427FF4B0AE0BE7232804BFAB
:10152000022204F8032C7EE6BCF1010F4FF0000606
:1015300002D004F8026C38E7D4F8C9300894234488
:10154000099308A8B4F8C130CDE90A66ADF828308F
:101550002CF0CEFBEDE754F80B0C33F083F954F884
:101560000B0CB04721E714F8033C002B3FF41DAFF0
:10157000D9F8842054F8071C521A632A7FF615AF55
:10158000012B28D0022B7FF410AF54F80B3CC5F888
:101590004C3C012285F84A2CC5F8503C0F4AC5F84E
:1015A000583C4023C5F8542C85F85C3C85F85D0C0C
:1015B0000B48C5F820AAC5F8A0AC43F015FD4FF4C0
:1015C000005035F0B1F9074843F004FD85F8A46CEC
:1015D00085F8A56CE9E6FFF7D1FD00BFE1A5040899
:1015E00034E107086AE10708836D1B6A5B681B78B2
:1015F000FF2B0AD190F8F030002B03F1FF3380F875
:10160000F03014BF0120022070470020704700BF57
:10161000826D136A5B681B78FF2B08D090F8F0305E
:10162000013BDBB280F8F0301BB101207047002095
:101630007047126A5268022013707047034B93F888
:101640002400003818BF0120704700BF881E00200A
:10165000202301480B807047E404002064230148E4
:101660000B80704704050020432301480B8070471E
:101670006805002010B5074CD4F8C800FF2807D033
:10168000054951F8042BF6F761FEFF23C4F8C83072
:10169000002010BDE4040020E8B80020EAE700BF05
:1016A00008B5D0F8E4355B6A9847002008BD00BF54
:1016B00008B5D0F8E4351B6A9847002008BD00BF84
:1016C000D0F8E43510B504461B689847D4F8E835DF
:1016D0009B689847002010BD08B5D0F8E435DB6959
:1016E00003B19847002008BD08B5042290F81211F4
:1016F000D0F8E83580F8131180F81221DB6898479C
:10170000002008BD10B5D0F8E83504461B6998479D
:10171000032384F81231002010BD00BF0B0630B443
:101720001CD401EB810200EBC202002300EB810517
:1017300082F8741382F8753301241A4604FA01F111
:101740006D6D61F31F4201696FF3CF332B60CB697D
:1017500023EA0203002030BCCB61704701F07F0117
:1017600001EB810400EBC404012200EB810500239E
:1017700084F81C1184F81D2102FA01F11A46AD69A2
:1017800061F30F02DFE700BF10B581210446FFF7C8
:10179000C5FF20460121FFF7C1FF024B0020187052
:1017A00010BD00BF306E002010B581210446FFF748
:1017B000B5FF20460121FFF7B1FF82212046FFF748
:1017C000ADFFF6F70BFE002010BD00BF38B50D468B
:1017D00004468321FFF7A2FF29462046FFF7E4FFD6
:1017E000002038BDF0B416460A063AD401EB810554
:1017F00000EBC5052824002204FB0104022B85F818
:101800007413C5F87C6385F8773385F8752304F580
:101810005D7448D0154600EB8107012202FA01F100
:101820007F6D61F31F45D7F800C01CF4004F11D144
:10183000E488204946F0805242F4004242EA834262
:1018400004F00F041C4B42EA845211400CEA0303DB
:10185000194339600269D3692B430020F0BCD3617E
:10186000704701F07F0101EB810500EBC5052824DD
:10187000012204FB0104022B85F81C11C5F8246128
:1018800085F81F31A5F8221185F81D2104F58E7405
:101890000CD0002500EB8107012202FA01F1BF699B
:1018A00061F30F05BFE722711546B4E700252571E6
:1018B000F0E700BFFF87CC13007833EC002310B5AE
:1018C000194604464022FFF78DFF80212046002361
:1018D0004022FFF787FFD4F8E835A078012284F88A
:1018E00012215B689847002010BD00BF70B44B7890
:1018F000012B26D00B784A6900EB83035C6D2568C9
:101900002369D2B18A684A6102F07F0223F400237E
:1019100023F07F0342F4002213432361C378012B99
:1019200004BF0B696361C5F3076363F07B0363F373
:101930001F652560002070BC70478A6802F07F0236
:10194000E4E782694C691568136944B38E68B44250
:101950008CBF06F07F0404F07F0423F4002323F0FF
:101960007F0344F4002443EA040388BF4E611361FB
:10197000C378012B1DD0C5F3076464F07B0464F3C6
:101980001F651560002BD5D14B69002BD2D00269A1
:101990000878516B012383400B435363CAE723F458
:1019A000002323F07F0343F400231361C378012B4A
:1019B000E1D10B780C6900EB8300C5F30763816903
:1019C00063F07B0363F31F654C610020156070BCFE
:1019D000704700BF2DE9F0434B78012B30D00B78D6
:1019E0004C6900EB83035E6D356837691CB38B6807
:1019F0001C44013CB4FBF3F4C4F3090203FB02F3FF
:101A0000C3F312034B61144643EAC44363F31C0758
:101A10003761C378012B04BF0B697361CB78012B4D
:101A200044D0C5F3076363F07B0363F31F65356040
:101A30000020BDE8F0838A680124C2F31203E3E7C3
:101A400091F800804E6900EB880EDEF818C0DCF8D3
:101A50000050DCF8107076B3D1F80890384A06EBE5
:101A60000904013CB4FBF9F402EAC444C6F31202CF
:101A70002243CC7807F060473A43012C174649D0FF
:101A8000CCF81020C278012A55D00269516B03FAB4
:101A900008F30B435363C5F3076363F07B0363F3FE
:101AA0001F65CCF800500020BDE8F0834B7973B37C
:101AB00045F00055B5E707F0604747F40027CC78BC
:101AC000CCF81070C378012B2FD0012CE3D1026920
:101AD0009268D20554BF45F0005545F08055C5F3D6
:101AE000076262F07B0262F31F65CCF80050002BA6
:101AF0009ED1B0B203308010DEF8D04098D0CA68D2
:101B000052F8041B216001339842F9D190E745F067
:101B1000805586E764F35E77CCF81070C378012BAC
:101B2000D5D10A69CCF81420D1E70A69CCF8142081
:101B3000012CB0D1CBE70B69CCF81430ABE700BF78
:101B40000000F81F0E4BDA68D20310D4DA68D10611
:101B50000FD4DA68D20510D4DA6812F0E00F0AD197
:101B6000DB6813F0020F14BF082009207047012022
:101B7000704706207047072070470220704700BF5B
:101B8000003C02400020704700207047104AD06897
:101B9000A8B113699BB188420FD88B4234BF002390
:101BA0000123DBB243B193695161994204D0094BDF
:101BB0009161142083F8CC0070470023F1E7A1F570
:101BC0009C53083BB3F57A7F2CBF00230123E9E740
:101BD000E8B80020E4040020054B5A7F19778A42B8
:101BE00004D0044A5977142082F8CC00704700BF13
:101BF000E8B80020E40400207047704728B1034B88
:101C0000987F012894BF002001207047E8B8002089
:101C100008B5FFF7F3FF50B1054AD37F127F5B0091
:101C200003F00203002A18BF43F001030B6008BD54
:101C3000E8B8002008B5FFF7E1FF10B1014B1B6ABF
:101C40000B8008BDE8B8002070B5FFF7D7FF50B192
:101C50000A4A958C35B1966A0023B3421C4603DBD1
:101C6000002000E00D7070BD02EB44040133A48D30
:101C7000AC42DBB2F1D10B70F5E700BFE8B8002051
:101C800008B5FFF7BBFF10B100230B70137008BD40
:101C90000420704728B1034B93F9CE00003818BFD9
:101CA00001207047E404002008B5FFF7F3FF50B1AE
:101CB000054B93F9CE20012AC3BF93F8D130C3F36B
:101CC00040030B60002008BDE404002008B5FFF7C6
:101CD000E1FF18B1024B93F8D0300B7008BD00BF84
:101CE000E404002070B5FFF7D5FF38B10E4C94F82E
:101CF000D130DB0703D500230B70137070BD0B4D83
:101D000094F9CF3095F83C6093FBF6F301330B70F8
:101D100094F9CF4095F83C1094FBF1F301FB134389
:101D200001331370EAE700BFE4040020E8B80020A4
:101D30000320704770B50A4A92F8403006255E1CB1
:101D4000B6FBF5F405FB146492F84150AC4205D0A3
:101D500002EBC303C3E9110182F8404070BD00BF2C
:101D6000E8B80020002230B504461046914200DC5D
:101D700030BDA35C0825584010F0800F4FEA4003A7
:101D800018BF83F0D503013DD8B2F5D10132EDE79C
:101D900010B5D9B10E4B586F814217DCB2B1DB6B75
:101DA0009A4213DC0B4C013A013903FB012184F800
:101DB000DC1004F1D8000521FFF7D4FF062184F8D8
:101DC000DD0004F1D800BDE81040B3E710BD00BF4E
:101DD000E8B80020E4040020024B93F878300B6050
:101DE00001207047E8B80020024BB3F87A300B802E
:101DF00001207047E8B80020024B93F87C300B704C
:101E000001207047E8B8002000230B7001201370F8
:101E10007047003818BF0120704701207047704795
:101E20000023038083708380C3800381704700BFD9
:101E3000074A084992F87D3009780133DBB29942AC
:101E400082F87D3004BF002382F87D30704700BFE8
:101E5000E8B8002080060010F8B5794CD4F880303E
:101E600083B1784B1B6893F82E305BB1764B94F8B6
:101E70008420A3FB0013012A4FEA931330D0022AD7
:101E800008D002B1F8BD714B9842FBD9012384F808
:101E90008430F8BDD4F8882064329A423ED894F851
:101EA0007D3004EB031393F8FC24FF2A06D0684925
:101EB0000132012083F8FC2481F8DE00FFF7B8FF2F
:101EC000644B1B780122092B84F88420DAD1B4F802
:101ED0007E35614A01339BB2A4F87E355380F8BD4C
:101EE00094F87D105B48C4F888308C2303FB0143D1
:101EF000007883F89E20002384F89A3004F190053E
:101F00000A2202230928C4F88C5084F89B2084F804
:101F10008430B7D1504B01311980F8BD94F89A2024
:101F200094F89B309A42ADD104F18F0004F19805EA
:101F3000002310F8012F082153405A0013F0800F9E
:101F400008BF5B0082F0070214BFD3B2DBB20139D5
:101F5000F3D18542EDD194F899209A4239D194F881
:101F60007D6094F8975094F89830B4F89300B4F8E2
:101F7000952094F891C004EB061743EA052394F8E2
:101F8000925087F8FC1440BA52BA81B292B245EA34
:101F90000C202F4DC7F800151BB294F99010C7F80C
:101FA0000425032E4FF00102A7F8FE04A7F8083518
:101FB00087F8FD1485F8DE2008D8264A12780C2A06
:101FC00029D00D2A02D1244B23F81610FFF730FF39
:101FD0005CE794F87D3004EB031393F8FC24FF2AAC
:101FE00006D01B490132012083F8FC2481F8DE0071
:101FF000FFF71EFF174B1B780122092B84F8842062
:102000007FF440AFB4F87C35134A01339BB2A4F897
:102010007C359380F8BD1149114A91F822100E4881
:1020200003EB830303EB830349089B0093FBF1F36A
:1020300082FB0312DB17C3EBA20320F81630C5E7BF
:10204000E8B8002024130010D34D62103F4B4C0021
:10205000E4040020C4590020C85900204C3000205E
:10206000676666660B4B93F89A1093F89B20914233
:102070000ED010B493F89A20D3F88C40511CD2B2F1
:10208000C0B2C9B283F89A10A0545DF8044B7047EF
:10209000704700BFE8B80020FD2870B522D0F028B6
:1020A00004D0EF2822D00224204670BD114D032019
:1020B000052641282E444FF0000405F1010580F06B
:1020C00080030DD0042B0BD9FFF7E6FF2044B54267
:1020D000C4B2E9D015F8010B412880F08003F1D19A
:1020E0000420F3E7044D0B200426E2E7034D0C2007
:1020F0000626DEE7FCE1070804E20708F4E107082A
:102100000F4B104AD3F88035B2F900005B0707D4B3
:1021100000EB8000400080B200F5C87080B27047CC
:10212000094B0A4AD3F8C430323382FB0312D81762
:10213000C0EBA20080B200F5C87080B2704700BF4B
:10214000E8B80020002F0010EC4A002067666666A1
:1021500000B5062983B00A464FF03203014628BF76
:1021600006220DF101008DF8003062F0EDF9044B0C
:102170006846D3F88435984703B05DF804FB00BF88
:10218000E8B800205E2810B511D05D2805D00D4BB1
:10219000BDE81040D3F8883518470A4CD4F8883584
:1021A0009847D4F888353D20BDE810401847054CC5
:1021B0005D20D4F888359847D4F888353E20BDE8AE
:1021C00010401847E8B8002070B5094E0546D6F80B
:1021D00088355E200C469847D6F8883528469847BB
:1021E000E0B2FFF7CFFFC4F30720BDE87040C9E7B6
:1021F000E8B8002003682DE9F041002B3D4D3E4F2B
:102200003E4EB8BF5B42A5FB0321890D07FB01379A
:10221000C7EB0717BF0096F8923585FB0725FA171D
:102220000446C2EBA555002B57D101EB810101EB10
:10223000810105EB810109B2DFF8BC801320FFF7B3
:10224000C3FF2F4908FB057581FB0531ED17C5EB71
:10225000A11109B21B20FFF7B7FF2368254D002B02
:10226000B4BF53214E212320FFF7AEFF636896F8D9
:10227000922583EAE376A6EBE376A5FB0631890D8A
:1022800008FB0168C8EB08184FEA880885FB083589
:102290004FEAE873C3EBA5552ABB01EB810101EBC3
:1022A000810105EB810109B21220FFF78DFF124B6E
:1022B000134903FB058581FB0531ED17C5EBA11122
:1022C00009B21A20FFF780FF6368002BBDE8F041D8
:1022D000B4BF57214521222076E7C1EB011105EB60
:1022E000810109B2A8E7C1EB011105EB810109B237
:1022F000DAE700BF6BCA5F6B806967FFE8B8002050
:10230000D34D621007B50DF1060211F009FA68B15C
:10231000084BBDF80620B3F8B0159A84914205D059
:102320000549A3F8B025142081F8CC0003B05DF86E
:1023300004FB00BFE8B80020E404002013B5044605
:10234000FFF7A8FC08B300230DF106022046ADF804
:10235000063011F0E5F9C0B10D4C9DF8062094F956
:10236000CE1084F8E320032908BF62F07F024FF00B
:102370000501084808BF84F8E320FFF7F3FC0621B5
:1023800084F8E4000348FFF7D5FC02B010BD00BF9D
:10239000E4040020C305002008B5044BD3F8B405BD
:1023A0003BF0F2FFB0FA80F0400908BDE8B8002029
:1023B0002DE9F04F204B85B04FF0000804461E2059
:1023C00093F800A093F801B09D78B3F80490DF88EB
:1023D0001E7ACDF80480ADF80C8026F02BF818B1E9
:1023E00017B1B9460125C246144A92F8B835D90743
:1023F0000AD492F8BF253AB9012E1BD0022E03D180
:1024000013F0020F08BF01258DF80C608DF804A0B1
:102410008DF805B08DF80650ADF80890ADF80A704B
:1024200001AB03CB1B88206020466160238105B08F
:10243000BDE8F08F3546E7E7986D0020E8B800204A
:10244000144B30B4D3F8E44514B300220F2583F8BD
:10245000EA15090A83F8E90583F8EB15C3F8EC25BA
:10246000C3F8F025C3F8F42583F8E85503F5BD60FB
:10247000012110F8015F01312A440E29D2B2F8D1AE
:1024800083F8F6252046044930BC10223BF04CBFAF
:1024900030BC7047E8B80020D0BE0020034B0021BC
:1024A00083F8F815C3F8FC15CAE700BFE8B80020A8
:1024B00013B504462620019125F0BCFF019920B9EF
:1024C000204602B0BDE81040BAE702B010BD2DE9C9
:1024D000F743B74CD4F8E4350D464BB14FF0020842
:1024E00000264FF00109D4F8E4053BF04DFF58B940
:1024F0000027A37F042B00F25781DFE813F08F0041
:10250000E400F7003D014601D4F8E4053BF034FF58
:10251000D4F8FC355A1C2344C4F8FC2583F8000683
:1025200094F8F835012B0AD0022B11D0002B70D172
:102530000F280CBF84F8F895C4F8FC35D3E7A0F158
:102540007203012B01D9762863D184F8F885CAE794
:10255000102AC8D197490023012211F8010F013236
:1025600003440E2ADBB2F8D194F80E2684F8F865FD
:102570009A42C4F8FC65B6D194F80F36002BB2D15C
:1025800094F80176732F37D0762F0DD0722FAAD101
:1025900094F8032694F8023653EA0223A3D0E360AA
:1025A000B4F804362361A4E794F8032694F80236BD
:1025B00053EA022397D094F8051694F8042694F869
:1025C0000906236242EA012294F80616E17794F89C
:1025D000071684F8121694F80816A4F8102641EA93
:1025E0000021A4F81416616901B96361A38C002B62
:1025F0007FF47FAFA2847CE794F8072694F8063630
:1026000043EA02231AB2002B3FF46DAFA4F816265A
:102610006FE784F8F865C4F8FC6564E7722F44D16D
:102620000123A3770022644B1B78402B2FD1634EEC
:1026300094F812C6A08CA37FB4F810E6338005028C
:102640004FEA0C33217F778005F4706503F4405323
:102650002B434FEA0E1543EA8133EDB22B43276A31
:1026600065691BB2BD4214BF0825002513432B43E7
:10267000704514BF042000201843514B614514BF1E
:102680000221002193F8CC30F3800143B180636FC5
:102690001BB1A36A002B40F09D804A494A481F2283
:1026A00003B0BDE8F04361F0EEBFD4F81836474AF6
:1026B000EB1A934201DC0022B5E77220FFF7EEFE31
:1026C000C4F81856F7E7762F03D10223A377002228
:1026D000A9E7D4F818363D4AEB1A9342EBDD762091
:1026E000FFF7DCFEC4F8185600229CE7344ED4F8FD
:1026F000183696F8CC20EB1A82B3344A934230DD78
:10270000E27FD2071BD46169226A91420ED089B25E
:102710004620FFF7CDFE96F8CC30C4F81856013BA2
:1027200086F8CC300423A37701227CE7A18CB4F88F
:1027300010268A4203D05020FFF7BAFEEBE7217F34
:1027400094F812268A4206D0B1FA81F1490949204B
:10275000FFF7AEFEDFE7142286F8CC201C4A934236
:10276000BDDC762FA7D17320FFF798FE0323A37754
:10277000C4F81856002256E7732F9CD0D4F81816C8
:10278000124B691A9942A0DC95E7D4F818360F4A23
:10279000EB1A93428FDD7620FFF780FE0223A377AA
:1027A000C4F8185600223EE70023A3771A463AE7FA
:1027B000E8B80020E8BE0020C4590020C859002015
:1027C000E40400206FE10708C90500203F0D030065
:1027D0003F420F00334DD4F81C662A2385F8E530BC
:1027E0000DF1020220230DF10101304685F8E6309B
:1027F00011F02DF830B19DF801109DF8027051EAEA
:10280000070339D1552385F8E730462385F8E830AA
:10281000202301A9304685F8E93011F012F803466B
:10282000214813B1BDF804209ABB20494DF0C2FDE8
:10283000B4F814761E4D87B30DF10301304611F044
:1028400003F850B39DF803100DF10602304610F066
:1028500067FF10B3BDF8062016493B46BA420CBFCD
:1028600020222A2228464DF0A5FDB4F81636A4F8F9
:10287000203603B0BDE8F083304610F0CDFF394676
:1028800085F8E700304610F0B3FF037885F8E830AC
:10289000BEE709494DF08EFDCAE7084928464DF0CC
:1028A00089FDE2E7E4040020CE05002091E107085D
:1028B000D205002089E107084A23080890E10708AB
:1028C00038B50B680E4D5A1C0A6005221A700B6849
:1028D00095F8CE200C46591C21601A70236895F893
:1028E000D120591C21601A70B5F8D41020464DF043
:1028F0001FFE236895F8D620591C21601A7038BD38
:10290000E40400202DE9F0472DED028BFFF7C2F91A
:10291000C8B31E4B93F9CE00012834DD93F804416F
:102920001B4F9FED1C8A15468E1E02EB44084FF08C
:102930003209454504D1BDEC028B2046BDE8F08745
:1029400037F802AB26F802AF07EE90AAF8EEE70AD6
:10295000B2EE040A60EE880A60F02EFCBCEEC00AFB
:10296000BAF10E0F10EE103A9BB209D91933B3FB2E
:10297000F9F39BB203EB830303EB83035B009BB28E
:1029800025F8023BD5E70024D5E700BFE40400208A
:102990000ABF0020CDCCCC3D38B50D46FFF77AF903
:1029A000044638B10C4890F8D130DB0704D5B0F8B4
:1029B000D2002880204638BD084A90F9CF3092F8DE
:1029C0003C2093FBF2F102FB11320132013100F5A0
:1029D000847010F0B9FEECE7E4040020E8B80020B1
:1029E00038B5134C94F8413094F840209A4219D0ED
:1029F00004EBC3030F49D3E911200023984212DCF2
:102A000093780D4AC4F834065B081370FCF77AF823
:102A100094F8413006210133B3FBF1F201FB12338C
:102A200084F8413038BDD55C01F8015B0133E5E73E
:102A3000E8B80020A26D0020D06D0020A1F5AF53B2
:102A4000B3F5AF7F10B51BD80E4BA3F87A104FF437
:102A50007A7303FB01F400204FF4C87154F0F0FFC7
:102A60002821B4FBF1F101F03F014FF42063012074
:102A7000B4FBF3F441EAC411BDE8104054F0E0BFE8
:102A800010BD00BFE8B8002013B500230DF1060209
:102A90000C46ADF8063010F043FE30B1044B9DF803
:102AA000060083F87C4055F047F802B010BD00BF27
:102AB000E8B80020194B37B593F8782004461D4636
:102AC00051B13AB9D3F83806012283F8782008B119
:102AD0003EF0C6FD03B030BD002AFBD0D3F8380667
:102AE00083F8781008B13EF0B5FD4FF4AF703AF0BE
:102AF00007FF95F97C1000230DF106022046ADF882
:102B0000063010F00DFE9DF8060055F015F8B5F8EA
:102B10007A102046FFF792FFDCE700BFE8B80020FC
:102B20002DE9F04FAC4B1B788BB08146002B40F069
:102B3000BB80AA4ED6F81C56002D00F0B580A84ADE
:102B4000D2F80C4104F0F021B1F1E02F6FD1C2F8BE
:102B50000C31D6F83C26944269D004930593ADF825
:102B60001830A04BC6F83C469A881F78ADF8142060
:102B700093F801C01A7A93F802A08DF810700DF145
:102B800010088DF811C08DF812A08DF8182098E863
:102B900007000DF11C0EAEE803009349AEF80020CB
:102BA000C4F34252895CC4F303428F4202F1010232
:102BB0001F4601D1944508D028468DF81C108DF889
:102BC0001D2010F0C1FDADF82000284611F07DF861
:102BD000032804F0070B37D0042839D001283BD153
:102BE000824B13F80B309A4501A9284618BF8DF87F
:102BF0001E3010F023FE48B1019BC4F3001103F016
:102C000001038B4202D0284610F016FF0A2207A9C2
:102C1000404661F0D2FC50B19DF81E30BDF81C203A
:102C2000BB703A80BDF82030BB804EF063FA96F856
:102C300040A6DFF8B0B104AF96F84036032B7DD83C
:102C4000DFE803F00C3578A5694B13F80B30CAE7C1
:102C5000684B13F80B30C6E70023C4E73946284613
:102C600010F0F2FD044658B107A8FFF7A1FB9DF84C
:102C70001E109DF810308B4260D0284610F088FF5F
:102C800096F84036013303F0030386F840360CB95A
:102C90009A45D1D196F8B835DB0700D524B12B6819
:102CA00049461B68284698470BB0BDE8F08F01A83D
:102CB000FFF77EFB96F8B8859DF8044008F0010800
:102CC000ECB1B8F1000F39D13A460DF103012846B5
:102CD00010F0BDFD044688B307A8FFF769FB9DF817
:102CE0001C109DF803309DF81D208B4203D19DF8E8
:102CF0001030934222D0284610F054FFC0E7B8F1BC
:102D0000000FBDD13946284610F09BFD0446A8B1FE
:102D100007A8FFF74DFBBDF82010BDF810308B421F
:102D20000CD086F8418686F842862B6828469B6937
:102D30009847A5E796F8B835D80701D500249FE74E
:102D400007A9284610F07AFD04460028F6D01E2078
:102D500025F070FB96F8433683428046EED086F825
:102D6000430660B1BBF80630002BE7D1079BD907BB
:102D7000E4D40121284610F05FFE444680E7079B1B
:102D8000DA07DBD50146284610F056FE78E73846CC
:102D9000FFF70EFB97E8070007AB03C31A809DF807
:102DA00010309BB10DF11D0207A9284610F04FFD10
:102DB0000DF11E01284610F047FD0A2207A93846EA
:102DC00061F0FBFB041E18BF012459E708A928463F
:102DD00010F037FDECE700BF526E0020E8B800208D
:102DE000E4040020986D002030E2070824E2070880
:102DF00018E207080CE20708024B0146D3F8440624
:102E00003BF0C6BAE8B800202DE9F041FD2984B0B6
:102E1000044600F0DD80F02900F0BC80EF2900F0CE
:102E20002F814AB10346861803AD002003F8010B39
:102E30009E4205F8010BF9D1994B0B2003F10905CE
:102E400001E013F8010F814200F0C780AB42F8D1D6
:102E50004B1E832B00F29280DFE813F03001370124
:102E600084004101AF01B501480153015F019000A9
:102E700090006501650165017B017B017B015F01BC
:102E80009000900086018E019000900090009000CC
:102E900090009000900090009000900090009000B2
:102EA00090009000900090009000900090009000A2
:102EB0009000900090009000900090009000900092
:102EC0009000900090009000900090009000900082
:102ED000900090009000900090009000A40190005D
:102EE0009000900090009000900090009000900062
:102EF0009000900090009000900090009000900052
:102F00009000900090009000900090009000900041
:102F10009000900090009000900090009000900031
:102F20009000900090009000900090009000900021
:102F30009000900090009000900090009000900011
:102F40009000900090009000900090009000900001
:102F500090009000900090009000900090009000F1
:102F60001D011D014F4B93F89715002900F0628158
:102F700001922DF0F9FC019AADF80C003AB122440F
:102F800003AB13F8011B04F8011BA242F9D104B0F2
:102F9000BDE8F081444F03214FF00508B8440025F7
:102FA00001370CE0FFF778F8064660193246FFF764
:102FB0002BFF70194745C5B2E9D017F8011B41290D
:102FC00081F08003084601D0042BEBD80426ECE7FF
:102FD000364F0B214FF00408E0E7324BD3F8800561
:102FE00080060CD4002AD2D0224403AB13F8011B74
:102FF00004F8011B9442F9D104B0BDE8F08193F8C4
:103000004806870741D52A4D287D052834BF02266A
:103010000326142916D97C39C8B20628E2D8062915
:10302000E0D801A050F821F00D3201080D3201085E
:10303000F7310108E52F01081D3201081732010898
:10304000233201080929CDD90A390A29CAD801A78A
:1030500057F821F0DD31010829320108E52F010878
:10306000E52F0108E52F0108E52F0108E52F0108EC
:10307000E52F0108E52F0108EF3101080D320108A5
:103080000C4F0C214FF0060888E7094B0B29187DDF
:10309000A8D10126C9E0084BD3F8C03003936DE7EF
:1030A000E8E10708E8B80020FCE1070804E20708A7
:1030B000846C0020F4E10708EC4A00200192FFF73D
:1030C0001FF8019AADF80C0058E76A4BD3ED037A6C
:1030D000FDEEE77A17EE903AADF80C304EE701922C
:1030E0002DF042FC019AADF80C0047E7624D95F8CF
:1030F000B835DE0700F1A780B5F87036ADF80C30B2
:103100003CE75D4B5D49B3F9943681FB0301DB1766
:10311000C3EBA103ADF80C3030E7574BB3F896364C
:10312000ADF80C302AE7564BDFED566AD3ED017A45
:103130000C39C9B203EB810393ED137A67EEA67ADB
:1031400067EE877AFDEEE77A17EE903AADF80C302D
:1031500014E7494B03EB4101B1F8723603EB8303EB
:103160005B00ADF80C3009E7434B93F8B83503F03A
:103170000103ADF80C3001E73F4BB3F88C16CD05D9
:103180005ABFCB4303F00103032311F0440F18BFD0
:10319000042311F0020F18BF072311F4806F18BF2A
:1031A0000923ABE70192FEF7ABFF374B019AD3F847
:1031B000C83043EAC0400390E0E62F4BD3F8803696
:1031C000ADF80C30DAE62C4BB3F87016002934D089
:1031D00001922DF0E1FB019A80B2CDE62B8A03EB40
:1031E000830303EB83039B00ADF80C30FAE6EB8915
:1031F000ADF80C30F6E6EB89244903EBC3039B00E2
:10320000A1FB03135B09ADF80C30EBE6B3F84A36CB
:10321000ADF80C30E6E66B680393E3E62B680393A6
:10322000E0E6AB680393DDE6F6B28DF80C608DF84E
:103230000D00D7E6B3F84C069EE6D3F8880680F377
:10324000100080B298E605F25465019225F058F915
:10325000D5ED037A019AFCEEE77A17EE903A9BB22D
:1032600000287FF44BAF0A49096811F0100F18BF0E
:10327000002343E73CBF0020E8B80020676666668D
:10328000002F001000007A44EC4A00201F85EB510B
:10329000F46B002070B5214D95F89836EA181C465D
:1032A00092F89C268AB11E4E09225C1CA6FB0413D0
:1032B0005B0803EBC303E31AE918DCB291F89C1630
:1032C00009B1013AF1D185F8984602681549561CB2
:1032D00006600C2616700268561C066000261670E2
:1032E0000268561C066003EB430603EB860314706A
:1032F00019440D224DF0B0F895F89816084B4A1C69
:10330000A3FB02035B08294403EBC3030120D31A88
:1033100081F89C0685F8983670BD00BFE8B800209B
:10332000398EE33890BF00202DE9F04FC31D85B0E2
:10333000544C03F4FC7300AFADEB030DD4F820370D
:1033400004F5E66B0DEB00025B4506468A46FA6023
:10335000E9462FD094F8701894F871C8D4F824571F
:1033600001F00F0040EA4C1001310DF101088DF819
:10337000000084F87018C7F8088007F10800ED1AFB
:10338000A2EB0808A845194644DD2A464DF064F82A
:10339000D4F82027B968C4F820B72A44A1EB090162
:1033A0004846C4F82427C9B2D04700201437BD4688
:1033B000BDE8F08F94F870C894F87108B4F92A57F2
:1033C0000CF00F0141EA401141F01001002DC9B28B
:1033D000D4F82457B8BF41F080010CF1010C01284A
:1033E00084F870C889F80010A5EB0B0822D1B8F159
:1033F000FE0F3ADDFF2394F8282789F8013007F102
:10340000080009F103031FFA88F1786089F80220A7
:10341000BB6020E042464DF01FF8D4F8202742441C
:1034200048463146C4F82027D04701201437BD460E
:10343000BDE8F08F94F82C37B4F8281789F80130DC
:1034400007F1080009F102037860BB604DF070F8E5
:1034500078681FFA88F14DF06BF8D7E90282D4F84A
:103460002457D4F82037786889E794F8281789F822
:10347000018009F1030889F80210C7F8088007F1F4
:1034800008007CE7E8B8002001297ED9F0B5037870
:10349000644CC3F34115032D83B084F8715803F0D5
:1034A0000F0700F0838013F01003164606D0012D9D
:1034B0006DD0052912D8002003B0F0BD94F844293E
:1034C000002AF8D094F84529013202F00F02BA42DE
:1034D00054D0184684F8443903B0F0BD437884F8DA
:1034E00040394388A4F83C3985884318811DC02D94
:1034F0007DD84D4AC4F8342915444FF0000C012002
:10350000C4F83859A4F83EC984F84409AA1A5B1AC9
:10351000934284F8457965DB444D002A5BD1B4F9C8
:103520003C39FA2B52D0404AD4F83439C4F83839EF
:103530002946151FC4F83429A2F5A276C4F82457E9
:10354000D4F84809C4F820670025A2F5AA7201AB97
:1035500084F84459C4F82857019533F0BFFB013073
:1035600058D0019B0BB100209847D4F82037C4F8FD
:1035700024370120C4F8206703B0F0BD4318D4F805
:103580003859D4F83429411CC0E70020704702297B
:1035900091D045788378A4F83C39FF2D1FD10429B8
:1035A00089D94318B0F80350411DA0E700232049F2
:1035B00084F8303704F5E66204F23173C4F8281752
:1035C000C4F82027C4F82437012075E7002EAAD0BC
:1035D00005233370A7E728464CF03EFF9FE74318CA
:1035E000C11C84E711481A464CF036FF63E7114BC3
:1035F000B4F83C09C4F82037032101334FF6F672C2
:10360000A4F82807C4F8243784F83017A4F82A2728
:10361000012051E7D4F820370222591CC4F82017A2
:103620001A709EE7E8B800205CC100201CC2002090
:103630000000F6FF18C000202DE9F0416A4ED6F8D0
:103640001C7684B0044638460D4610F03EFB86F8E2
:103650004C0957B10DF1090202A9384610F0F7F8EC
:10366000002840F0838096F84C090023ADF808301C
:103670008DF80A301A46431EDBB20021FF20FD2BD5
:103680008DF80C20ADF80E108DF80B0003D900203A
:1036900004B0BDE8F0819DF80830042B00F09D8057
:1036A000052B00F09D80032B00F09C80022B00F086
:1036B0009380012B08BF042100F08F809DF8093012
:1036C0009DF80A10D6F81C06013B0DF10E028DF88C
:1036D000093010F025F896F84C39032B7AD0042BDA
:1036E00076D0012B64D0D6F85029029B3F4F9A42E6
:1036F0000DF108084FD023680D22591C21601A7063
:1037000023680022591C21601A7023689DF8082044
:10371000591C21601A7023689DF80920591C2160EA
:103720001A7023689DF80C20591C21601A702368B8
:103730009DF80A20591C21601A70BDF80E10204611
:103740004CF0F6FE23689DF80B20591C21602046A2
:103750001A700721FAF7C0FB98E8030087E8030016
:103760000120C6F8585904B0BDE8F08101A93846D7
:1037700010F064F800283FF476AF38460DF10A01E6
:1037800010F062F800283FF46EAF019B96F84C09E8
:1037900003F001026FE77A68D8F804309A42AAD1A0
:1037A000D6F85839124AEB1A93427FF670AFA2E767
:1037B000104A9DF80A000121002304E00133082B80
:1037C00091D012F8011F8142F8D38DF80A308AE7B0
:1037D000094AEEE7094AECE703218DF808106DE786
:1037E0000121FAE70221F8E7E8B8002038C20020FA
:1037F00080841E0024E207080CE2070818E207088C
:103800002DE9F0412A4C2B4AD4F88036B4F85C7983
:10381000B4F8886682FB0352DB17C3EBA2031FFADE
:1038200083F8474582B00D4603D1B4F85E39B34200
:1038300033D002680190511C342301601370026878
:103840000023511C0160137041464CF071FE019839
:1038500031464CF06DFE019847F6FF714CF068FE62
:10386000019847F6FF714CF063FE019847F6FF712F
:103870004CF05EFE019847F6FF714CF059FE01983E
:103880000221FAF729FB0120A4F85C89A4F85E69FB
:10389000C4F8605902B0BDE8F081D4F86039064A36
:1038A000CB1A9342C5D8002002B0BDE8F08100BF1A
:1038B000E8B800206766666680841E00026810B55E
:1038C0007F21541C0460117002680024511C0160A7
:1038D0000E211470FAF700FB012010BD2DE9F04F06
:1038E000C24B1B68804613F0800083B000F07181EA
:1038F000BF4B93F8480610F0020000F06A81DFF831
:1039000010B39BF81430052B40F26881DBF80030CF
:10391000B84D0093002BB8BF5B42A5FB0342B648ED
:10392000B649920D00FB0233C3EB03139B0085FBEA
:10393000034502EB8202DC1702EB8202C4EBA554C2
:1039400000FB043304EB8204A4B281FB0321DB17E8
:10395000C3EBA111BCB10025A94F2E46A7FB043231
:10396000D20802EB8203A4EB4303E8B2A4469BB265
:1039700080008340BCF1090F94B246EA030605F1CA
:103980000105EBD8340489B2B9B100259C4F2E460D
:10399000A7FB0132D20802EB8203A1EB4303E8B29A
:1039A0008C469BB280008340BCF1090F91B246EA7D
:1039B000030605F10105EBD83443DBF804E08D4D37
:1039C0008D4E8E498EEAEE70A0EBEE70A5FB0032B4
:1039D000920D06FB0200C0EB0010830085FB035034
:1039E00002EB8202DD1702EB8202C5EBA05506FB5B
:1039F000053305EB8205ADB281FB0321DB17C3EB79
:103A0000A111C5B10020DFF8F8C10646ACFB0532B4
:103A1000D20802EB8203A5EB4303C7B2A9469BB2CF
:103A2000BF00BB40B9F1090F95B246EA030600F1A9
:103A30000100EBD8350489B2C1B10020DFF8C0C164
:103A40000646ACFB0132D20802EB8203A1EB430332
:103A5000C7B289469BB2BF00BB40B9F1090F91B212
:103A600046EA030600F10100EBD83543DBF80830E5
:103A7000634A0193002B1846B8BF5842A2FB00309E
:103A8000604E6149030AA6FB0363DB0901FB03F1F6
:103A9000C1EBD00189B2B9B1002691463746A9FBE6
:103AA0000132D20802EB8203A1EB4303F0B28C4651
:103AB0009BB280008340BCF1090F91B247EA030733
:103AC00006F10106EBD8B9B2BBF81070DFB10026E1
:103AD000DFF82CA1B446AAFB0732D20802EB82031E
:103AE000A7EB43035FFA86F938469BB24FEA890990
:103AF00003FA09F3092897B24CEA030C06F1010610
:103B0000E9D81FFA8CF7BBF812303D4AA2FB030636
:103B1000F608632E28BF6326092B63D9002093463D
:103B20008146ABFB0632D20802EB8203A6EB4303CD
:103B30005FFA80FAB4469BB24FEA8A0A03FA0AF3A4
:103B4000BCF1090F96B249EA030900F10100E8D877
:103B50005FFA89F9009B019A002BCCBF39233823E7
:103B60001616BEF1000F26F07F0635DD274A3343D7
:103B7000964543F00206C8BF43F00606D8F8003069
:103B80001622581CC8F800001A70D8F8003000221D
:103B9000581CC8F800001A7040464CF0C9FC214679
:103BA00040464CF0ADFC294640464CF0A9FC40464E
:103BB00039464CF0BDFCD8F800305A1CC8F800203B
:103BC00083F80090D8F800305A1CC8F80020012073
:103BD0001E7003B0BDE8F08F1E43CFE7002003B096
:103BE000BDE8F08F4FF00009B4E700BFF46B002090
:103BF000E8B800206BCA5F6B806967FFD34D621025
:103C0000CDCCCCCCC55A7C0AA0860100FFC99A3B1A
:103C1000846C00202DE9F047AB4B1B68064613F07F
:103C2000800084B000F09E80A84B93F8480610F006
:103C3000020000F09780A64F397D052940F2978059
:103C4000632900F292800024DFF898C289B22546E9
:103C5000ACFB0132D20802EB8203A1EB4303E0B2DA
:103C60008E469BB280008340BEF1090F91B245EAB7
:103C7000030504F10104EBD8EDB2BB68954A82FB61
:103C80000312D917C1EB623189B2002900F0188103
:103C90004FF0000CDFF84CE26446AEFB0132D20874
:103CA00002EB8203A1EB43035FFA8CF088469BB2E0
:103CB00080008340B8F1090F91B244EA03040CF18B
:103CC000010CEAD8E4B2FB8983494FF4F36707FBA0
:103CD00003F7A1FB0737C7F38F1742F20F739F4219
:103CE00049D8CFB10020DFF8FCE18446AEFB0732B3
:103CF000D20802EB8203A7EB4303C1B2B8469BB2E2
:103D000089008B40B8F1090F97B24CEA030C00F11F
:103D10000100EBD81FFA8CF7704BD3E90023134353
:103D20003ED14FF0FF3833681722591C31601A70AA
:103D300033680022581C306039461A7030464CF007
:103D4000F7FB414630464CF0DBFB33685A1C3260CF
:103D50001D7033685A1C326030461C700621FAF719
:103D6000BBF8012004B0BDE8F087992585E7002065
:103D700004B0BDE8F0870021DFF868C10F46ACFB56
:103D80000302D20802EB8200A3EB40039BB28B40FC
:103D90000431102947EA030793B2F0D1BFB2BBE761
:103DA00001A84CF05DFF9DF80810002900F08A8002
:103DB0004FF0000CDFF82CE1E046AEFB0132D208F8
:103DC00002EB8203A1EB43035FFA8CF089469BB2BE
:103DD00080008340B9F1090F91B248EA03080CF161
:103DE000010CEAD84FEA08289DF80910E1B100203B
:103DF000DFF8F0E08446AEFB0132D20802EB82032A
:103E0000A1EB43035FFA80F98A469BB24FEA890926
:103E100003FA09F3BAF1090F91B24CEA030C00F16D
:103E20000100E8D848EA0C089DF80A104FEA082873
:103E3000E1B10020DFF8ACE08446AEFB0132D208ED
:103E400002EB8203A1EB43035FFA80F98A469BB23F
:103E50004FEA890903FA09F3BAF1090F91B24CEA62
:103E6000030C00F10100E8D848EA0C08BDF80C305A
:103E70001B49632BA1FB03214FEA08184FEA51119C
:103E80007FF651AF0020DFF85CE08446AEFB0132E4
:103E9000D20802EB8203A1EB43035FFA80F98A4662
:103EA0009BB24FEA890903FA09F3BAF1090F91B2FB
:103EB0004CEA030C00F10100E8D848EA0C0832E7AC
:103EC0000C4600E788468FE7F46B0020E8B8002036
:103ED000846C002089B5F814D34D621050C20020C4
:103EE0001F85EB51CDCCCCCC08B5A0F10103B3FAC2
:103EF00083F302284FEA531301D0184608BD0F2060
:103F000024F00AFA30B9064B93F8B83503F00103F0
:103F1000184608BDBDE808400F2024F08BBA00BF4A
:103F2000E8B8002030B5104A104B8DB0014682F839
:103F3000F01002F15800069302A900230DF10705C5
:103F40000124CDE9073302938DF8143009938DF8DD
:103F500028300B93CDE9035440F020F8F5F79CFC92
:103F60009DF807000DB030BD881E0020E91501083E
:103F700008B5F5F791FC0A2039F088FA024B186E63
:103F8000BDE808403DF06CBB881E0020014B1B685B
:103F90001B6A1847DC610020024B186808B183696E
:103FA00018477047DC610020024B186808B143696C
:103FB00018477047DC61002010B5074C606D40B1B8
:103FC0003EF0B0FE94F8513013B180F00100C0B261
:103FD00010BD012010BD00BF881E002010B5FFF7E6
:103FE000EBFF0E4C48B194F82430032B10D8237EFD
:103FF0000133DBB2072B237603D9002384F8243066
:1040000010BD074A01231268626184F8243010BD94
:10401000044840F069F9A4F85C00E8E7881E002035
:10402000A42F0020801A060030B40A490A480A78F2
:10403000531CDBB20525042B00EBC20400F8325000
:1040400008BF00234FF404520B7062604FF0FF3042
:1040500030BC7047FC6D0020006E0020037870B407
:10406000FBB10446C0F10106A31914F8015FDBB2ED
:10407000002DF9D101335B00DCB2032513800C70F5
:104080004D7004785CB1022300255A1CD2B2CC5486
:104090008D5410F8014F0233DBB2002CF5D170BC07
:1040A000704702242346E8E70B0617D401EB81038F
:1040B00000EBC30310B400EB81000124002283F85D
:1040C000764383F8741383F87523426D5DF8044BCF
:1040D000136843F4001300201360704701F07F0160
:1040E00001EB810300EBC303012200EB810083F8A5
:1040F0001C1183F81E2183F81D2182691368002B8F
:1041000001DA43F0804343F400131360002070474A
:1041100070B501F07F0505EB850400EBC404282190
:1041200001FB05010126C4F830310023C4E94A220D
:1041300084F81C5184F81D61C4F8343101F58E7186
:104140001DB9FDF7D3FB002070BDFDF743FC002037
:1041500070BD00BF2249F8B5D1F870390F2B04D0DB
:104160005A1CC1F870290020F8BD1E4C2578002388
:10417000C1F87039002DF6D11B4E1C4B3268B2F5D8
:10418000006F17D01B689A4227D017D9C2F5006379
:10419000402B15D9403B02F14005C1F87439012389
:1041A0002370356092B2402311490A448121FFF700
:1041B000AFFFD8E71B6835607BB12A469B1AE7E75B
:1041C0004FF0000502EB0307C1F874590CBF022140
:1041D0000121376092B22170E6E700232370C2E725
:1041E000E8B800209C270020842700208827002092
:1041F000A0270020AEE700BFF8B51D4C2378012BA7
:1042000003D0022B09D00020F8BD01461948D0F890
:10421000743953B923700020F8BD00231A46812158
:10422000FFF776FF00232370F5E7402B11D9124CDE
:104230002268403B02F14005C0F87439256092B213
:1042400040230E4C084622448121FFF761FF0020E5
:10425000F8BD094D2A684FF0000603EB0207C0F8CD
:10426000746908BF02202F6092B208BF2070E8E78F
:104270009C270020E8B8002084270020A0270020E9
:1042800038B5134602250A46C0E94E3380F811516D
:104290000021FFF73DFF002038BD00BF10B50C78AE
:1042A00014F0600413D0202C0AD14B78023B092B68
:1042B00018D8DFE803F01B21171717171717272E39
:1042C00022490122FFF7DCFF0024204610BD4B7875
:1042D000062B24D00A2BF3D01D4B8A78C3F88029F3
:1042E000204610BDFAF744FC0224EEE719490122EA
:1042F000FFF7C6FF0024E8E717490122FFF7C0FFD8
:104300000024E2E74B88124A1B0AC2F87C390024D9
:10431000DBE70F4B8A78C3F878290024D5E74B8870
:104320001B0A222B0CD0212B04D021462246FFF75A
:10433000A7FFCAE7CA880949092A28BF0922F6E760
:10434000CA880749362A28BF3622F0E768C200200B
:10435000E8B8002064C2002060C200203E060020B1
:10436000F405002038B501EB810400EBC4040D46D0
:10437000002184F87453C4F88C1384F87513C4F8BE
:104380008833C4F88023C3782821012B01FB050161
:1043900008BFEDB201F55D7108BFC4F884231DB9F3
:1043A000FDF7A4FA002038BDFDF714FB002038BD4E
:1043B000144B9A6870B5044662B1134A1B7B92F89D
:1043C00084592B4316D081212046FFF76DFE022D24
:1043D00009D070BD0C4B93F8845981212046FFF71A
:1043E00063FE022DF5D12046064ABDE870401F232A
:1043F0000121B7E70121FFF757FE20468121BDE8E3
:10440000704051E6DC6D0020E8B8002070B5094A24
:10441000094D1173094B13600021044629700D23C7
:104420008121FFF775FE2046054ABDE870401F2335
:10443000012197E73C6E0020306E00205553425317
:10444000DC6D002010B5064B597B0446FAF79EFB45
:10445000002800DB10BD20460121BDE81040D5E753
:10446000DC6D00202DE9F041314D2C7834B1012C68
:1044700001D1FFF7E7FF0020BDE8F0812D4FDFF805
:10448000D080B0F8B4337A68C8F804201F2BBA681B
:10449000C8F80820064606D1274B3A689A4202D14E
:1044A000797B01291AD9254A25491378052401F871
:1044B000334001EBC3000133DBB2042B08BF002300
:1044C0004FF4005113701F4B41600222304683F8B5
:1044D0008429FFF76DFF0020BDE8F081BB7B013B25
:1044E0000F2BE0D8FAF752FB002819DB2B78013BA1
:1044F000022BC0D9144B1988B1B1BB68D8F8082079
:1045000088F80C408B4228BF0B46D11A0424C8F807
:1045100008100E4A2C7030468121FFF7F9FDAAE7FA
:104520003046FFF745FFA6E73046FFF76FFFA2E7EB
:10453000306E0020DC6D002055534243FC6D00209E
:10454000006E0020E8B80020246E00209490002027
:104550003C6E002008B5084B1B78022B07D0033BAC
:10456000012B02D80021FFF751FF002008BDFFF703
:1045700069FF002008BD00BF306E002010B501EBC0
:104580008101084A00EBC1010446B1F88C131046C2
:10459000F3F730FE034A204640230121FFF7E2FEF5
:1045A000002010BD70C20020E8E700BF70B50A7897
:1045B00012F060050C46064611D0202D16D1CD888C
:1045C000D5B113062AD52A461F496078F3F7BEFEF7
:1045D000E2881D493046FFF753FE00250AE04B787C
:1045E0000A2B16D00B2B0ED0062B03D13046FAF730
:1045F000BFFA0225284670BD022260781144F3F705
:10460000A5FE284670BD8B78D3B9104BC3F8C859A6
:10461000F0E70F490122FFF733FEEBE70D4964781D
:104620000A4AC1F8C8400321C0E9E45542F8045BD6
:104630002B4680F811110021FFF794FE0025D9E7E1
:10464000FAF796FAD6E700BFECB80020E8B80020E9
:10465000B0C20020E40400200B7803F00303012B18
:1046600003D0022B04D0002070478B881BB915E6BD
:104670008B88832BFBD099E710B502230446402298
:104680008121FDF7AFF82046022340220121FDF7EA
:10469000A9F88221204603230822FDF7A3F8064B40
:1046A00002229A80F3F7A2FE044A20464023012109
:1046B000FFF758FE002010BDA001002070C20020AE
:1046C00038B509220D46044603238321FDF78AF8F5
:1046D00029462046FFF7D0FF002038BD82B00023D6
:1046E000016801930B6901930E4B03E00A69019283
:1046F000013B13D0019A002AF8DA019A094B42F0E3
:1047000001020192019A0A610A69019203E00A69B1
:104710000192013B02D0019AD207F8D4002002B0E6
:10472000704700BF400D0300436D064A1A61C2780E
:10473000012A06D100F2CC5058614FF0802219684E
:104740001A6070471800086010B500230422044660
:10475000194680F811211A46FFF7DAFC2046FFF7C8
:10476000E3FF002010BD00BF10B5044629B990F842
:104770001131032B0DD0002010BDD0F8E4359B691A
:10478000002BF8D090F81221032AF4D1984700208A
:1047900010BDD0F89013D0F87C33994214D9C0786A
:1047A000D4F880230128A1EB030104BFD218C4F878
:1047B00080238B4228BF0B46C4F890139BB220463F
:1047C0000021FFF7CFFDD6E7D0F8E4351B691BB118
:1047D00090F81221032A03D02046FFF7B5FFCAE75D
:1047E0009847F9E7F0B5012190F8D17590F8D365B5
:1047F00090F8CFC590F8CE5590F8D03590F8D225E6
:1048000080F8111190F8CC1585B005EB0C2503EB61
:10481000072302EB062201F01F06AFB292B290F816
:10482000CD558DF808109BB2012E0446ADF80A70E4
:10483000ADF80C30ADF80E20C0F840218DF80950CD
:1048400017D0022E1FD036B101F08001FFF72CFCEB
:10485000002005B0F0BD092D0FD8DFE815F0BF002E
:10486000AC000E00D5000E00EA0085000E007700B7
:10487000540090F81221032A2FD02046FAF778F935
:10488000002005B0F0BD01F060012029DAB234D07B
:10489000012D00F02081032D00F00681002DD7D1DD
:1048A00090F81211022900F0DF800329E5D11B06E0
:1048B00000F14B8102EB820200EBC20393F87633E6
:1048C000002B00F04D81BF4B0122C3F8DC29BE490B
:1048D00020460222FFF7D4FCBAE7DAB2012ACCD88C
:1048E000D0F8E43502A99B689847BDF80E30002B3C
:1048F000AED12046FFF728FFAAE7D0F8E43502A999
:104900009B689847A4E7F9B2AE4D012985F8CC1908
:10491000B3D890F81231022B00F02781032BACD1D1
:10492000002900F0868190F810110129E1D0D0F81B
:10493000E4355B68984795F8CC1984F81011204647
:10494000FCF7BEFE2046FFF7FFFE81E7012A94D167
:1049500090F81231022B00F01781032B8DD100F556
:104960008871FFF78DFC73E73D0A022DADF8062034
:1049700000F05081032D00F00B81012D7FF47DAFFD
:10498000D0F8EC3580781B680DF106019847BDF82A
:104990000620002A3FF45CAFBDF80E30002B3FF438
:1049A00057AF9A4228BF1A4601462046ADF8062066
:1049B000FFF766FC4CE790F81231023B012B3FF603
:1049C0005CAF012F7FF444AFD0F8E43500229B6840
:1049D000C0F8182102A9204698478AE790F81231BA
:1049E000023B012B3FF649AF764BD0F8182100214E
:1049F000C3F8D41912B10222C3F8D429734920464E
:104A00000222FFF73DFC23E7012F00F09880022FE0
:104A10007FF41EAF13F0FF0F7FF41AAF02691B0A79
:104A2000023B5268032B00F21D81DFE803F03935A9
:104A300031241A437FF421AF90F81231032B3FF455
:104A40001CAF036907F07F0580F81451196867F3FC
:104A50000A120A431A60FFF777FE002D00F0E58086
:104A6000022384F81231F3E651063FF4F1AE114609
:104A7000FFF71AFBECE6052363F30612514B012105
:104A800084F816112046C3F8D829FFF75DFEDFE64B
:104A9000042363F30612F1E7032363F30612EDE741
:104AA000022363F30612E9E790F81231022BDBD000
:104AB000032B7FF4E2AE27B9550602D01146FFF76B
:104AC000F3FAD4F8E43502A99B68204698472046BB
:104AD000FFF73AFEBCE690F812110229C4D0032970
:104AE0007FF4CBAE002F7FF4B3AE12F07F013FF422
:104AF00000AF180600F1A78002EB820304EBC303AA
:104B000004EB810083F8767383F8741383F875736C
:104B1000282303FB0243416D03F55D73DA780B68CC
:104B2000023A6FF35553012AD4F8E42598BF43F0B5
:104B300080530B602046936802A99847D9E6D0F8C5
:104B4000E435C0F818719B6844E702F07F0202EB7D
:104B5000820200EBC20393F81E31002B7FF4B3AE48
:104B6000184B0022C3F8DC29B1E600293FF4C1AE9E
:104B70000121032380F8101180F81231FCF7A0FD09
:104B80002046FFF7E1FD63E61149FFF779FB5FE699
:104B9000FDB2052D3FF671AEDFE805F0342C241C84
:104BA0000B03D0F8EC3580789B690DF1060198472E
:104BB000EDE6D0F8EC3580785B690DF10601984799
:104BC000E5E600BFE8B80020C4C20020BCC2002057
:104BD000B8C20020D0F8EC3580781B690DF10601D1
:104BE0009847D4E6D0F8EC358078DB680DF1060103
:104BF0009847CCE6D0F8EC3580789B680DF106013B
:104C00009847C4E6D0F8EC3580785B680DF1060172
:104C10009847BCE6D0F8E43580789B6A0DF1060130
:104C200098474570C4F8F005B1E6012384F81231C5
:104C30000EE60222D0F8E43580F8101180F8122137
:104C40005B68984755E6282202FB014304EB81008C
:104C500083F81E7183F81C1183F81D51816903F5D7
:104C60008E735BE7012363F3061207E770B5044612
:104C700049B990F81131022B1BD094F81631012B51
:104C80000DD0002070BDD0F8E4355B69002BF8D062
:104C900090F81221032AF4D19847002070BD2A4AC7
:104CA0002369D2F8D8295A60002384F816310020ED
:104CB00070BDD0F83831D0F82451AB4217D9C27842
:104CC000012AD0F82821A3EB050308BF5219C0F828
:104CD000383108BFC0F828219BB20021FFF718FA2D
:104CE00000231A4619462046FFF73CFBC5E7D0F8DB
:104CF0003C31B3FBF5F605FB163666B99D420AD882
:104D0000D0F84021934206D233463246FFF700FAEC
:104D1000C4F84061E4E7D4F8E435DB681BB194F8EB
:104D20001221032A0CD00023052284F811211946F0
:104D30001A462046FFF716FB2046FFF7F5FC9CE7D6
:104D400020469847EFE700BFE8B8002082B0002374
:104D50000193019A094B42F010020192C168019A35
:104D60000A610A69019203E00A690192013B02D0DB
:104D7000019AD206F8D4002002B07047400D03001B
:104D800082B000230193019A0B4B42F02002019262
:104D9000019A61F38A120192C168019A0A610A6953
:104DA000019203E00A690192013B02D0019A920646
:104DB000F8D4002002B07047400D0300F8B50B781E
:104DC00013F060050C4606461CD0202D17D14A78FA
:104DD000FE2A44D0FF2A3DD14A88002A56D1CD88E8
:104DE000002D53D11B0651D43749384B0D7001218A
:104DF00083F88419364A1F23FFF7B4FA00E0002530
:104E00002846F8BD4B780A2B4BD00B2B44D0012BF6
:104E1000F6D191F904308988002B47DBFFF796FF24
:104E200021792A4F3046FCF779FC02232179402270
:104E30003046FCF7D7FC97F88439022B3BD094F925
:104E40000420002ADCDA012BDAD030460121FFF7FA
:104E5000DDFAD5E70225F9F78BFE2846F8BD4D8827
:104E6000A5B9CC88012C11D11A060FD5194B1B6896
:104E70009B6998471549C0B281F8E00930B12246D4
:104E800001F51E613046FFF7FBF9B9E73046022510
:104E9000F9F76EFE2846F8BD0C4B4A8883F8E129E5
:104EA000AEE70D490122FFF7EBF9A9E701F07F0119
:104EB000FFF766FFB4E730468121FFF7F5F80023DE
:104EC00087F884399CE700BF306E0020E8B80020E6
:104ED000DC6D0020206E0020C9C2002038B50446D9
:104EE000FCF752FC2046022340228121FCF77AFC89
:104EF0002046022340220121FCF774FC0C4B0D4993
:104F00001B680D4A00250D701B6882F884592846DD
:104F100098472046FFF71AFF20460121FFF730FF90
:104F2000064A20461F230121FFF71CFA284638BDF8
:104F3000206E0020306E0020E8B80020DC6D0020DC
:104F4000012905D008B50321FFF71AFF002008BD8D
:104F5000FFF752B90B88F0B433BB028C4C880E8932
:104F60008B88C98822F001021204120C0284058B7E
:104F7000028CADB225F0F30592B22B4322F00A0267
:104F800043EA061322439BB242F0010203830284E8
:104F9000038B23F00C031B041B0C0383038B9BB2BA
:104FA0001943F0BC01837047042B048C2CD0082BD0
:104FB0004E888A880D89C98851D024F480542404ED
:104FC000240C0484838B078C2C0344EA022440F6CF
:104FD000FF421A4045F6FF733B4043EA0633224343
:104FE0009BB292B243F4805382830384828B22F477
:104FF00040621204120C8283838B9BB243EA01232A
:105000009BB2F0BC8383704724F010042404240C6A
:105010004D880F898A88C9880484068B038C120204
:105020009BB242EA073423F0A00340F6FF4232402D
:1050300043EA051322439BB292B243F0100302836A
:105040000384028B22F440621204120C0283038B4D
:105050009BB243EA01239BB2F0BC0383704724F464
:1050600080742404240C0484848B038CA4B29BB22B
:1050700024F0F30423F42063224343EA062342EAA4
:1050800005129BB243F4807392B282830384838BB4
:1050900023F00C031B041B0C8383838B9BB21943EB
:1050A000F0BC8183704700BF214A038890429BB2C5
:1050B00012D002F5806290420ED0B0F1804F0BD03A
:1050C000A2F58032904207D002F58062904203D070
:1050D00002F58062904203D14A8823F070031343A3
:1050E000144A904218D002F58062904214D030B435
:1050F00023F440730C894D6802F56C429BB2234344
:1051000090420C880380C56204850DD18B7A03869A
:10511000012330BC8382704703800B884A68C262D7
:105120000385012383827047034B9842EED0EFE75B
:10513000000001400010004000040140104B70B41A
:10514000DA684378017886780E4CD243C2F30222A3
:10515000C2F10405E8B283400F2040FA02F2324067
:10516000DBB2134360181B0101F01F05012249093E
:10517000DBB2AA4080F8003344F8212070BC7047AD
:1051800000ED00E000E100E0C27802B1D6E703786C
:1051900005485A09203203F01F03012101FA03F3E5
:1051A00040F82230704700BF00E100E082B0064BBB
:1051B000002201920193019B03EB80000190019B6F
:1051C000186802B0704700BF5028004082B0064BFC
:1051D000002201920193019B03EB80000190019B4F
:1051E000196002B0704700BF502800400023C0E99A
:1051F0000033C0E90233C0E90433C0E90633C0E933
:105200000833C0E90A33C0E90C338363704700BF39
:105210000B6870B4D1E90524CD682B431343D1E961
:10522000072523431343D1E909422B43D1E90D65F7
:105230002343134304680B4A334322402B43134355
:105240000360D1E90B3442690D6922F00702234360
:105250001343D1E9014243614560846070BCC26080
:10526000704700BF3F801CF002683649002310B42D
:1052700022F00102212488420260036043608360BF
:10528000C3600361446138D02F4B98422ED02F4B1E
:1052900098423CD02E4B984240D02E4B984232D070
:1052A0002D4B984241D02D4B984246D02C4B9842E2
:1052B00017D02C4B98423CD02B4B984216D02B4BFE
:1052C000984224D02A4B984228D02A4B98421AD090
:1052D000294B984229D0294B98422ED0284B9842EE
:1052E00008D14FF03D5243F8AC2C03E04FF4746208
:1052F00043F8202C5DF8044B7047224B5DF8044BBB
:105300003D229A607047204A43F8642CF2E74FF43C
:1053100074125DF8044B43F8382C70474FF07462F8
:105320005DF8044B43F8502C7047184A43F87C2C26
:10533000E0E73D2243F8082CDCE7154A43F8942CBB
:10534000D8E700BF10600240286002404060024081
:10535000586002407060024088600240A0600240D5
:10536000B860024010640240286402404064024079
:10537000586402407064024088640240A0640240A5
:10538000B8640240006002403D000020400F002051
:1053900000003D2000B583B009238DF80730FCF7ED
:1053A000D1FB8DF807009DF80730012BF7D09DF851
:1053B000070003B05DF804FB024A536A23EA0000C9
:1053C0005062704700380240024A136A23EA000024
:1053D0001062704700380240484B98422ED0B0F11E
:1053E000804F32D0464B984236D0464B98421ED022
:1053F000454B984237D0454B98423BD0444B98425E
:105400003FD0444B98424BD0434B984240D0434B03
:1054100098424CD0424B984251D0424B984256D081
:10542000414B98425AD0414B98425ED07047404A17
:10543000136A43F0040313620420C5E73C4A536A2D
:1054400043F0010353620120B6E7394A136A43F07F
:10545000010313620120B7E7354A136A43F00203E0
:1054600013620220B0E7324A136A43F00803136262
:105470000820A9E72E4A136A43F010031362102094
:10548000A2E72B4A136A43F02003136220209BE714
:10549000274A536A43F4803353624FF480308BE7DA
:1054A000234A536A43F002035362022084E7204AEE
:1054B000536A43F4003353624FF400307CE71C4AD4
:1054C000536A43F4802353624FF4802074E7184AF0
:1054D000136A43F040031362402075E7144A136ACD
:1054E00043F08003136280206EE7114A136A43F48D
:1054F000807313624FF4807066E700BF00000140C4
:105500000004004000080040000C00400010004073
:1055100000140040000401400040014000440140EC
:105520000048014000180040001C004000200040DE
:1055300000380240224A936803F00C03042B10B495
:1055400021D0082B22D01F4B03601D4C1E4AA1689E
:10555000C1F30311114491F86C11CB404360A16871
:10556000C1F38221114491F86C1123FA01F1816099
:10557000A1685DF8044BC1F342310A4492F86C21F2
:10558000D340C3607047114B0360DEE75468516835
:1055900052686302C2F388124CBF0C4B094B01F0F6
:1055A0003F01B3FBF1F303FB02F3054A5268C2F378
:1055B000014201325200B3FBF2F30360C5E700BFC2
:1055C000003802400024F400E404002000127A00B5
:1055D0002DE9F04700230F6801264FF0030C02E08D
:1055E0000133102B41D006FA03F232EA0704F7D157
:1055F000D0F800E05C000CFA04F52EEA050EC0F8C5
:1056000000E091F80490D0F800A009FA04FE09F136
:10561000FF394EEA0A0EB9F1010FA846C0F800E0C2
:105620006FEA050515D8D0F808E005EA0E05856093
:105630004D79D0F808E0A54045EA0E05856045683B
:1056400025EA020242608A7945689A4092B22A436A
:105650004260C26822EA0802C260CA79C568A240F4
:1056600001332A43102BC260BDD1BDE8F0870B4B3C
:1056700093F8B825D20703D5012283F8E2297047B1
:1056800093F8E2294AB9D3F81C3633B1044B1A789F
:1056900010445A781870114459707047E8B80020C7
:1056A000986D002010B50E4C40F0080284F880215F
:1056B00094F9CE20022A06DD420704D583071CBFD9
:1056C000012384F8D63005210648FCF74BFB062160
:1056D00084F88101BDE810400248FCF72BBB00BFF5
:1056E000E40400206006002010B5FCF7D3FAA8B34C
:1056F0001B4C94F9CE30012B30DD59B3022B2DD049
:1057000094F8D6309BB971B180230521154884F8EF
:105710008631FCF727FB062184F88701BDE810409D
:105720001048FCF707BBBDE810400420BAE7002989
:1057300014BF0020042094F8D1301A0748BF40F06D
:1057400002005B0701D411B108B940F00100BDE8C7
:105750001040A7E7022BD3D10420ECE710BD00BF17
:10576000E404002066060020F8B5224C04F5C47756
:10577000030A84F88D0105460621384684F88C31E9
:10578000FCF7F0FA94F8D13084F88E01DB072AD4C4
:10579000B4F8D220AA4226D1174DD4F88831C5F8E2
:1057A000E339C3B285F8E93941F26F714FF6FF73FF
:1057B0008A4218BF0123134405F6E316C3F30722F8
:1057C0000621304685F8E72985F8E839FCF7CAFA5A
:1057D000072185F8E9093046FCF7ACFA052104F207
:1057E0008F10FCF7A7FABDE8F84004480721FCF742
:1057F000A1BA00BFE4040020E8B800206C06002035
:1058000008B5FCF747FA48B1A1F59C53083BB3F53E
:105810007A7F03D2BDE808400846A5E708BD2DE918
:10582000F0476B4E3368002B3AD06A4D6A4C05F155
:10583000CE07306838F0A8FD002833D1674B1988AF
:1058400009291D4609D95F8864227A43B2FBF1F227
:10585000452A40F3A1811880588094F8213A012B01
:1058600000F0C581022B00F0E08133B95C480521CE
:10587000FCF760FA012384F8213A5A4B1D685A4B11
:105880001B78002B00F0DB81584B1B68EB1A782B40
:1058900040F2D581D4F83406F9F734F9C4F8245A23
:1058A000BDE8F087306838F067FD94F8EA39804643
:1058B000052BBED8DFE803F00309171D3745AA28DA
:1058C000B7D1012384F8EA39B3E7552803D102237D
:1058D00084F8EA39ADE7414A938801339380002385
:1058E00084F8EA39A5E7032384F8EB0984F8EA3958
:1058F0009FE7132884F8EC09C4F8040A07DD374A47
:10590000D3880133D380002384F8EA3991E718B9AA
:10591000052384F8EA398CE70023C4F8083A042305
:1059200084F8EA3985E7D4F8083AE218013382F8B6
:10593000ED09D4F8042AC4F8083A93427FF479AF09
:10594000E6E7D4F8043A2A4803F1020A4FFA8AF14A
:10595000FCF708FA804594F8EB9940F01481262072
:1059600022F068FD204B48B100221A701B4A538870
:1059700001335380002384F8EA395AE71A784A45FC
:1059800019D100221A7009F1FF33102B00F2F680B2
:10599000DFE813F030008E008E00DE008E00F40091
:1059A000F400F4003000F400F400F400F400F4001B
:1059B000F400F4003000B9F1090F02D0B9F1110F71
:1059C00001D1012ADDD0054A538901335381DAE739
:1059D000946D0020E4040020E8B80020C26D00208F
:1059E00073060020A42F0020D06D0020D46D00206D
:1059F000D3C20020BAF1060F5ADDB9F1010F06D06B
:105A0000B9F1090F0CBF4FF002094FF0030994F8E8
:105A1000F00994F8F11994F8EF2994F9EDE994F963
:105A2000EFC994F8EE3985F8CE9041EA002109B229
:105A3000900785F8CFE085F8D1C0A5F8D21006D53B
:105A400012F00C0F14BF0122002285F8D620B9F104
:105A5000030F13D1BAF1090F2ADD94F9F329082AAB
:105A6000A8BF082222EAE27285F80421002043B28E
:105A70009A4200F1010059DC94F8F239D4F828A0D8
:105A8000002002469BB25245904657DB7C4B85F87E
:105A9000D0001B78232B0BD109EB8903794A03EB48
:105AA00083030CEB83031380A2F802E09180D08083
:105AB000754976480A225EF080FD10B1002384F813
:105AC000163A714B3A681A607A685A603A891A81B4
:105AD00094F8163A2BBB95F8D6306D4A002B14BFBC
:105AE0000223012384F8163A95F8D130117884F80E
:105AF000181A13F001031CBFB1FA81F35B09517846
:105B000084F8191AD8B29188927884F8170AA4F800
:105B10001A1A84F81C2A13B109B1A4F81E1A84F8C1
:105B2000200A0EF04FFF0EF04DFF1FE704EB430875
:105B3000234493F8F539A8F8223698E704EB48088F
:105B40000132B8F82C8052B2984508BF10469AE747
:105B5000BAF1040FACDD94F8ED2994F8EE3943EA7C
:105B6000022359041AB204D5C3F30D03A5F8D430A7
:105B70009EE7002AF8DBA5F8D23099E7454A9389D9
:105B800001339381F2E619F0010F7FF4F3AE414A3D
:105B9000138901331381EDE63F4BD3F89421B3F819
:105BA0009811012A1AD141F25632914203D14FF095
:105BB000FF32C3F89421D3F89421306802EB8202BB
:105BC00002EB820201EB420189B2A3F8981103684B
:105BD0001B69984700232B806B803EE60132EAD197
:105BE000B1F5965F04BF0122C3F89421E3E72A4D83
:105BF00095F9CE60002E3FF440AE022E11D14FF445
:105C00008040FFF7B1FD84F8216A95F9CE30012B71
:105C10007FF733AE95F8D130C3F3400385F8D63023
:105C20002BE6032384F8213AEFE71B4BB3F8D4307B
:105C3000002B3FF422AE032384F8213A1DE694F8AA
:105C4000402094F841309A4204D0FCF7C9FEC4F8D1
:105C5000245A25E6D4F8243AEB1AB3F57A7FBFF438
:105C60001FAE0E4B1B68ED1A952D7FF619AE0C4832
:105C70000521FCF75FF8BDE8F047FCF7B1BE00BFB7
:105C8000C4590020C8590020F4C20020B2050020E9
:105C9000986D0020C26D0020E4040020D46D002027
:105CA00073060020104BD3F81C0610B5D8B10F4C6A
:105CB000217841B162780DF047FDA38883421ABF75
:105CC000A08001210021E2885AB141F28833934239
:105CD000B8BF13469A4204D0E380BDE810404BF0B1
:105CE00009BA0029F9D110BDE8B80020986D00204C
:105CF00010B401440446002014F8013B0822584027
:105D0000430010F0800F08BF400083F0070314BF6A
:105D1000D8B2C0B2013AF3D18C42EDD15DF8044B58
:105D2000704700BF30B54FF4806085B030F0F4FAB2
:105D300048B3164C90F9040094F8283A144A002B02
:105D400018BF08234FF4E1310125CDE9015300913B
:105D500000234FF4806130F03CFBFF23C4F8800047
:105D6000003818BF012084F8FC3484F80C3584F81E
:105D70001C3584F82C3584F83C3584F84C3584F88F
:105D80005C3584F86C3505B030BD00BFE8B8002044
:105D900065200108374B1B6813F000635CD02DE9C8
:105DA000F04F354B1F78B84251D3FF2856D1334BB3
:105DB00093F8DE30002B47D0DFF8D4A00022CAF8D9
:105DC0002C2ACAF8302ACAF8342AAAF8382A002F0E
:105DD0004CD00AF2FC4310461446114615461646AE
:105DE00003EB071BB946B3F802C09F8993F8008004
:105DF00093F901E061443A444645D3E901C738BF0D
:105E0000464610337545B8BF75469B4509B212B278
:105E100064443844E7D191FBF9F192FBF9F28AF836
:105E20002C6A8AF82D5ACAF8304ACAF8340A144B38
:105E3000AAF82E1A1B781149AAF8382A092B4FF014
:105E4000000281F8DE200CD00E48BDE8F08F0E4A2B
:105E500002EB0010BDE8F08F184670470020BDE847
:105E6000F08F0A4B9AF82C2ADA80EDE73A46394649
:105E7000DDE700BFF46B002080060010E404002082
:105E8000C459002014C30020E4BD0020C8590020DC
:105E9000E8B800200268F8B53A4E3B4CB6F93C3AF7
:105EA000511C01607E2111700168054603EBC3039C
:105EB00084FB0302481CDC17002328600B70FF20C2
:105EC000C4EB6204FFF766FF2034304BA4B2002815
:105ED0004DD01B78B0F90C1023BB2D4BA1F57A7275
:105EE0009A4246D82B48B0FBF1F189B228464AF0D5
:105EF000F9FA96F897357BB12AF036FD0146284627
:105F00004AF0F0FA214628464AF0ECFA28460821E1
:105F1000F7F7E2FF0120F8BDB6F84C1628464AF024
:105F2000E1FAEFE71C4B1F78002FD6D01B48002367
:105F300000EB830201339289BB421144F8DB184B1A
:105F40009FED186A93F8223007EE103A07EE901A88
:105F5000B8EEC77AF8EE676AC6EE077A67EEA67AF9
:105F6000FCEEE77A17EE901AB1FBF7F1B5E71B7874
:105F700013B94EF69C21B9E7074B1F78002FF8D0D4
:105F80000146D3E7E8B8002067666666281300106C
:105F90001783930300879303800600105C2F001083
:105FA0004C300020000048432DE9F8434A4C427829
:105FB00094F83E3A02F00F05C3B9EDB92B46002123
:105FC00084F8401AEB1AD9B20E290BD8234493F85F
:105FD000981539B102F0F002802A4AD0902A5FD099
:105FE000A02A0DD000273846BDE8F8830021AB4237
:105FF00084F8401AF6D8E5E784F83E5A2B46DEE7E7
:10600000412966D081F08003042B62D90846FCF751
:1060100043F8031D0246DBB2304884F8403A65F08D
:106020005F0584F8415AFCF7EFFE94F8407A002FA0
:10603000D8D0BE1E16F0FF0024D1FF25A9460227A6
:1060400056B1DFF89C80464418F8011BD4F8640A66
:1060500038F09EF94645F7D1D4F8640A494638F03D
:1060600097F9D4F8640A294638F092F93846BDE821
:10607000F88365F07F050427022684F8415A84F8E6
:10608000407A3046164A4FF6FF71104412F8015B11
:10609000491B904289B2F9D15FFA81F90D0ACFE725
:1060A000412914D081F08003042B10D90846FBF756
:1060B000F3FF65F06F050627042684F8430A84F889
:1060C000415A84F8421A84F8407A3046DAE70420CC
:1060D000EFE7082304229FE7E8B800202AC3002046
:1060E00028C300200B4B93F86E2612B1B3F8A825F5
:1060F0004AB9B3F99436084AD81782FB0323C0EB98
:10610000A30000B27047D3F8880690FBF2F000B20B
:10611000704700BFE8B8002067666666F8B5184C9F
:10612000C6B205463146D4F8680A38F031F994F819
:106130006C1AD4F8680AC5F307274E40394684F82C
:106140006C6A38F025F994F86C1AD4F8680AC5F32B
:1061500007464F40314684F86C7A38F019F994F8C4
:106160006C1AD4F8680A2D0E4E40294684F86C6AE1
:1061700038F00EF994F86C1A4D4084F86C5AF8BD5A
:10618000E8B8002070B50C4DC6B231460446D5F8CB
:10619000680A38F0FDF895F86C1AD5F8680A240AF0
:1061A0004E40214685F86C6A38F0F2F895F86C1A82
:1061B0004C4085F86C4A70BDE8B8002038B50B4CEF
:1061C000002305462421D4F8680A84F86C3A38F094
:1061D000DFF8D4F8680A542138F0DAF8D4F8680AFD
:1061E0002946BDE8384038F0D3B800BFE8B80020F1
:1061F0002DE9F043DFF894932DED028B99F86D4A69
:1062000083B00E461546002C00F03982013C89F817
:106210006D4A9FEDD88AD84FDFF874833378002B0E
:1062200062D099F86D4A002C5ED135B137F0CEF9C5
:106230002B68C01A002880F2028499F86E4A002C5C
:1062400040F0A68399F86F0A062840F2D781CB4A1E
:1062500092F8A13192F8A011994200F00082D2F890
:106260009C1199F870CA31F813406444013001332D
:1062700002F5CE72A4B2C0B2DBB2B4F5E06F89F819
:106280006F0A537100F0D18100F2AA80B4F5806FDB
:1062900000F0F88264D9B4F5A06F00F0CC823CD94C
:1062A000B4F5A16F25D8601EC0B2FFF773FDC8B169
:1062B000B0F90C30B24AADF8014092F82210D9F88A
:1062C000842503EB830303EB830349089B0093FBC3
:1062D000F1F31021CDF803308DF800106846904797
:1062E00000233370002D99D103B0BDEC028BBDE8C3
:1062F000F083B4F5C06FF5D1B9F87036002B00F01B
:1063000054832AF049FB10220024CDF80300062311
:106310008DF800208DF801401FE2B4F5826F00F087
:106320005082B4F5846F40F0358199F848369A0769
:10633000D8D5B9F84A36CDF80330102120220423ED
:106340008DF800108DF801208DF80230D9F88435D1
:106350006846002498473470002D7FF45FAFC3E790
:10636000B4F5067FBED8B4F5007FC0F02C81A4F54B
:106370000073182BB6D801A252F823F0F966010871
:10638000E7660108E7660108E7660108E7660108B5
:10639000E7660108E7660108E7660108E7660108A5
:1063A000E5620108E5620108E5620108E5620108AD
:1063B000E5620108E5620108E5620108C3660108BB
:1063C000AD660108AD660108AD660108AD6601085D
:1063D000AD660108AD660108AD660108AD6601084D
:1063E000B4F5116F00F0E0815BD8B4F5026F00F0F6
:1063F000BF8121D9B4F5036F00F07282B4F5046F48
:106400007FF470AFB9F99436D9F8842503EB830390
:106410005B001020CDF80330402108238DF80000E8
:106420008DF801108DF802306846002490473470D2
:10643000002D7FF4F3AE57E7B4F5E46F00F07881F8
:10644000B4F5006F76D199F8482691077FF54AAFE9
:1064500013F0010F4B4B00F005835A6882EAE27398
:10646000A3EBE27303EB5303A7FB0313DB08002A40
:10647000ACBF43F0004343F0404310210024082206
:10648000CDF803308DF800108DF80140D9F884352F
:106490008DF80220684698473470002D7FF4BEAE18
:1064A00022E745F230239C4200F0B1811DD945F22C
:1064B00040239C4200F0298245F250239C427FF405
:1064C00011AFD9F88836CDF803301021502252236D
:1064D0008DF802308DF80010D9F884358DF8012040
:1064E000684600249847347036E7B4F5376F00F0FB
:1064F00031826FF437616318072B3FF6F3AEA4F1D6
:106500007100C0B2FFF746FC00283FF4EBAE90F9F3
:106510000130CDF8033010238DF80030ADF8014084
:10652000D9F884356846984700233370002D7FF4EE
:1065300075AED9E6B4F5E26F7FF4D4AE124B93EDAD
:10654000140AD3ED017A20EE270A002420EE080A6F
:106550005CF056FD10230722CDF803008DF80030C3
:106560008DF801308DF80220D9F8843568469847B7
:10657000347092E70000C8421F85EB51E40400200C
:106580004C300020846C0020002F0010E8B8002060
:10659000C5B3A29140F201439C427FF4A3AEB9F986
:1065A0003C3ACDF803301021012204238DF802304B
:1065B0008DF80010D9F884358DF801206846002444
:1065C00098473470C8E6B4F5807F00F01481B4F5C4
:1065D000887F7FF487AEB9F99636CDF80330012273
:1065E00010238DF800308DF801308DF80220D9F895
:1065F00084356846002498473470ADE60130CD4AB2
:10660000C0B292F8A91192F8A8318B4222D04B1C4B
:10661000DBB24900D2F8A441C74A645A89F86F0A2C
:10662000B4F5E06F53717FF42FAEC44B93ED130AB2
:10663000D3ED017A20EE270A002420EE080A5CF050
:10664000DFFC10220723CDF803008DF800208DF821
:10665000014082E0002182F8A9110123DAE7B8495C
:1066600099F8703A097882F8A1410133DBB201311F
:106670008B4289F8703A00F087810120C1E7002839
:106680003FF4C7AD0378303B012B3FF6C2AD01307C
:1066900009F66D220621FCF7F7FE99F86D3A89F8A4
:1066A0006E0A002B3FF4B5AD3470B2E5A4F11100D1
:1066B000C0B2FFF76FFB00283FF414AEB0F9023010
:1066C00027E799F89735002B40F0B081B9F84C06D0
:1066D000CDF80300102302228DF800308DF8013030
:1066E0008DF8022083E7601EC0B2FFF753FB00283D
:1066F0003FF4F8AD43680CE7D9F880369149D9F8F2
:10670000842581FB0301DB17C3EBA10300241021C7
:10671000CDF8033002238DF800108DF801408DF87C
:106720000230684690473470002D7FF477ADDBE58A
:10673000824B93ED150AD3ED017A20EE270A00244F
:1067400020EE080A5CF05CFC102320228DF800305B
:10675000CDF8030007238DF801208DF8023068463C
:10676000D9F8843598473470002D7FF457ADBBE5D8
:1067700099F848369B077FF5B5AD734AD9F884354B
:106780009268CDF80320102220218DF800200822E5
:106790008DF801108DF80220684600249847347067
:1067A000002D7FF43BAD9FE52AF0DEF8102309228F
:1067B000CDF803008DF800308DF801308DF80220FF
:1067C00015E7D9F8803513F0200440F0F1805F4BD5
:1067D0001B681B0640F13981102304228DF8034009
:1067E0008DF804408DF805408DF806408DF8003096
:1067F0008DF801304AE6D9F8743ACDF8033010220A
:10680000002401238DF800208DF80140A5E7B9F997
:106810009236CDF803301021302252238DF8023009
:106820008DF80010D9F884358DF8012068460024D1
:106830009847347090E5FF20FFF7ACFA00283FF44A
:1068400051ADB0F90C304249D9F8842591F82210A5
:1068500003EB830303EB83031020490800249B0010
:1068600093FBF1F305218DF80000CDF803308DF88E
:1068700001408DF80210684690473470002D7FF477
:10688000CDAC31E599F8783A0133DAB2042A00F058
:10689000D08042F2107389F8782A03FB02F3D9F80A
:1068A0007C2A002A00F0C080023399F8B825D2076C
:1068B000B9F88C2648BF0433D40748BF0A33900781
:1068C00048BF1433D10548BF2833540748BF643349
:1068D000500648BF03F57A63102100240422CFE557
:1068E00099F8483698077FF5FDAC174BD9F8842501
:1068F000D9894FF4F36303FB01F3A7FB03135B098F
:106900001020CDF80330302187E5B9F99036CDF865
:1069100003301021402252238DF802308DF80010F0
:10692000D9F884358DF801206846002498473470E2
:1069300012E500BFE404002088060020002F0010AC
:106940008006001067666666846C0020F46B002089
:106950004C300020FF20FFF71DFA00283FF4C2ACA6
:1069600090F90130CDF80330102170220B238DF8FF
:1069700002308DF80010D9F884358DF80120684672
:10698000002498473470E7E489F8704A012038E61B
:106990005C490620FCF7C8FC002389F86E0A3370B6
:1069A00003B0BDEC028BBDE8F083D9F88806AAE4F9
:1069B000554A99F84816538A643BC3EB4370C3EBBE
:1069C000C00388FB03401844DB17C3EB20230933C3
:1069D000092BA8BF092323EAE37303EB830311F018
:1069E000020F03EB830314BF4FF47A7000209B0067
:1069F000C90748BF00F5FA60117DD9F884259BB21C
:106A000003440B44042010218DF80200CDF803301C
:106A10008DF800108DF801106846002490473470FE
:106A2000002D7FF4FBAB5FE401333EE729F09CFFD0
:106A30004EE6012389F8783A42F210732FE734705A
:106A400003B0BDEC028BBDE8F08399F89635002BBE
:106A50003FF448AC99F8803A032B4ED8DFE803F0B6
:106A600043392A111A6882EAE273A3EBE27303EB5B
:106A70005303A7FB0313DB08002AB8BF43F080438E
:106A8000FBE4D9F8882A537A907AD17A03F14073DB
:106A900003EB0023002203EB014389F8802A102234
:106AA0000421CDF803308DF800208DF801208DF8F9
:106AB00002104BE4D9F8841A8A7D087C897A120482
:106AC00002EB00220A44591C89F8801A02EB036386
:106AD000E5E7D9F8841A4A7DC87B497A120402EBAB
:106AE00000220A44EFE7D9F8841A0A7D887B097AE4
:106AF000120402EB00220A44E5E75A1C89F8802AB6
:106B00001B06CCE751210108846C002030B5A0F1B0
:106B10007D03012B044683B00D46104608D921465B
:106B200037F036FC15B1288804442C8003B030BD02
:106B30007D21019237F02CFC019884F0200137F080
:106B400027FCEFE730B50F4B85B0D3F8B425002311
:106B50000446C51DADF80E3014F8010B01920DF17D
:106B60000E01FFF7D3FFA542019AF5D10DF10E00FA
:106B700018F00CF8019A9DF80E000021FFF7C6FFEF
:106B800005B030BDE8B800207E28F8B50F4652D0D9
:106B9000324E96F8AC4164B9314D95F8941A51B122
:106BA0001B2885F8944A3DD00D2837D0012386F85C
:106BB000AC310020F8BD7D284AD095F8982A1AB14A
:106BC00080F0200085F8981A95F8932A062A14D8A0
:106BD000B5F8964A511C2A440444C9B2A5F8964A0D
:106BE00085F8931A82F88C0A002BE2D10729E0D1AC
:106BF00001231C4886F8AC31F8BDB5F8963A184424
:106C0000C0F3072353FA80F0FF284FF00103A5F8E3
:106C1000960A86F8AC31CCD11248F8BDA5F8964A50
:106C20002046F8BD90470028C0D0012320463B7085
:106C300086F8AC31F8BD0A4B084A0024012183F8DC
:106C4000934A83F8941A3C7082F8AC412046F8BD10
:106C50000123084685F8983AF8BD00BFE4040020F7
:106C6000E8B8002074C30020044AD2F89C3A43F4E8
:106C7000DF2343F48063C2F89C3A7047E8B80020F1
:106C8000013070B5094EC4B203E04AF00FFD013483
:106C900048B9E5B2152D21463046F6D9162D04BF68
:106CA000034B93F8A05A284670BD00BF84C3002050
:106CB000E8B8002000B1D7E7044AD2F89C3A23F4A0
:106CC000DF2323F48063C2F89C3A7047E8B80020C1
:106CD00070B5114C84B00546D4F8A40A0E462FF0C6
:106CE000D9FA94F8902594F89135003A18BF01220A
:106CF0000BB142F00802CDE9016200234FF4964146
:106D000095F9000000911A4608212FF062FBC4F8A3
:106D1000A40A04B070BD00BFE8B8002010B5064C4E
:106D200003E0D4F8A40A37F027FBD4F8A40A37F01C
:106D30002BFB0028F5D110BDE8B8002010B50D4C94
:106D4000D4F8A83A1B791E3B012B0DD9D4F8A40A1C
:106D500001213830FFF7BCFF0023C4F8AC3A84F8B7
:106D6000B03ABDE81040D9E7D4F8A40A012137F0C1
:106D7000FBFAF1E7E8B800200B2814D810B401EBB7
:106D80004103094C01EB83032344184490F8A836CF
:106D9000934205D02144002380F8A82681F89C3630
:106DA0005DF8044B70477047E8B80020F0B5444CDC
:106DB00094F8B13A012B83B005464FD994F8B21A32
:106DC0004048DFF810C194F8B37A4A1CA0FB026077
:106DD00000F4FE7606EB90001944121A5CF821606C
:106DE00084F8B22A2FB1D4F8B41A04F6B82291422A
:106DF0000DD06EB9344A0133A2FB031222F0010117
:106E000001EB52029B1A84F8B13A03B0F0BD2F4E49
:106E100094F8CC3A93B92E4B019348F2A501123B5A
:106E200015226F46A4F8D01A009384F8D22A294676
:106E30003846B04758B994F8B13ADBE76F46384660
:106E400016F072FC29463846B0470028F3D094F873
:106E5000CC1A49B1384616F0E1FBECE71D4A52F86E
:106E60002360002EC6D0D3E7009E1B4A964214D959
:106E7000013A013E41F2210512F8013F81EA032166
:106E8000082311F4004F85EA41000ABF490081B28E
:106E900089B2013BF5D19642EED1384649F048FB24
:106EA0000E49009D6D1A152DA8BF15252A4601F122
:106EB00018005DF049FB94F8B13A84F8FD5A99E75F
:106EC000E8B80020CDCCCCCCABAAAAAA9532010858
:106ED000CDC3002078480708BBC30020B8C30020FA
:106EE00070B50C4E054606F60231D52249F0B0FFCA
:106EF0002C686C6006F53061641A182CA8BF182441
:106F00002960224606F618305DF01EFB86F8304BED
:106F100070BD00BFE8B80020F0B58BB004461F4B31
:106F20001F4A2049009302A81F4B49F043FA2668E4
:106F30000025731C2360357023682922591C2160A9
:106F40001A702368EA22591C21601A702368C8222B
:106F5000591C216002A81A705AF010F9471C02A9A6
:106F60003A4620685DF0F0FA236829461F440C2356
:106F700000E027687A1C013B22603970F9D1226851
:106F8000511C2160137023680122991821601A7026
:106F900023689B1B33700BB0F0BD00BF23C40020DF
:106FA000A0E00708A0E1070898E1070870B50568A8
:106FB0002C4E00236A1C02602B7003682122591C8E
:106FC00001601A7096F8B835DB0704461ED5B6F88E
:106FD0008C36590510D52449204649F02BFA96F8ED
:106FE000B835DB071DD523680022591C21601A70B3
:106FF00023685B1B2B7070BD1A0524D4D80524D4DC
:10700000D90724D49A0724D51849E5E7D6F87C3A5D
:107010006BB11749204649F00DFA96F8B835DB07F1
:10702000E1D423682A22591C21601A70DBE7114B36
:107030001B681806CBD596F8483603F00303032BDC
:10704000C5D00D49C8E70D49C6E70D49C4E70D494C
:10705000C2E796F8442B0C490C4B002A18BF19467E
:10706000BAE700BFE8B80020C8E10708ACE10708AC
:10707000B8E10708F46B0020C0E10708D0E1070879
:10708000D4E10708DCE10708B0E10708E4E10708FC
:1070900038B50368394D591C082201601A7003681D
:1070A0001E22591C01601A70B5F99236B3F5E16FD2
:1070B000044650DDA3F561631BB2B3F5E16FF9DC63
:1070C00007EE903A9FED2E7AF8EEE77A204667EECB
:1070D000877AFDEEE77A17EE903A99B249F002FA14
:1070E000B5F99036B3F5E16F3CDDA3F561631BB2F2
:1070F000B3F5E16FF9DC07EE903A9FED217AF8EEF7
:10710000E77A204667EE877AFDEEE77A17EE903A47
:1071100099B249F0E7F9B5F99436B3F5E16F28DD96
:10712000A3F561631BB2B3F5E16FF9DC07EE903AAA
:107130009FED137AF8EEE77A204667EE877AFDEE48
:10714000E77A17EE903A99B2BDE8384049F0CAB9EB
:1071500003F561631BB213F5E16FF9DBB0E703F5EB
:1071600061631BB213F5E16FF9DBC4E703F56163FB
:107170001BB213F5E16FF9DBD8E700BFE8B80020D8
:1071800058A08B41026810B40421541C0460117093
:1071900002680B24511C016014705DF8044BC82177
:1071A00049F0A0B938B50368214D591C0A22016085
:1071B0001A7003680822591C01601A7095F89735F7
:1071C00004466BB329F0D0FB1A490530A1FB00310E
:1071D000C1F3CF01204649F085F9D5F88036164A2B
:1071E000D91782FB0323C1EBA30189B2204649F0E2
:1071F00079F929F0D1FBD5F8885623682A0C591C57
:1072000021601A7023682A0A591C21601A702368A9
:107210005A1C22601D7023685A1C2260187038BDE9
:1072200029F0AEFB0146204649F05CF9D5E700BFE6
:10723000E8B80020CDCCCCCC676666660368112226
:10724000591C70B501601A7003681D4D1D4E5A1C03
:10725000026002221A700446296849F02BF9696815
:10726000204649F027F9E98901EBC1018900323153
:10727000A6FB0131C1F34F11204649F033F9298AA9
:1072800001EB8101490089B2204649F02BF90E4AF1
:107290000E4BD2F8741A9942A8BF194621EAE1713F
:1072A000A6FB0131490901F57A7189B2204649F0FE
:1072B00019F923682A7D591C21601A7070BD00BF1E
:1072C000846C00201F85EB51E8B8002020A1070046
:1072D000F8B50B4D0B4F06462946D52249F0B8FDAF
:1072E00034687460A91E641A402CA8BF4024316021
:1072F000224607F648305DF027F987F8884BF8BD3D
:10730000C25A0020E8B8002070B5104E104B0A4653
:10731000151D014696F8890B03F83F5C82B003F80F
:107320003D0C7B25C82003F83C0CA3F13B0403F87B
:10733000400C03F83E5C68460193009449F08CF8D9
:107340006846FFF7C5FF02B070BD00BFE8B8002077
:10735000005B0020F0B5424C94F88C3BD90783B019
:10736000054637D594F88D3B0F2B54D900210F4695
:107370003C4B94F88C2B3C4843F8400CA3F140065E
:1073800040F6C82CC2F38202712003F8381CA6F81C
:1073900004C0B11C0193B071373B6846F271BA2248
:1073A000009349F055FD009A731CD21A727016F0C2
:1073B000DDF96846FFF78CFF16F0D8F994F88C3B9E
:1073C000C4F8905B23F0030343EA470384F88C3B43
:1073D00003B0F0BD9A0726D5D4F8900B2D1AB5F559
:1073E0007A6FF5DB94F88D3BD4F8940B0F2B96BF96
:1073F0001E4A1F4902EB83031E4A98BFD9690368DE
:1074000011601B69984794F88C3B6FF3410384F833
:107410008C3B03B0F0BD184B93F834301F1E18BFDF
:1074200001273946A4E7154B1B685B05D0D4124BE6
:1074300093F83430002BCBD00A4B0193C821A3F131
:107440003F02684603F8401C0092FFF79BFE16F0CF
:107450008DF96846FFF73CFF16F088F9B8E700BFE2
:10746000E8B80020005B0020C80032EC784807082C
:10747000A0680600201E0020A4650020F46B0020F8
:107480002DE9F843254E96F8984B804634BBD6F844
:10749000FC3B6BB306F69C374FF001090DE001355C
:1074A0002C44EFF31183502282F31288D6F8FC2B80
:1074B000944220DADBB283F311883319601C93F80D
:1074C0009C5B384429460022FBF7DEFF0028E6D00B
:1074D00096F8883BD3B186F8989BE0E796F8883B0E
:1074E00033B901463A20FBF71FFF044686F8980B94
:1074F0002046BDE8F8830022DBB2C6F8FC2B96F8E4
:10750000984B83F311882046BDE8F88341463A2022
:10751000FBF70AFF86F8980BC1E700BFE8B8002028
:10752000044BD3F8AC3530EA030314BF012000202C
:10753000704700BFE8B80020AB4A38B508200023E8
:1075400082F8A931FFF7ECFF002800F08C80D2F818
:10755000A4314FF4806102204FF48264198082F8D4
:10756000A90101465C804FF40020FFF7D9FF50B11C
:107570004B1CD2F8A401DBB240F2014482F8A931DD
:1075800020F811401946994C94F86D36002B6CD1B7
:1075900094F86E36002B40F088804FF40070FFF7AF
:1075A000BFFF50B14B1CD2F8A401DBB24FF404650D
:1075B00082F8A93120F811501946D4F88045A50762
:1075C00000F11881600700F1EB80894B1B681B06F6
:1075D00000F1A38000234FF4803082F8A81182F8D4
:1075E000A93182F8A131FFF79BFFD0B3D2F89C31CB
:1075F00001214FF4047082F8A11118804FF400406B
:10760000FFF78EFF50B14B1CD2F89C01DBB24FF458
:10761000007482F8A13120F8114019464FF400306F
:10762000FFF77EFF50B14B1CD2F89C01DBB24FF448
:10763000A06482F8A13120F8114019464FF480204F
:10764000FFF76EFF38B1D2F89C014FF437644B1C42
:1076500020F81140D9B2002382F8A01182F8A1319C
:1076600038BD0146CAE701467DE70120FFF758FF14
:1076700000288DD04FF48030FFF752FFD2F8A4518C
:1076800028B94FF4047325F811300131C9B20BB297
:10769000481CC1B24FF4116082F8A91125F81300FB
:1076A00094F86E36002B3FF478AF0220FFF738FFD6
:1076B00000283FF472AF4FF40040FFF731FF50B99C
:1076C0004B1CD2F8A401DBB24FF4007582F8A9314B
:1076D00020F8115019460420FFF722FF50B14B1C2F
:1076E000D2F8A401DBB24FF4C06582F8A93120F8CA
:1076F000115019464FF48010FFF712FF00283FF495
:107700004CAF4B1CD2F8A401DBB245F2502582F8F5
:10771000A93120F8115019463FE74FF40050FFF708
:10772000FFFE50B14B1CD2F8A401DBB24FF403644E
:1077300082F8A93120F8114019464FF48050FFF724
:10774000EFFE68B1D2F8A4014B1C4FF40064DBB229
:107750008D1C20F81140E9B282F8A91120F81340DD
:107760004FF48040FFF7DCFE50B14B1CD2F8A4016F
:10777000DBB24FF4846482F8A93120F81140194635
:107780004FF48060FFF7CCFE00283FF423AFD2F81F
:10779000A4014FF402644B1C20F81140D9B219E740
:1077A0004FF48060FFF7BCFE50B14B1CD2F8A4012F
:1077B000DBB24FF4807482F8A93120F811401946E9
:1077C0004FF40060FFF7ACFE00283FF4FEAE4B1C08
:1077D000D2F8A401DBB24FF4887482F8A93120F802
:1077E00011401946F1E600BFE4040020E8B800208B
:1077F000F46B00208020FFF793FE50B14B1CD2F8B1
:10780000A401DBB245F2302582F8A93120F81150ED
:1078100019464FF48070FFF783FE50B14B1CD2F82D
:10782000A401DBB245F2402582F8A93120F81150BD
:1078300019461020FFF774FE50B14B1CD2F8A4017A
:10784000DBB24FF4E06582F8A93120F811501946F7
:107850002020FFF765FE50B14B1CD2F8A401DBB22B
:107860004FF4E26582F8A93120F811501946402002
:10787000FFF756FE00283FF4A5AE4B1CD2F8A4013A
:10788000DBB24FF4E46582F8A93120F811501946B3
:1078900098E600BFF0B5C94C94F8043CD4F88015C4
:1078A000C4F8000C0133880785B084F8043C12D476
:1078B00011F0340F34D1090794F8042C41D412F09C
:1078C00007055AD0282A00F0DA80D4F888355E20DF
:1078D000984705B0F0BD7020FFF722FE0028E7D0E2
:1078E000B74E2425A6F14C07F6EC017A97ED017A04
:1078F00067EE877A2846FDEEE77A013517EE901A93
:10790000C1EB411301EB8301C90009B2EDB2FAF7F3
:107910005BFC272DE8D1D4F8801511F0340FCAD0C4
:107920004FF40060FFF7FCFD002840F0278194F839
:10793000042C12F0030100F0FD80D4F88015090733
:10794000BDD54FF40070FFF7EBFD0028B7D012F063
:107950000305B4D19B4AB4F99436D91782FB0323AB
:10796000C1EBA30109B21420FAF72EFC29461C2012
:10797000FAF72AFC94F8042CA1E7FF20FEF70AFA94
:10798000002800F001810378FF2B00F09A8090F925
:1079900001100220FAF718FCFF20FEF7FBF900287F
:1079A00000F091800378FF2B00F08D80B0F90C205F
:1079B000854B844893F8221002EB820202EB82028C
:1079C0009300490893FBF1F3D91780FB0320C1EB27
:1079D000A00001B20320FAF7F7FB94F86D36002BF4
:1079E00079D1D4F880359A0640F198804FF4005050
:1079F000FFF796FD002840F0CB80744D4FF4806077
:107A0000FFF78EFD002840F04D816B8A94F8042C1E
:107A1000297DB3F5967F02D9100740F1128194F8C1
:107A20009335002B40F0B280A1F1200307EE903A8D
:107A30009FED677AF8EEE77AF6EE006A67EE877AEE
:107A4000BEEE007AF5EEC07AF1EE10FA58BFB0EE55
:107A5000667A77EE877AFDEEE77A17EE903A19B2FA
:107A60000520FAF7B1FB4FF48050FFF759FD0028CD
:107A700040F0BE8094F8042C282A7FF426AF554AA3
:107A8000554B15685549A3FB0535AD09A1FB0536D6
:107A90007609A1FB06314909C1EB0111A6EB810171
:107AA0000902C6EB0616002309B21720A5EB8606CD
:107AB00084F8043CFAF788FB31B21820FAF784FB0B
:107AC00003E7294665E700210320FAF77DFB94F8D8
:107AD0006D36002B85D00120FFF722FD002840F0F5
:107AE000F38094F86E36002B3FF47BAF0220FFF753
:107AF00017FD002840F041810420FFF711FD002808
:107B00003FF46FAFB4F87036002B00F0438128F0DB
:107B100043FF01B20420FAF757FB62E71B07A9D520
:107B20002F4B93E8030002AB83E803001846FAF7F3
:107B300061FB9FE74FF48060FFF7F2FC00283FF401
:107B4000FCAE284BD4F8002CD4F8745A9A4240F278
:107B5000F180254BE91783FB0523C1EB63136421F7
:107B600001FB13510DB219B21020FAF72DFB294673
:107B70002120FAF729FB94F8042CDEE6B4F99616D6
:107B80003020FAF721FBD2E6014602E709B267E7A7
:107B900094F848369F075AD44FF48060FFF7C0FC32
:107BA0000A4D00283FF431AF002631460120FAF794
:107BB0000BFB31460920FAF707FB26E7E8B800205F
:107BC0004C2F0010676666664C300020846C0020E5
:107BD000E4380E3FA42F0020D34D62108988888896
:107BE000D44807083F4B4C001F85EB510050C3475A
:107BF00094F8482600239207CDE9003347D494F83F
:107C0000083C012B43D0B4F98C355FED086A07EED0
:107C1000103AB4F98E3507EE903AB8EEC77AF8EE1E
:107C2000E77A27EE267A67EEA67ABDEEC77AFDEEF2
:107C3000E77A02A88DED027ACDED037AFAF7DAFA47
:107C400018E742F20F719942A8BF1946E7E6544D72
:107C5000544BE9894FF4F36606FB01F14909A3FB94
:107C60000131C9091120FAF7AFFAE9894E4B06FB39
:107C700001F1A3FB01214909A3FB01235B09642254
:107C800002FB131109B21920FAF79EFAB6E6D5E9FC
:107C9000002301216846CDE9002384F8081CFAF787
:107CA000A9FAE7E694F848369E077FF57DAFAB6802
:107CB0003D4AD91782FB0302C1EB6211642606FB21
:107CC000113636B209B271E794F8051C00293DD18E
:107CD0000B460620A4F8063CFAF776FAB4F8063C00
:107CE0000133A4F8063C28F04BFE94F8943594F840
:107CF000052C012B94F897351ED000EB800086B23E
:107D000013B10AB1B6FBF2F6274BA3FB062343F3EC
:107D10004F113A205D09FAF757FA642101FB15610A
:107D2000224B89B20531A3FB0131C9083B20FAF788
:107D30004BFAD6E60D4617E71BB112B1B0FBF2F0D5
:107D400080B201B23920FAF73FFACAE6B4F8060C5D
:107D5000B4F84C26B0FBF1F301FB1303642000FBE5
:107D600002129BB24900B2FBF1F2110241EA031187
:107D7000C2F30322114309B2ABE7D4F880360C49B1
:107D8000DA1781FB0313C2EBA30319B22820FAF719
:107D90001BFAB1E6D4F8883683F3100319B2B9E6BA
:107DA000846C0020C55A7C0A1F85EB51CDCCCCCC0D
:107DB0006766666603685A0607D513F4057F04D024
:107DC00007298CBF00200120704703F48253B3F5CC
:107DD000825F03BFC81FB0FA80F0400900207047DF
:107DE00070B5BC4C94F8093C012B84B000F04D8177
:107DF00094F8150CFCF778F894F8163C8342054685
:107E00001FD0002800F0D680D4F8A83ACBB194F85F
:107E1000912593F90400002A18BF08224FF49641D7
:107E200000230325CDE9015200911A4608212EF0C6
:107E3000D0FAC4F8A40A20B1FEF780FF012384F829
:107E4000163C94F8173C012B00F0C180D4F8206C4C
:107E50003EB1A14B30465978FFF7ACFF002840F007
:107E6000F28094F8250CFCF73FF894F8243C834208
:107E7000054621D0002800F0F680EEB1337A002BC1
:107E800000F01881954A02EB8303DB6994F8902592
:107E900096F904000093003A18BF01220221002342
:107EA000CDE901121A4610212EF093FAC4F8680A9F
:107EB00010B1012384F8243CD4F8286C3EB1864BE1
:107EC00030465978FFF776FF002840F0AC8094F8F0
:107ED000340CFCF709F894F82C3C8342054622D078
:107EE000002800F0C980F6B1337A002B00F0E5805D
:107EF0007A4A02EB8303DB6994F8902596F9040033
:107F00000093003A18BF012202210023CDE901129B
:107F10001A464FF400712EF05CFAC4F8300C10B120
:107F2000012384F82C3C94F8350CFBF7DDFF94F822
:107F3000363C8342054631D090B3694BD4F8386C57
:107F4000D3F800354FF47A721A613EB34FF4805281
:107F5000402130462EF0CCF90546F8B994F890351A
:107F600096F90400002B14BF0921082103224FF4C5
:107F7000E133CDE9012100932A462B464FF480518D
:107F80002EF027FAC4F83C0C40B10123C4F8640A6F
:107F900084F83E5A84F8405C84F8363C04B070BDE6
:107FA000D4F83C0C2EF076F9C4F83C5C84F8365CCE
:107FB00004B070BDD4F8A40A2EF06CF994F8173C04
:107FC000C4F8A45A012B84F8165C7FF43FAF94F8F0
:107FD000180CFBF789FF0546002871D0D4F8B4359A
:107FE000002B7FF433AFD4F81C2C002A3FF42EAFC3
:107FF00094F8915594F8901592F90400002D14BF4F
:1080000008220022002908BF42F0010203254FF494
:108010006141CDE9015200911A4620212EF0D9F993
:10802000C4F8B40512E794F82C3C002B7FF47BAF26
:10803000D4F8103C002B3FF476AF0122C4F8303C5A
:1080400084F82C2C6FE794F8243C002B7FF434AF99
:10805000D4F8103C002B3FF42FAF0122C4F8683A4B
:1080600084F8242C28E7D4F8680A2EF013F9C4F811
:10807000685A84F8245C1FE7D4F8300C2EF00AF913
:10808000C4F8305C84F82C5C4DE7D4F80C5C124BDF
:1080900028465978FFF78EFE20B3D4F84436002BDB
:1080A0007FF4A6AED4F8103C002B3FF4A1AEC4F888
:1080B00044369DE64FF49643E8E64FF461431BE7F0
:1080C000D4F8B40500283FF4C1AE2EF0E3F8C4F8AC
:1080D000B455BBE6E8B80020806500207848070862
:1080E000B84C002094F8140CFBF7FEFE0646D8B1FD
:1080F000D4F84436002B7FF47BAE002D3FF478AEED
:1081000094F8902595F90400B2FA82F252094FF4DE
:1081100016510225CDE9015200911A4604212EF094
:1081200058F9C4F8440663E6D4F8440600283FF43E
:108130005FAE2EF0AFF8C4F8446659E670B5D44C83
:1081400094F8093C002B00F0BF8108202EF0E4F8E1
:10815000C4F8A80A00283CD008212EF0D3F8002645
:108160000346CC49CC4884F8153C0522C4F8486C39
:108170003AF0EEFF41F208530122C748A4F84C3C04
:1081800084F8502C0DF0DEFC31462B22C3485CF005
:108190003CFA48F67C607D25E02331462B22A4F88A
:1081A000580CBF4884F85B3C84F8835C5CF02DFA83
:1081B00048F67C21A0224EF27B0384F8AF5C84F861
:1081C000B26C84F85B5DA4F8841C84F8872CA4F856
:1081D000B03C94F8173C002B00F0438110202EF0A7
:1081E0009BF81021C4F8200C2EF08CF8AD4B84F8CD
:1081F000250C3A2140F23B1094F86D2618809F25FB
:108200004AF21E40197100219D7198601973002A6D
:1082100040F00D8194F86E36002B71D1D4F8803582
:10822000580700F1FD80990700F1F1801A0700F16D
:10823000E7809D4D2868C0F3C010FEF73BFD00208D
:10824000FEF71EFD03464FF4007084F8A03A2EF0AE
:1082500063F84FF40071C4F8280C2EF053F8D4F8EA
:108260005C3D84F8340C002B14BF0123002384F8F8
:10827000603D40F09180D4F8943B002B14BF012363
:10828000002384F8693D42D1D4F8AC2E0023C4F811
:10829000FC3B002A00F0DB80012284F8CC3A84F811
:1082A000B02E002381488249C4F8BC3A06223AF035
:1082B0004FFF40F609437D48A4F8C03A0DF042FC58
:1082C0004FF480502EF028F84FF48051C4F8380C49
:1082D0002EF018F8D4F8B83E764A84F8350C02F53A
:1082E000A075581C0021C4F82027C4F82457C4F8EE
:1082F0004839C4F8B80E84F8361CBDE870406FE504
:10830000D4F89C3A43F00403C4F89C3A86E7D4F8C6
:108310008005002310F0020084F86A3D84F86B3D6C
:1083200040F0EB80024694F86D362BB10120FFF748
:10833000F7F8002840F0F38094F86E36002B40F0F8
:10834000E8800820FFF7ECF820B1A318042183F897
:108350006C1D01322B681B0600F10281564B102167
:108360009818053300F8011B8342FBD10521092031
:1083700042F2090384F8711D84F8950E4F49504864
:10838000A4F8A03E2025042284F8965E3AF0E0FE90
:108390004B480DF0D7FB77E794F86D362BB10120F1
:1083A000FFF7BEF8002840F0C08094F86E26002A3F
:1083B00040F0E3802B681B0600F1BB80D4F88015E9
:1083C0004E070CD54FF48060FFF7AAF838B1A31818
:1083D000082183F8641D013284F8682D4BE70807F3
:1083E00005D54FF40070FFF79BF80028EFD1090581
:1083F000F2D54FF40060FFF793F80028ECD0E6E7E1
:10840000D4F89C3A43F48073C4F89C3A11E7D4F84A
:108410009C2A42F4601242F0C002C4F89C2A05E78C
:10842000D4F89C2A42F40272C4F89C2AFBE6D4F8E1
:108430009C3A94F86E2643F00201C4F89C1A002A74
:108440003FF4ECAE43F03603C4F89C3AE6E6D4F8C9
:10845000B43E002B4CD0012384F8B03E84F8CC3AD3
:108460001FE720202DF058FFC4F81C0C00283FF413
:10847000B5AE20212DF046FF124BC4F8843584F8A8
:10848000180CFFF759F8012384F8173CA6E600BF43
:10849000E8B80020DC4807082CC5002040C50020B3
:1084A0006CC500209C6C0020F46B0020A0C3002051
:1084B0008449070818C0002054C600203049070826
:1084C00080C70020456B010804202DF025FFC4F86B
:1084D0000C0C00283FF439AE04212DF013FF2A4A7A
:1084E00084F8140C0123C4F8882584F8093C2CE690
:1084F00084F8B03E84F8CC3AE2E64FF46070FFF7BF
:108500000FF800283FF40EAF012084F86C0D0246EE
:1085100009E70620FFF704F800283FF412AFA3187C
:10852000022183F86C1D01320BE7012284F8642DCF
:1085300040E74FF4A050FEF7F3FF20B1A31802214B
:1085400083F8641D01324FF40850FEF7E9FF00285C
:108550003FF434AFA318042183F8641D01322DE7E2
:108560004FF45850FEF7DCFF00283FF4F7AEA31895
:10857000082183F86C1D0132F0E60620FEF7D0FFDB
:108580000028D2D1024615E7F92D010800000000AD
:1085900030B40023022515244FF4167140F2D9326D
:1085A00005808471018130BC428143808380838156
:1085B0007047084B5A881B88801A9B1AC00090FB92
:1085C000F3F00628A8BF062020EAE070C0F196006C
:1085D000C0B270474CBF0020074B084A33F8101058
:1085E000127802EAD122520705D0DA6F511CD967FE
:1085F000134483F8800070472CC8002094060020A4
:1086000010B5164B42681B7803F00303032B21D1EE
:10861000134B1B88DBB1134B1349B3F9BE30B1F9CF
:1086200004100A2491FBF4F15B1A1B0103F5B95302
:1086300014334FF4B471B3FBF1F3C3F1080303F047
:108640000F0360331370436800225A7010BD052376
:108650001370F8E72D231370F5E700BF30BF00203B
:1086600032BF00202CC8002078BF0020436872224F
:108670001A70436873225A70436874229A70436870
:108680000022DA7070470F4B4268B3F904300A21B8
:1086900093FBF1F31B0110B503F5B9530A4C4FF4EA
:1086A000B4711433B3FBF1F303F00F031919E3585A
:1086B00013604B6853600B7A1372436800225A723E
:1086C00010BD00BF78BF00205CE90708044B93F899
:1086D000C53013F0FD0F14BF9E209D20704700BFD2
:1086E0002CC80020094B93F8C53013F0FD0F06D1BC
:1086F00042F210735843064B90FBF3F0704724236B
:1087000058434FF47A7390FBF3F070472CC8002065
:1087100040D20600064B07EE900A93F8C530B8EE3B
:10872000E70A1BB9DFED037A20EE270A704700BF86
:108730002CC8002048F9514010B5104B93F82C215B
:10874000012A10D1D3F83021811A00290BDD022132
:10875000B3F8264183F82C110949B1FBF4F142B179
:108760000A44C3F8302193F82C01013818BF0120C6
:1087700010BD0844C3F83001F5E700BF2CC8002045
:1087800040420F00831E00F17A02EA2123F8021F03
:108790009342FBD14E2243F64913C280CE22438539
:1087A0000281CD2323228380A0F87220A0F87830A4
:1087B000704700BF08BB1F48B0F8343103F0010315
:1087C0006BBB30B490F83841ACB11B4A02F1F005F4
:1087D00002E00133A3420ED052F8041B4904F8D53D
:1087E00090F8241200EB8101D1F8BC1145F8231058
:1087F0000133A342F0D130BC70470E48B0F83421A9
:10880000032A4FEA52030BD90A68A0F8343102F563
:10881000C332A03203F001030A60002BD1D07047AD
:108820000B6803F5C333A03348F205020B60A0F8D0
:10883000342170472CC8002068C900202DE9F04180
:1088400000283AD12D4A92F8380180B32C4A2D4B9A
:1088500092F804E092F905C092F90680CEF1FF0784
:10886000AEF17F06FFB2F6B203EB800003F1F00237
:10887000002403E0834202F1040218D053F8041BE1
:108880008904F7D5E1B2A1EB0C0181EAE175A5EB12
:10889000E175012D0DDC71B1414514BF39463146FA
:1088A0008342D17004F1010402F10402E6D1BDE873
:1088B000F0810821F4E77146F2E7114B1A79F02AAA
:1088C00009D802F10F000D4A18710B6803F58243B5
:1088D0001A330B60B7E7094A93F9054092F83A0159
:1088E0007F2584421D71987905DB4042C0B29871A2
:1088F00020445871E9E7002CFADAF6E72CC800208A
:108900009406002068C90020F0B5384E78B196F87A
:10891000AC32002B46D0364A013BDBB286F8AC3293
:108920001378DC0741D4334B0A681A440A6096F87E
:1089300038414CB3304B2E4F03EB840403F1F0016C
:10894000002503E09C4201F104011DD053F8042BE3
:10895000C2F303200628F5D13878C00715D596F85C
:10896000AC0296F83BE100EB050CBCFBFEF00EFB05
:1089700010C00128CCBF0020012058B99C4205F14D
:10898000010501F10401E1D1F0BDE84300F001006F
:108990000028F3D0C2F3834206EB8202D2F8BC2156
:1089A0000A60EBE796F83B31B5E7144A144BD2ED79
:1089B000037A144CFDEEE77A642017EE902AA2F5B4
:1089C0007A7200FB02F283FB0230D317C3EBA013D1
:1089D00003EB4303C3EB031384FB0302DB17C3EB7B
:1089E00062130533084A92FBF3F39DE72CC800207D
:1089F000A0BE0020400D030068C90020486D002083
:108A0000D34D62101F85EB5140420F00F0B4524C21
:108A1000002868D194F8AD02002856D04F4BD3ED12
:108A2000007AB3EE097AF4EEC77AF1EE10FA4EDC72
:108A3000BBEE097AF4EEC77AF1EE10FA4CBF0827C4
:108A40000027D3ED017AB3EE097AF4EEC77AF1EE9E
:108A500010FA3EDD47F0010794F83851ADB3404AB3
:108A6000DFF808C102EB850502F1F00014E094F98B
:108A7000B062B142ACBF0221002194F9B162B342AD
:108A80001CDB41F004010F421CBFDCF80C3003601A
:108A9000954200F1040018D052F8043BD903F7D5F1
:108AA00094F9AF6203F00F01B142C3F30313DEDCAC
:108AB00094F9B162B3424FF00101E2DA94F9B26283
:108AC000B342D8BF41F00801DDE7F0BC704704278E
:108AD000B7E7BBEE097AF4EEC77AF1EE10FA48BFB9
:108AE00047F00207B8E794F8AE3263B31B4B1D4D55
:108AF000D3ED007A93ED017A0A6894F8AD02F0EEB6
:108B0000E77AB0EEC77AF4EEC77AF1EE10FAB8BFA2
:108B1000F0EE477AFDEEE77A80F0010017EE903A2A
:108B2000193B03EB4303C3EB031385FB0365DB171F
:108B3000C3EBE51305330C4DB5FBF3F31A440A60A0
:108B400084F8AD0268E70B6894F8AD0203F543338F
:108B500003F5A0730B605FE72CC800203CBF00202A
:108B600068C90020353AFC4440420F000C4A07080F
:108B7000F0B40B4F97F8386186B107F59E72054641
:108B800007F50B77002352F8044B35EA040004BFC5
:108B9000086847F823000133B342F4D1F0BC7047B2
:108BA0002CC8002030B42A4B60B92A48027DCAB9CB
:108BB00093F825322849203301EB830130BC4FF470
:108BC000A060D5E793F8B322F2B1013A214883F8C7
:108BD000B3220A6802F5C32202F520720A60027D00
:108BE000002AE5D01D4A12689106E1D51C4A93F887
:108BF000B312127892071AD511BB93F8273216498F
:108C0000203301EB8301D9E7124893F8B442057D84
:108C1000A54205D8042483F8B42283F8B342D8E7E8
:108C20000134012283F8B44283F8B322D1E700294A
:108C3000BED193F826320849203301EB8301BDE70A
:108C400093F823320449203301EB8301B6E700BFD8
:108C50002CC80020846C002068C9002068BE002059
:108C600030BF002010B41E4A48B91E4C92F8B5021D
:108C70000B6823440B6098B15DF8044B704792F881
:108C8000B63203B3012B16D092F8B5020B68164C1E
:108C900080F00100234482F8B5020B600028EBD17C
:108CA00092F8233211495DF8044B203301EB830124
:108CB0004FF440705CE792F8B5020D4C80F0010073
:108CC00082F8B502D4E70B685DF8044B03F5742312
:108CD00003F5107301200B6082F8B502704700BFE6
:108CE0002CC8002040420F0048E8010068C900205D
:108CF00020A107003C4AA0B992F8B7326BB192F8B4
:108D0000B8128A081341DB070AD501F00101032AD2
:108D100006D8DFE802F05048403892F8BA3253BB28
:108D2000704792F8B832013303F00F0382F8B8327B
:108D30003BB192F8B732086800F5C330A030086044
:108D4000DCE72A4882F8B732437A002B44D128481E
:108D5000C07818B143F0040382F8B7322548007890
:108D6000C00730D592F8B9020028E4D043F00803D8
:108D700082F8B732DFE792F8C6321F4901EB830170
:108D80004FF40030F4E61C4B03F13002002914BF0D
:108D900019461146F4E7194B03F1180200290CBFDC
:108DA00019461146ECE7144B03F10802002914BFE1
:108DB00019461146E4E7104B03F11802002914BFCD
:108DC00019461146DCE70E4800680028CAD043F077
:108DD000010382F8B732C5E792F8B632002BB6D05D
:108DE000022382F8B732B2E72CC800204CBF002023
:108DF000A4BE0020A0BE00200C4A07081C4A070899
:108E000064C3002030B4022340F203154FF4FA7417
:108E1000322146F20142C37000238580C480018163
:108E200030BC42810380704770B40B4C0B490C4B33
:108E300022680E680D6883F8E002002122F020020B
:108E400083F8E412C3F8D062C3F8DC522260C3F89E
:108E5000D81270BC704700BF68BE0020A42F00204D
:108E60002CC8002090F8603043B9426901210720E6
:108E700082F84430A2F8460082F848107047044B4C
:108E80000449B3F908304068012247F093BA00BFA3
:108E9000940600208AE10708064B07491A88074B09
:108EA00040681B68534342F2107293FBF2F247F0A2
:108EB00081BA00BF34BF002036E2070868BF002037
:108EC000044A05495378127840680133013247F06B
:108ED00071BA00BF1CC400203BE207080B4B40687E
:108EE000B3F904300A2293FBF2F31A0102F5B952E6
:108EF0004FF4B4711432B2FBF1F2C2F1080202F085
:108F00000F020349603247F055BA00BF78BF002016
:108F100041E20708034A044992684068072347F082
:108F200049BA00BF68BF002048E2070807B5144AE5
:108F3000406892F8E812B2F8EA32012909D10093A8
:108F400092F8EC320F497B2247F034FA03B05DF817
:108F500004FB022906D10C497B2203B05DF804EB27
:108F600047F028BA0A22534340F2FF32B3FBF2F330
:108F70009BB2092B054928BF09237B22EDE700BFDF
:108F80002CC800204EE207085DE3070858E20708F6
:108F900013B54468FFF79AFB0F4B1B789B070246FB
:108FA00012D50E4B93F8F7120D4B59B19889FFF774
:108FB00099FB0C49009203467022204647F0FAF9CB
:108FC00002B010BDD889F2E7009007492D23702226
:108FD000204647F0EFF9F3E730BF00202CC800200F
:108FE000846C002037E307085EE20708034B04495E
:108FF000D3F8FC22406847F0DDB900BF2CC8002040
:1090000065E20708044B1B78DB0703D4034940687B
:1090100047F0D0B9704700BFA0BE002069E2070842
:1090200007B5094A0949B2F906300193B2F904308B
:109030000093B2F902304068B2F9002047F0BAF963
:1090400003B05DF804FB00BFC859002072E20708B6
:10905000084BD3F80C23002A0ADD074B03EB8203ED
:109060005A6B2AB1054B0649DB68406847F0A2B944
:10907000704700BF2CC800200C4A07089406002047
:1090800086E207081FB5938802939378019353787B
:10909000009313780A46034947F08CF905B05DF850
:1090A00004FB00BF8EE20708024B03491A684068C0
:1090B0001432E7E76CC30020A1E20708024B034922
:1090C0001A6840680832DDE76CC30020A5E2070893
:1090D000024B03491A6840680E32D3E76CC3002084
:1090E000A9E20708044B93F829310BB127F03CBCE7
:1090F000024B1888704700BF2CC8002034BF0020E6
:1091000010B5184CA379CBB194F82230DFED166A74
:1091100007EE903AF8EEE77A144B86EEA77AC0B2E3
:1091200003EB8000838907EE903AF8EEE77A67EE6A
:10913000277AFDEEE77A17EE900A10BD0C4B1B68FC
:1091400013F000630CD0C0B2FCF724FE80896423C6
:1091500010FB03F094F822305B0890FBF3F0ECE78F
:109160001846EAE74C300020000048435C2F00100E
:10917000F46B002008B5FFF7C3FF3C2390FBF3F02E
:1091800008BD074B93ED6E7AD3ED6B7AB4EEE77AB8
:10919000F1EE10FA03DD034940685BF05ABA7047FC
:1091A000C0140010EEEA070810B50C4698B9174A2B
:1091B000174892F8101323680344236001B110BDCF
:1091C00092F8233213492033BDE8104001EB8301AC
:1091D0004FF48060CCE414F00BFD32280ADD2368E4
:1091E0000A4A03F5742303F510730121236082F802
:1091F000101310BD054A92F81013142881F00101D4
:10920000CCBF0548054882F81013D4E72CC80020CD
:1092100040420F0068C9002020A1070048E8010073
:1092200010B5044624F078FD034903460422606823
:10923000BDE8104047F0BEB88AE10708224B1B8802
:109240005A0510B5446805D520462049BDE81040B0
:109250005BF0FFB9180505D520461D49BDE8104053
:109260005BF0F7B9590605D520461A49BDE810400C
:109270005BF0EFB9DA0705D520461749BDE8104085
:109280005BF0E7B99B0705D520461449BDE81040BF
:109290005BF0DFB925201FF0CDF828B1204610493A
:1092A000BDE810405BF0D5B90E4B1B782BB12046C2
:1092B0000D49BDE810405BF0CCB920460B49BDE834
:1092C00010405BF0C6B900BF74BF0020ADE20708D4
:1092D000B2E20708B7E20708BCE20708C1E20708E4
:1092E000C6E207082CC40020CBE20708D0E207083A
:1092F000032811D8DFE800F00A0C0206074BD3F868
:1093000018037047064B1B78DB0701D434F05EB9B5
:10931000024BD3F814037047002070472CC800207C
:10932000A0BE002037B504462A4800EB4303B3F83B
:10933000C65005F00F0049B1022804F101011DD803
:10934000002814BF9C239B2323700C460AB3C5F34B
:109350000315FFF7CDFF3C21012D1F4BB0FBF3F3AD
:10936000B3FBF1F201FB123315D0022D23D01B49C0
:10937000204603B0BDE8304047F01CB8032806D1B2
:10938000174B1B7803F00103653BDBB2DCE72023BE
:10939000DAE71546DDE7642542F21071B0FBF1F122
:1093A000B1FBF5F005FB101000900E49204647F088
:1093B00001F803B030BD0A250B49B0FBF1F1B1FB58
:1093C000F5F005FB101000900849204646F0F2FF2A
:1093D000EFE700BF2CC8002040420F00D5E207088D
:1093E000A0BE0020DFE20708A0860100EEE2070829
:1093F000037840680122053B114693E7F0B52B4BFB
:109400002B4E1C68317887B0074620460AF004FAD4
:109410007178054620460AF0EBF900220592B278F1
:109420008DF8132003466CB1039005A920460AF07D
:1094300005FA327A039B2AB10DF1130120460AF096
:1094400003FA039B9DF81310ECB1E1B1194A1268BD
:10945000914218DC184A02EB8102D2F84043039390
:1094600026201EF0E7FF0599039B70B911F0010F4C
:1094700014BF502200228907786808D50F4946F0AA
:1094800099FF07B0F0BD0E4CE9E74422F3E732B193
:10949000CDE900420B492A4646F08CFFF1E70A4924
:1094A00000942A4646F086FFEBE700BF04BF002089
:1094B000986D002010B900202CC80020FDE207089C
:1094C000BEEC070805E3070811E30708F8B50446F2
:1094D0002D4B4178827893F8E10023780138302BC6
:1094E0002A4B4FEA8000034429480BBF93F8BC5035
:1094F00093F8BE5093F8BD6093F8BF6000EB85050C
:10950000D5ED007AFDEEE77A00EB860017EE903A93
:10951000D0ED007A40F2CF75FDEEE77AAB4217EE60
:10952000900AA8BF2B46B3F57A7FB8BF4FF47A7381
:10953000A8424FF47A77A8BF2846A3F57A73B842B9
:10954000C3EB0313B3FBF7F3C3F10E03B8BF384605
:10955000DBB24FF0030CB3FBFCFC0CEB4C0EA3EBAB
:109560000E03A0F57A706244C0EBC0000833B0FB74
:10957000F7F73944DBB2D2B2C9B22046F5F7B6FAF2
:1095800000232373F8BD00BF2CC800200C4A070835
:10959000486D00202DE9F04790F8029090F8018086
:1095A00009F1020704460026FFB2002508EB060A6F
:1095B000032E1BD108F10301022DC9B20ED10B23DA
:1095C0003A462046F5F792FA0135052DF0D10136DD
:1095D000072EEAD100232373BDE8F08709EB0502CB
:1095E0001623D2B22046F5F781FAEDE7022DEBD132
:1095F00017233A465FFA8AF12046F5F777FAE3E750
:1096000070B504466FF00205A278617852FA85F2CF
:1096100007391323D2B2C9B22046F5F767FAA27808
:109620006178EEB2324407311323D2B2C9B2204678
:109630000135F5F75BFA042DE6D16178A278063999
:109640000323C9B22046F5F751FA6178A2780631B2
:109650000223C9B22046F5F749FA0023237370BDEF
:109660002DE9F8432B49054691F8D03091F8D120E7
:10967000294891F8DF10B0F90040002902EB82027E
:1096800014BF4FF0FF31012152004C43C2F10008DA
:1096900003EB830344454FEA430303DB9442A8BF33
:1096A0001446A046B0F902205C424A43A24203DBC2
:1096B0009A42A8BF1A4614461BB11922544394FB80
:1096C000F3F4293C4FEA88066FF003074FF00909CD
:1096D000002E3346B8BF06F13F03C4EBA313512B52
:1096E0000FD893FBF9F101EBC1029B1AAA780A4447
:1096F0006978803B3944DBB2D2B2C9B22846F5F76B
:10970000F5F90137052FA6EB0806E1D100232B73ED
:10971000BDE8F8832CC8002078BF002010B50446AF
:1097200014F0A2FA642202FB00F3C3F38F23632B2D
:1097300060680449BDE8104028BF6323012246F059
:1097400039BE00BF5DE307081D4B1E499A68B1F89A
:10975000C0309FED1D7A406807EE902AF8EEE76A68
:1097600007EE903AF8EEE77A67EE877AF4EEE76A6A
:10977000F1EE10FA02D8154946F01CBE934202DA07
:10978000134946F017BE9B1A07EE903AB8EEE77AF7
:10979000D1EDC57A0F4AF8EE677A3C2167EE277A59
:1097A00087EEA67AFDEEC77A17EE903AB3FBF2F396
:1097B000B3FBF1F201FB1233074946F0FBBD00BFDA
:1097C00068BF00202CC80020CDCCCC3D1AE3070890
:1097D00020E3070840420F00D5E20708244A00238F
:1097E0004361D2F8D41041F45C5130B541F02C0102
:1097F0000124C2F8D4104471D2F8CC1004FA03F555
:109800000133112B41EA0501F8D121F4F0314FF475
:109810002063C2F8CC10C38040F601230381154BAE
:109820000360142303718023037642F6140350224D
:10983000114903824FF6FF734383A0F8562003F5C6
:109840008C036FF07E42C0E91612C3610B4A40F2EE
:10985000012303844FF0A0640023C0E9184280F87C
:10986000223080F8333080F84430A0F8683030BDC2
:109870002CC8002098086400C4FF00FF180B0C00DF
:109880002DE9F84305461CF099FB1D4EDFF8749056
:10989000074600244FF0880833786968A3422144C2
:1098A00003DC00230B70BDE8F88337B3D6ED427AB2
:1098B000FDEEE77A09EB840317EE900AD3ED007A08
:1098C000FDEEE77A17EE902AD6ED437AFDEEE77AC1
:1098D000121A17EE903AD2001B1A92FBF3F3C3F15F
:1098E00088030B702046FFF70BFCB0F57A7F02DA95
:1098F0006B6853221A550134CEE781F80080FAE7ED
:1099000080060010E02F001013B5374BC1789A681D
:10991000364B02299B89044641D0032945D00129B1
:1099200005D19A1A9A42A8BF1A4622EAE272D3B126
:109930009A1A9A42A8BF1A4622EAE27207EE902AC1
:109940000B20B3FBF0F307EE103AF8EEE77AB8EE2F
:10995000C70A87EE800A59F0C5FAFCEEC07ACDED51
:10996000017A9DF8043062688A21117001226168D1
:109970009342ACBF8B208D20885401320C2AF6D143
:1099800062688F2111735A1E092A03D86268134432
:109990008E225A70636800225A7302B010BD9A1A60
:1099A0009A42A8BF1A4622EAE272ABB107EE902AA9
:1099B000B8EEE70ADFED0E7A20EE270A07EE903ABE
:1099C000F8EEE77A80EE270A59F01AFB642803467E
:1099D000A8BF642323EAE37306496068072202B044
:1099E000BDE8104046F0E6BC68BF00204CBF002038
:1099F0000000C84226E30708084B93F8C53007EE7D
:109A0000900A4BB9F8EEE77A9FED057A9FED050ACB
:109A1000A7EE870A59F0F4BA704700BF2CC800209F
:109A20006766E63F000000420D4B1B681B0137B51F
:109A300014D50C4C4568D4F8643393F90100FFF752
:109A4000DBFF94F8C5200849002A0CBF0D220E2226
:109A50000346009228467A2246F0ACFC03B030BDA3
:109A6000F46B00202CC800202DE307080B4B13B526
